:100000000C9426100C94C6360C949B360C947036C7
:100010000C9445360C941A360C94EF350C94C43578
:100020000C9499350C9457100C9457100C9457104D
:100030000C9457100C944A370C9457100C9457108A
:100040000C9457100C94F3830C9457100C94571085
:100050000C9457100C9457100C94E03E0C94943967
:100060000C9457100C94AC950C9481960C945710EA
:100070000C9457100C9457100C9457100C94571064
:100080000C9457100C9457100C9457100C94571054
:100090000C9457100C9457100C9457100C94571044
:1000A0000C9457100C9457100C9457100C94571034
:1000B0000C9457100C9457100C9457100C94571024
:1000C0000C9457100C9457100C9457100C94571014
:1000D0000C9457100C9457100C9457100C94571004
:1000E0000C945710262E292E182E1C2E222E602EF0
:1000F0002D2E312E372E3B2E3F2E452E492E4D2EA6
:10010000602E532E572E5B2E0F3814381938233893
:100110002D38A63837383F38473851385B3865387E
:1001200074387E38A638883892389C38DB95E1954B
:10013000F295FD9505961B9609961B960D961196C0
:100140001B9617968BA58BA592A592A592A599A50E
:1001500099A599A5A6A5A0A5A0A5A0A5084AD73BA5
:100160003BCE016E84BCBFFDC12F3D6C74319ABD86
:1001700056833DDA3D00C77F11BED9E4BB4C3E91AA
:100180006BAAAABE000000803F05A84CCDB2D44E99
:10019000B93836A9020C50B9918688083CA6AAAA9B
:1001A0002ABE000000803F004E414E494E4954593E
:1001B000494E46CDCCCC3D0AD7233C17B7D1387732
:1001C000CC2B329595E6241FB14F0A000020410048
:1001D00000C84200401C4620BCBE4CCA1B0E5AAE92
:1001E000C59D74434F4D4D554E49434154494F4E63
:1001F0000044525952554E004552524F52530049F5
:100200004E464F004543484F0047322F4733206248
:10021000616420706172616D65746572730A00506B
:10022000726F62696E67206661696C6564004D314A
:10023000313720426564206C6576656C696E672095
:100240006661696C65642E0A4730205A31300A476E
:10025000302045300A4D333030205032352053386D
:1002600038300A4D333030205035302053300A4D6D
:100270003330302050323520533838300A4D333047
:1002800030205035302053300A4D3330302050323A
:100290003520533838300A4734205331004D31313E
:1002A000372050726F626520737563636573736680
:1002B000756C0A0050524F4245204641494C20433C
:1002C0004C45414E204E4F5A5A4C450A004D313054
:1002D0003420533137300A4D313137205265776938
:1002E00070696E67206E6F7A7A6C650A4D313231B3
:1002F0000A4730205A31300A4732382058302059C6
:10030000300A4D313137205265776970696E672048
:100310006E6F7A7A6C650A47313220503020533143
:10032000322054300A4D3132300A4D3131372050AD
:10033000726F62696E672062656400205A3A20001D
:1003400020593A200042656420583A2000507269D2
:100350006E742074696D653A2000000125301D0C13
:100360001E2829FF24311C0B184527FF232F1B0AA9
:10037000174443FFFFFFFF040806FF06222B1A4124
:1003800042FF043803FF3646696C616D656E742068
:10039000757365643A200053746174733A20002CBD
:1003A000204C6F6E67657374206A6F623A20005448
:1003B0006F74616C2074696D653A200053746174C8
:1003C000733A20002C204661696C65643A20002C49
:1003D0002046696E69736865643A20005072696EE0
:1003E00074733A200053746174733A20000402FF5E
:1003F00001F801F101E3016F66660044454255478B
:100400003A004D3131332053006F6B0020573A00D2
:1004100020573A002F2F20007A5F6D61783A200034
:100420007A5F6D696E3A2000795F6D61783A2000DD
:10043000795F6D696E3A2000785F6D61783A2000CF
:10044000785F6D696E3A20005265706F7274696EE4
:100450006720656E6473746F702073746174757354
:100460000A00205400205200416363656C6572618C
:1004700074696F6E3A2050004B64200023646566F7
:10048000696E652044454641554C545F004B6920D8
:100490000023646566696E652044454641554C54A9
:1004A0005F004B70200023646566696E65204445DB
:1004B0004641554C545F00504944204175746F7457
:1004C000756E652066696E69736865642120507574
:1004D0007420746865206C617374204B702C204B01
:1004E0006920616E64204B6420636F6E7374616E6B
:1004F00074732066726F6D2062656C6F7720696E11
:10050000746F20436F6E66696775726174696F6E90
:100510002E680A00504944204175746F74756E65E9
:10052000206661696C6564212074696D656F7574FE
:100530000A00453120544845524D414C2052554EF9
:10054000415741590042454420544845524D414C81
:100550002052554E4157415900546865726D616C87
:100560002052756E6177617900453120486561746C
:10057000696E67206661696C656400426564206825
:10058000656174696E67206661696C6564004865C1
:100590006174696E67206661696C656400504944E6
:1005A000204175746F74756E65206661696C656451
:1005B000212054656D706572617475726520746F69
:1005C0006F20686967680A00204B643A2000204B5E
:1005D000693A2000204B703A20000A20436C617376
:1005E00073696320504944200A002054753A200062
:1005F000204B753A2000206D61783A2000206D690B
:100600006E3A200020643A200020626961733A202B
:1006100000504944204175746F74756E65206661A1
:10062000696C656421204261642065787472756428
:100630006572206E756D6265720A005049442041F2
:1006400075746F74756E652073746172740A0042FC
:100650006564204C6576656C696E6720004661694B
:100660006C656420746F20656E61626C6520426504
:1006700064204C6576656C696E670A00426564208B
:100680004C6576656C20436F7272656374696F6E3A
:10069000204D61747269783A00454550524F4D20A3
:1006A0004F4B0A003A200050726F6265205A204F6B
:1006B0006666736574003F5A206F7574206F6620FC
:1006C00072616E676520282D3220746F2035290AEB
:1006D000003F4B2076616C7565206F7574206F66E6
:1006E0002072616E67652028302D3130292E0A0076
:1006F000416476616E6365204B3D004163746976A9
:10070000652045787472756465723A2000496E768A
:10071000616C69642065787472756465720A0000A2
:100720000020002300260029002C002F00320000AA
:100730000100000301060109010225697300256912
:100740006D20256973002569682025696D2025695C
:100750007300256964202569682025696D20256955
:100760007300256979202569642025696820256939
:100770006D2025697300486F6D696E672066616939
:100780006C656400656E7175657565696E672022BC
:10079000004C696E65204E756D626572206973202C
:1007A0006E6F74204C617374204C696E65204E75B9
:1007B0006D6265722B312C204C617374204C696E14
:1007C000653A20005072696E7465722073746F70A0
:1007D0007065642064756520746F206572726F7235
:1007E000732E2046697820746865206572726F7276
:1007F00020616E6420757365204D39393920746F1E
:1008000020726573746172742E202854656D706552
:100810007261747572652069732072657365742ED8
:100820002053657420697420616674657220726556
:100830007374617274696E67290A004E6F20436891
:1008400065636B73756D2077697468206C696E657C
:10085000206E756D6265722C204C617374204C693A
:100860006E653A2000636865636B73756D206D6912
:10087000736D617463682C204C617374204C696ED5
:10088000653A20004D3131300020496E76616C6947
:10089000642065787472756465722000000040C041
:1008A0000000E0C0000000C000002243CDCC364371
:1008B00000001F432066697273740A005A005900D1
:1008C0005800486F6D6520001000C90210012C010E
:1008D0004001220170011801B0010E01F001040174
:1008E0005002FA00B002F0003003E600D003DC0052
:1008F0009004D2007005C800A006BE000008B40035
:10090000B009AA00D00BA000600E960060118C0008
:100910000015820020197800C01D6E00A02264001E
:10092000B0275A00902C500000314600E0343C00C3
:1009300010383200903A2800603C1E00A03D1400A0
:10094000803E0A00203F00006265640A002C20738C
:10095000797374656D2073746F70706564212048BD
:1009600065617465725F49443A200042656420689D
:10097000656174696E67206661696C6564004865CD
:100980006174696E67206661696C65640045312039
:1009900048656174696E67206661696C65640048CA
:1009A000656174696E67206661696C6564004B49B6
:1009B0004C4C45442E20001000AD0330016A01501C
:1009C000022B0170030A019004F500B005E500D088
:1009D00006D800F007CE001009C500300ABE00504E
:1009E0000BB700700CB100900DAB00B00EA600D09C
:1009F0000FA200F0109D00101299003013950050C6
:100A000014920070158E0090168B00B0178700D0DE
:100A1000188400F0198100101B7E00301C7B0050F0
:100A20001D7900701E7600901F7300B0207000D0FA
:100A3000216E00F0226B0010246900302566005002
:100A40002663007027610090285E00B0295C00D00A
:100A50002A5900F02B5600102D5400302E51005012
:100A60002F4E0070304B0090314800B0324500D01E
:100A7000334200F0343E0010363B00303737005030
:100A800038330070392E00903A2900B03B2300D053
:100A90003C1B00F03D1100103F0100F03F000045FD
:100AA00031204572723A204D415854454D50004511
:100AB00072723A204D415854454D502042454400F1
:100AC0004D415854454D5020747269676765726591
:100AD00064004531204572723A204D494E54454DCF
:100AE00050004572723A204D494E54454D502042B7
:100AF0004544004D494E54454D5020747269676716
:100B00006572656400202F002042403A0020403A80
:100B1000000A0A426564204C6576656C20436F725A
:100B200072656374696F6E204D61747269783A0002
:100B3000202B000A436F72726563746564204265FE
:100B400064204865696768742076732E2042656466
:100B500020546F706F6C6F67793A0A00202B000A7F
:100B60004265642048656967687420546F706F67D8
:100B700072617068793A0A2020202B2D2D2D204299
:100B800041434B202D2D2B0A2020207C202020208B
:100B9000202020202020207C0A204C207C20202087
:100BA00020282B29202020207C20520A2045207C30
:100BB00020202020202020202020207C20490A20C6
:100BC00046207C20282D29204E20282B29207C20DF
:100BD000470A2054207C2020202020202020202074
:100BE000207C20480A2020207C20202020282D291D
:100BF000202020207C20540A2020207C202020201F
:100C0000202020202020207C0A2020204F2D2D2055
:100C100046524F4E54202D2D2B0A2028302C30299F
:100C20000A004D65616E206F662073616D706C65A2
:100C30006420706F696E74733A200020643A20005B
:100C400020623A200045716E20636F6566666963B5
:100C500069656E74733A20613A20003474682070BC
:100C6000726F626520706F696E742C206469737492
:100C7000616E63652066726F6D20706C616E653A9F
:100C80002000202844525952554E2900473239201D
:100C90004175746F20426564204C6576656C696EA1
:100CA00067003F20284C2C522C462C4229206F757F
:100CB00074206F6620626F756E64732E0A003F5059
:100CC000726F626520706F696E74732028592920D5
:100CD000697320696D706C61757369626C65202839
:100CE000322D32292E0A003F50726F626520706FDC
:100CF000696E74732028582920697320696D706C9F
:100D000061757369626C652028322D32292E0A00C4
:100D10003F2856296572626F7365206C6576656C35
:100D200020697320696D706C61757369626C6520F0
:100D300028302D34292E0A0050726F746563746553
:100D4000642050696E0A00205A3A0020593A002067
:100D5000436F756E7420583A0020453A00205A3A85
:100D60000020593A00583A003A004361703A005462
:100D70004845524D414C5F50524F54454354494FA2
:100D80004E004155544F5245504F52545F53445FAB
:100D900053544154555300454D455247454E4359D0
:100DA0005F50415253455200434153455F4C4947C0
:100DB00048545F4252494748544E45535300544F9C
:100DC00047474C455F4C494748545300534F46549E
:100DD000574152455F504F574552004255494C4488
:100DE0005F50455243454E54004C4556454C494E84
:100DF000475F44415441005A5F50524F42450041C1
:100E000055544F4C4556454C005052494E545F4A3C
:100E10004F420050524F4752455353004155544F93
:100E20005245504F52545F54454D5000564F4C550B
:100E30004D455452494300454550524F4D0053458E
:100E40005249414C5F584F4E5F584F464600464905
:100E5000524D574152455F4E414D453A4D61726C7E
:100E6000696E20204649524D574152455F564552C2
:100E700053494F4E3A312E312E392E3238204558B3
:100E80005452554445525F545950453A53696E6720
:100E90006C6545787472756465724165726F56321F
:100EA00020534F555243455F434F44455F55524C85
:100EB0003A68747470733A2F2F636F64652E616C97
:100EC0006570686F626A656374732E636F6D2F64FB
:100ED0006966667573696F6E2F4D41524C494E209D
:100EE00050524F544F434F4C5F56455253494F4E0B
:100EF0003A312E30204D414348494E455F545950B8
:100F0000453A4C756C7A426F74204D696E69204584
:100F1000585452554445525F434F554E543A312030
:100F2000555549443A33353134383762362D63618B
:100F300039612D346331612D383736352D643636BD
:100F40003862316461363538350A00205A0020593C
:100F500000580020204D61783A2000205A00205986
:100F600000580020204D696E3A20004F6E20004F3F
:100F7000666600536F667420656E6473746F707379
:100F80003A200020466C6F773A200020643A002017
:100F9000693A0020703A00496E76616C6964206598
:100FA000787472756465720A0020643A0020693AA8
:100FB0000020703A0043290A0061626C65642028B1
:100FC0006D696E2074656D702000436F6C642065E0
:100FD00078747275646573206172652000546F6F58
:100FE000206661722066726F6D207265666572653B
:100FF0006E636520706F696E740A004E6F206361C6
:101000007365206C696768740A0020746F6F206CC8
:101010006F6E6720657874727573696F6E20707279
:101020006576656E7465640A0020636F6C64206584
:101030007874727573696F6E2070726576656E7400
:1010400065640A002020506C616E6E6572427566A0
:1010500066657242797465733A2000204672656550
:10106000204D656D6F72793A2000436F6D70696C29
:1010700065643A204E6F7620203220323031380AB3
:1010800000207C20417574686F723A2028416C659D
:101090007068204F626A6563747320496E632E2CFA
:1010A000204C756C7A426F742047697420526570C9
:1010B0006F7369746F7279290A004E6F762020323F
:1010C000203230313831343A33343A303100204C28
:1010D00061737420557064617465643A2000312E28
:1010E000312E390A004D61726C696E0020536F66B3
:1010F00074776172652052657365740A00205761C8
:10110000746368646F672052657365740A002042D7
:10111000726F776E206F75742052657365740A0064
:101120002045787465726E616C2052657365740A2F
:1011300000506F77657255700A0073746172740A9B
:1011400000205A3A0020593A0020583A00656E644F
:1011500073746F7073206869743A2000454550526B
:101160004F4D206461746173697A65206572726F96
:10117000722E0A00290A002062797465733B20638D
:101180007263200053657474696E67732053746FC3
:10119000726564202800290A002062797465733B17
:1011A0002063726320002073746F7265642073651E
:1011B0007474696E677320726574726965766564AC
:1011C000202800202863616C63756C617465642954
:1011D000210A0020213D2000454550524F4D20431B
:1011E0005243206D69736D61746368202D202873EC
:1011F000746F7265642920002053697A653A200073
:10120000496E6465783A2000204D61726C696E3DCC
:10121000563535290A0028454550524F4D3D004569
:101220004550524F4D2076657273696F6E206D691F
:10123000736D61746368200024F4D43050C38E2031
:10124000C2A24017828B7011127A910D816CD90A5B
:10125000A861E108C7586607615143061E4B5D054A
:10126000C145A7041A411104093D9803713931039E
:101270004036DB0265339102D4305402802E1D02C9
:10128000632CEE01752AC501B028A0011027810149
:101290008F2564012B244B01E0223401AC211F0176
:1012A0008D200D01801FFC00841EED00971DDF00C6
:1012B000B81CD200E61BC600201BBC00641AB2009A
:1012C000B219A8000A19A0006A189900D117910054
:1012D00040178B00B516840031167E00B3157900D7
:1012E0003A157300C7146F0058146A00EE136600B5
:1012F0008813630025135E00C7125B006C12570051
:1013000015125400C111510070114F0021114B00F2
:10131000D61049008D1047004610440002104200CC
:10132000C00F4000800F3E00420F3C00060F3B0004
:10133000CB0E3800930E37005C0E3500270E3400BC
:10134000F30D3200C10D3100900D3000600D2E0004
:10135000320D2D00050D2C00D90C2B00AE0C2900F0
:10136000850C29005C0C2700350C27000E0C26008C
:10137000E80B2400C40B2400A00B23007D0B2300EA
:101380005A0B2100390B2100180B2000F80A1F000E
:10139000D90A1E00BB0A1E009D0A1D00800A1D00FE
:1013A000630A1C00470A1B002C0A1B00110A1A00C2
:1013B000F7091A00DD091900C4091900AB09190061
:1013C000920917007B091800630917004C091600E1
:1013D00036091600200916000A091500F50815003F
:1013E000E0081400CC081400B8081400A408140085
:1013F000900813007D0812006B08130058081200B3
:1014000046081200340811002308110012081100C8
:1014100001081100F0071000E0071000D0071000CD
:10142000C0071000B0070F00A107100091070E00C1
:1014300083070F0074070F0065070E0057070E00A3
:1014400049070E003B070D002E070E0020070D0078
:1014500013070D0006070D00F9060C00ED060D0040
:10146000E0060C00D4060C00C8060C00BC060C00FC
:10147000B0060C00A4060B0099060C008D060B00AC
:1014800082060B0077060B006C060B0061060A0053
:1014900057060B004C060A0042060A0038060A00EE
:1014A0002E060A0024060A001A060A001006090081
:1014B00007060A00FD050900F4050900EB0509000F
:1014C000E2050900D9050900D0050900C705090092
:1014D000BE050900B5050800AD050800A505090011
:1014E0009C050800940508008C0508008405080088
:1014F0007C050800740508006C05070065050800F8
:101500005D050700560508004E0507004705070062
:101510004005080038050700310507002A050700C7
:10152000230507001C050600160507000F05070028
:101530000805060002050700FB040600F504070085
:10154000EE040600E8040600E2040700DB040600DF
:10155000D5040600CF040600C9040600C304060033
:10156000BD040600B7040600B1040500AC04060083
:10157000A6040600A00405009B04060095040500CF
:10158000900406008A040500850405008004060016
:101590007A04050075040500700405006B0405005D
:1015A00066040500610405005C040500570405009D
:1015B000520405004D0405004804050043040500DD
:1015C0003E0404003A04050035040500300404001C
:1015D0002C04050027040400230405001E04040055
:1015E0001A04040016040500110404000D0404008C
:1015F000090405000404040000040400FC030400C2
:10160000F8030400F4030400F0030400EC030400F6
:10161000E8030400E4030400E0030400DC03040026
:10162000D8030400D4030400D0030400CC03040056
:10163000C8030300C503030024F404D9201BC40C11
:101640005C0E9804C4095F0265077101F405F90096
:10165000FB04B30048048700C10369005803550028
:1016600003034500BE023A008402310053022A00FF
:101670002902250004022000E4011C00C801190011
:10168000AF011700980114008401130071011000CC
:101690006101100051010E0043010D0036010B00E5
:1016A0002B010B0020010B00150109000C010900A2
:1016B00003010800FB000800F3000800EB0007002E
:1016C000E4000600DE000600D8000600D200060096
:1016D000CC000500C7000500C2000500BD000400E5
:1016E000B9000400B5000400B1000400AD0004001E
:1016F000A9000400A5000300A20003009F0004004D
:101700009B00030098000300950002009300030073
:10171000900003008D0002008B000300880002008F
:101720008600020084000300810002007F000200A6
:101730007D0002007B0002007900020077000100BA
:1017400076000200740002007200010071000200C5
:101750006F0002006D0001006C0002006A000100D1
:1017600069000200670001006600010065000100D9
:1017700064000200620001006100010060000100DD
:101780005F0002005D0001005C0001005B000100E1
:101790005A000100590001005800010057000100E3
:1017A00056000100550001005400010053000000E4
:1017B00053000100520001005100010050000100DF
:1017C0004F0001004E0000004E0001004D000100DE
:1017D0004C0001004B0000004B0001004A000100DA
:1017E00049000100480000004800010047000100D6
:1017F00046000000460001004500000045000100D1
:1018000044000100430000004300010042000000CA
:1018100042000100410000004100010040000100C1
:101820003F0000003F0001003E0000003E000100BC
:101830003D0000003D0001003C0000003C000000B5
:101840003C0001003B0000003B0001003A000000AA
:101850003A000100390000003900010038000000A2
:101860003800000038000100370000003700010098
:101870003600000036000000360001003500000090
:101880003500000035000100340000003400000085
:101890003400010033000000330000003300010079
:1018A0003200000032000000320001003100000070
:1018B0003100000031000100300000003000000065
:1018C000300001002F0000002F0000002F0000005A
:1018D0002F0001002E0000002E0000002E0001004D
:1018E0002D0000002D0000002D0000002D00010043
:1018F0002C0000002C0000002C0000002C00010037
:101900002B0000002B0000002B0000002B0001002A
:101910002A0000002A0000002A0000002A0001001E
:101920002900000029000000290000002900000013
:101930002900010028000000280000002800000005
:1019400028000000280001002700000027000000F8
:1019500027000000270000002700010026000000EB
:1019600026000000260000002600000026000100DE
:1019700025000000250000002500000025000000D3
:1019800025000000250001002400000024000000C4
:1019900024000000240000002400010023000000B7
:1019A00023000000230000002300000023000000AB
:1019B000230000002300010022000000220000009C
:1019C000220000002200000022000000220001008E
:1019D0002100000021000000210000002100000083
:1019E0002100000021000000210001002000000073
:1019F0002000000020000000200000002000000067
:101A00002000000020000000200001001F00000056
:101A10001F0000001F0000001F0000001F0000004A
:101A20001F0000001F0001001E0000001E0000003B
:101A30001E0000001E000000C23100001C26000035
:101A4000F4190000D80F0000EB080000C0040000EB
:101A50007502000040010000526573656E643A2013
:101A6000002042002050006F6B0020746F6F206CCC
:101A70006F6E6720657874727573696F6E2070720F
:101A80006576656E7465640A0020636F6C6420651A
:101A90007874727573696F6E2070726576656E7496
:101AA00065640A00627573793A20706175736564C4
:101AB00020666F7220696E7075740A0062757379A2
:101AC0003A2070617573656420666F722075736566
:101AD000720A00627573793A2070726F636573736E
:101AE000696E670A004B494C4C45442E20004B4917
:101AF0004C4C2063617573656420627920746F6F4C
:101B0000206D75636820696E616374697665207401
:101B1000696D65202D2063757272656E7420636F28
:101B20006D6D616E643A20005072696E746572204A
:101B300068616C7465642E206B696C6C2829206365
:101B4000616C6C6564210A00000040C0CDCC364356
:101B500000001F430000F0410000F0410000004180
:101B6000000000005761726E696E673A20486F6D21
:101B7000696E672042756D702044697669736F7273
:101B8000203C20310A000202040000A0400000A016
:101B9000400000004000002543CDCC3D4300002123
:101BA00043FF010148617264636F646564204465AA
:101BB0006661756C742053657474696E6773204C2C
:101BC0006F616465640A0028230000282300006414
:101BD000000000E803000000009643000096430068
:101BE000000041000020420000C9420000C942003C
:101BF00000C8440000D2433A0A0020286D6D290035
:101C0000204500205A0020204D39303720580053FD
:101C1000746570706572206D6F746F722063757279
:101C200072656E74733A0A0020204D393030204BB3
:101C3000004C696E65617220416476616E63653A3D
:101C40000A0020204D383531205A005A2D50726F2D
:101C50006265204F66667365740020440020490069
:101C600020204D33303420500020440020490020F3
:101C7000204D333031205000504944207365747436
:101C8000696E67733A0A0020204D343230205300C9
:101C90004175746F20426564204C6576656C696E91
:101CA000673A0A00205A0020590020204D32303671
:101CB000205800486F6D65206F66667365743A0A38
:101CC00000204500205A00205900205800205400D0
:101CD00020530020204D32303520420020453C6DFD
:101CE00061785F655F6A65726B3E0020583C6D618C
:101CF000785F785F6A65726B3E20593C6D61785FF2
:101D0000795F6A65726B3E205A3C6D61785F7A5FDD
:101D10006A65726B3E00416476616E6365643A2069
:101D2000423C6D696E5F7365676D656E745F746963
:101D30006D655F75733E20533C6D696E5F666565CA
:101D400064726174653E20543C6D696E5F747261AB
:101D500076656C5F66656564726174653E002054EB
:101D60000020520020204D32303420500041636367
:101D7000656C65726174696F6E2028756E69747325
:101D80002F7332293A20503C7072696E745F616320
:101D900063656C3E20523C726574726163745F616E
:101DA0006363656C3E20543C74726176656C5F6160
:101DB0006363656C3E0A00204500205A00205900EC
:101DC00020204D3230312058004D6178696D756D9D
:101DD00020416363656C65726174696F6E2028755C
:101DE0006E6974732F7332293A0A00204500205A15
:101DF0000020590020204D3230332058004D6178AA
:101E0000696D756D206665656472617465732028FF
:101E1000756E6974732F73293A0A00204500205AA1
:101E20000020590020204D3932205800537465702D
:101E3000732070657220756E69743A0A0020204D17
:101E40003230302044300A0020204D3230302044DF
:101E5000002044697361626C65640A0046696C61C4
:101E60006D656E742073657474696E67733A0020D3
:101E700020473231202020203B004D6963726F7370
:101E80007465707320756E617661696C61626C65F2
:101E90000A0045303A20005A3A2000593A200058AA
:101EA0003A20004D53312C4D53322050696E730A45
:101EB000004572726F722077726974696E67207460
:101EC0006F20454550524F4D210A00556E6B6E6F85
:101ED000776E20636F6D6D616E643A2022006563DA
:101EE000686F3A0000000A0B02090C0D0E08070388
:101EF00004010000000000000000000000000000DD
:101F000000000000000000000000000000000000D1
:101F1000121110000000000000000000000000008E
:101F20000000000000000000000050726F62696E47
:101F300067206661696C65640A00205A3A200020B7
:101F4000593A200042656420583A20004572726F69
:101F5000723A00453120544845524D414C2052556B
:101F60004E415741590042454420544845524D4145
:101F70004C2052554E4157415900546865726D616D
:101F80006C2052756E617761790000002200250097
:101F900028002B002E003100340002010000050152
:101FA00008010B0100002100240027002A002D0059
:101FB0003000330001010000040107010A0105059A
:101FC0000505070508080808020202020A0A0808AF
:101FD00004040404010101010101010103030303DD
:101FE00003030303040707070C0C0C0C0C0C0C0C6C
:101FF0000202020206060606060606060B0B0B0B7D
:102000000B0B0B0B010210202008081020401020A1
:1020100040800201020108040201010204081020AC
:1020200040808040201008040201800402018040AA
:102030002010080402010804020101020408102013
:10204000408001020408102040804CA111241FBED2
:10205000CFEFD1E2DEBFCDBF00E00CBF13E0A0E0C8
:10206000B2E0E6E3F3E601E00BBF02C007900D9299
:10207000A231B107D9F72EE0A2E1B3E001C01D9271
:10208000A63CB207E1F710E1C6E2D0E100E006C0ED
:1020900021970109802FFE010E9453B1C532D1075B
:1020A00080E00807A9F70E947A740C9499B10C9407
:1020B00000002F923F924F925F926F927F928F9289
:1020C0009F92AF92BF92CF92DF92EF92FF920F93C7
:1020D0001F93CF93DF93CDB7DEB7C559D1090FB6A4
:1020E000F894DEBF0FBECDBFC157DF4F8883CF58F6
:1020F000D04021E02093D30C8091F50D8D3411F464
:102100000C94FB1A843511F40C94AA28873411F02E
:102110000C94EE28E090F30DF090F40D3AE1E31604
:10212000F10409F440C7CCF454E0E516F1044CF492
:1021300082E0E816F1040CF062C0F7FE34C00C94A3
:10214000F71A94E0E916F10409F4FDC5ACE0EA16CB
:10215000F10409F4FCC50C94F71ABEE1EB16F10486
:1021600011F40C9466194CF4FCE1EF16F10409F437
:1021700051C70CF41CC70C942C193BE5E316F10471
:1021800011F40C94391A4CE5E416F10411F40C9492
:102190003D1A5AE5E516F10411F00C94F71A109265
:1021A00016030C94F02880911102882311F40C94EA
:1021B000F0288AE50E947233482F89E5CF56DF4F19
:1021C0004883C159D0400E947233682F88E5C057B8
:1021D000DF4F6883C059D0400E947233CF56DF4F23
:1021E0004881C159D040C057DF4F6881C059D040A5
:1021F0000E94102F81110C94F0280C94FD2841E0CE
:1022000061E081E00E94102F81110C94F0288091F0
:102210001102882311F40C94F02811E082E0E816F2
:10222000F10409F010E00E94A54782E50E94B9334D
:10223000882309F442C10E943F336B017C01209145
:10224000110E3091120E4091130E5091140E2EA7C4
:102250003FA748AB59AB8091150E9091160EA091F7
:10226000170EB091180E8AAB9BABACABBDAB2091F7
:10227000180D3091190D40911A0D50911B0D2EAB78
:102280003FAB48AF59AF80911C0D90911D0DA091AF
:102290001E0DB0911F0D8AAF9BAFACAFBDAF20E05C
:1022A00030E0A901C701B6010E9413AA882309F4EE
:1022B00030C52EA53FA548A959A96EA97FA988AD0B
:1022C00099AD0E9413AA81110DC02AA93BA94CA95E
:1022D0005DA96AAD7BAD8CAD9DAD0E9413AA88232C
:1022E00009F417C520E030E0A901C701B6010E943A
:1022F00013AA881F8827881F181307C0412C512C48
:1023000040E8642E4FE3742E06C0412C512C30E877
:10231000632E3FEB732E2EA53FA548A959A96EA9A0
:102320007FA988AD99AD0E9476AE26966CAF7DAF41
:102330008EAF9FAF26972AA93BA94CA95DA96AAD8C
:102340007BAD8CAD9DAD0E9476AE2A966CAF7DAF15
:102350008EAF9FAF2A9726962CAD3DAD4EAD5FADAB
:102360002697CA01B9010E9478AA4B015C012A96FE
:102370002CAD3DAD4EAD5FAD2A97CA01B9010E94AB
:1023800078AA9B01AC01C501B4010E9477AE0E94FE
:10239000E2B022966CAF7DAF8EAF9FAF229720E068
:1023A00030E040E05FE30E9478AA4B015C01A701A6
:1023B0009601C701B6010E9478AA6B017C01A501B4
:1023C0009401C501B4010E9478AA9B01AC01C70128
:1023D000B6010E9476AE0E94E2B09B01AC01C3013F
:1023E000B2010E9478AA2B013C012EA93FA948AD59
:1023F00059AD6EA57FA588A999A90E9477AE20E066
:1024000030E040E05FE30E9478AA6B017C012A96ED
:102410006CAD7DAD8EAD9FAD2A97905822962CADB8
:102420003DAD4EAD5FAD22970E9453AF9B01AC0115
:10243000C301B2010E9478AA9B01AC01C701B60199
:102440000E9477AE2EA53FA548A959A90E9476AE55
:102450006B017C012AAD3BAD4CAD5DAD6AA97BA99A
:102460008CA99DA90E9477AE20E030E040E05FE3B8
:102470000E9478AA4B015C0122962CAD3DAD4EAD79
:102480005FAD229726966CAD7DAD8EAD9FAD269744
:102490000E9453AF9B01AC01C301B2010E9478AA14
:1024A0009B01AC01C501B4010E9477AE2AA93BA9EA
:1024B0004CA95DA90E9476AE14C089E40E94B9338C
:1024C000882329F00E943F336B017C0103C0C12C9B
:1024D000D12C76018AE40E94B9338823D9F00E9476
:1024E0003F336EAB7FAB88AF99AF20E030E0A901FE
:1024F000C701B6010E9413AA81111AC020E030E082
:10250000A9016EA97FA988AD99AD0E9413AA811176
:102510000FC0FFC320E030E0A901C701B6010E944F
:1025200013AA882309F4F5C31EAA1FAA18AE19AE70
:10253000A701960150582EA73FA748AB59AB8EA9CB
:102540009FA9A8ADB9ADB0588AAB9BABACABBDAB46
:10255000CA01B9010E9478AA4B015C012AA93BA9D2
:102560004CA95DA9CA01B9010E9478AA9B01AC01DE
:10257000C501B4010E9477AE0E94E2B066966CAFCE
:102580007DAF8EAF9FAF66972091110E3091120EE6
:102590004091130E5091140E2AAF3BAF4CAF5DAF7C
:1025A000A70196016AAD7BAD8CAD9DAD0E9477AE63
:1025B0002A966CAF7DAF8EAF9FAF2A978091150E94
:1025C0009091160EA091170EB091180E22968CAF16
:1025D0009DAFAEAFBFAF22972EA93FA948AD59AD71
:1025E000BC01CD010E9477AE6A966CAF7DAF8EAF15
:1025F0009FAF6A972091180D3091190D40911A0DD7
:1026000050911B0D26962CAF3DAF4EAF5FAF269776
:102610002A962CAD3DAD4EAD5FAD2A9726966CAD9A
:102620007DAD8EAD9FAD26970E9476AE6B017C018D
:1026300080911C0D90911D0DA0911E0DB0911F0D4C
:102640002E968CAF9DAFAEAFBFAF2E976A962CADD6
:102650003DAD4EAD5FAD6A97BC01CD010E9476AE37
:102660004B015C012091190E30911A0E40911B0E06
:1026700050911C0E62962CAF3DAF4EAF5FAF62978C
:102680006091200D7091210D8091220D9091230D6C
:102690000E9476AE2B013C018091240D9091250D76
:1026A000A091260DB091270DA2968CAF9DAFAEAF35
:1026B000BFAFA29720911D0E30911E0E40911F0EAC
:1026C0005091200E6E962CAF3DAF4EAF5FAF6E9720
:1026D000A70196016EA57FA588A999A90E9478AA4D
:1026E000A6966CAF7DAF8EAF9FAFA697A501940164
:1026F0006AA97BA98CA99DA90E9478AA9B01AC011B
:10270000A6966CAD7DAD8EAD9FADA6970E9477AEBF
:10271000A6966CAF7DAF8EAF9FAFA697A501940133
:102720006EA57FA588A999A90E9478AA4B015C0192
:10273000A70196016AA97BA98CA99DA90E9478AAE4
:102740009B01AC01C501B4010E9476AEA6962CADEA
:102750003DAD4EAD5FADA6970E94EAAE6B017C0128
:1027600020E030E0A9010E9413AA87FF0AC02BEDE8
:102770003FE049EC50E4C701B6010E9477AE6B011F
:102780007C01112351F02BED3FE049EC50E4C701EF
:10279000B6010E9476AE6B017C0120E030E0A90119
:1027A000C701B6010E9413AA811126C026962CAD3E
:1027B0003DAD4EAD5FAD26976AAD7BAD8CAD9DADA9
:1027C0000E9413AA811118C02E962CAD3DAD4EADBE
:1027D0005FAD2E9722966CAD7DAD8EAD9FAD2297ED
:1027E0000E9413AA811108C02BEDC22E2FE0D22E19
:1027F00029ECE22E20E4F22EA701960166966CAD3C
:102800007DAD8EAD9FAD66970E9478AA4B015C01AD
:1028100020E030E0A901C301B2010E9413AA88237D
:10282000C9F0A5019401C501B4010E9478AA4B0129
:102830005C01A3019201C301B2010E9478AA9B012D
:10284000AC01C501B4010E9477AE0E94E2B04B0119
:102850005C010DC020E030E0A901C501B4010E9477
:102860009DB087FF04C0B7FAB094B7F8B0942FE6D4
:1028700032E143E85AE3C501B4010E9413AA87FF7D
:1028800002C00C94F028C501B4010E94ECAF0E9474
:10289000C0AF1B01672B19F422242394312CB10102
:1028A00080E090E00E9417AA4B015C019B01AC0103
:1028B000C701B6010E9453AF6AAF7BAF8CAF9DAF2B
:1028C000A5019401C301B2010E9453AF66966CAF9B
:1028D0007DAF8EAF9FAF66976E962CAD3DAD4EAD82
:1028E0005FAD6E97A2966CAD7DAD8EAD9FADA2979C
:1028F0000E9476AEA50194010E9453AFA2966CAFE0
:102900007DAF8EAF9FAFA2972AAD3BAD4CAD5DAD15
:10291000CA01B9010E9478AA20E030E040E05FE3FC
:102920000E9478AA9B01AC0160E070E080E89FE320
:102930000E9476AE2E966CAF7DAF8EAF9FAF2E9776
:1029400062968CAD9DADAEADBFAD629789879A871B
:10295000AB87BC876E962CAD3DAD4EAD5FAD6E972F
:102960002D873E874F87588B60914D0270914E02A4
:10297000072E000C880B990B0E9419AA209159026E
:1029800030915A0240915B0250915C020E9478AAF9
:102990002AE037ED43E25CE30E9478AA6AA77BA7AE
:1029A0008CA79DA70E94E9389B01AC0128533F4F9B
:1029B0004F4F5F4F62962CAF3DAF4EAF5FAF629708
:1029C0004EA45FA468A879A841E050E024965FAFC8
:1029D0004EAF249759E15EAF24962EAD3FAD2497BC
:1029E0002215330509F43AC10E942F420E94E938AA
:1029F000DC01CB0162962CAD3DAD4EAD5FAD629773
:102A0000821B930BA40BB50BB7FD10C00E94E938D5
:102A10009B01AC0128533F4F4F4F5F4F62962CAF45
:102A20003DAF4EAF5FAF62970E9487903EAD315091
:102A30003EAF332309F441C02E962CAD3DAD4EADD3
:102A40005FAD2E976AA97BA98CA99DA90E9478AA3F
:102A50006B017C012AAD3BAD4CAD5DADB201C30154
:102A60000E9478AAA70196010E9477AE7B018C0193
:102A70002E962CAD3DAD4EAD5FAD2E97B201C3018C
:102A80000E9478AA4B015C012AAD3BAD4CAD5DAD17
:102A90006AA97BA98CA99DA90E9478AA9B01AC0177
:102AA000C501B4010E9476AE2B013C01C701D801DB
:102AB0008AAB9BABACABBDAB53C024964EAD5FAD08
:102AC0002497BA0180E090E00E9417AA2AAD3BAD9E
:102AD0004CAD5DAD0E9478AA4B015C010E9450AFE5
:102AE0006B017C01C501B4010E94D8B04B015C01AF
:102AF000A70196016EA57FA588A999A90E9478AA29
:102B00002B013C01A50194016EA97FA988AD99AD67
:102B10000E9478AA9B01AC01C301B2010E9477AE6A
:102B20002B013C01A50194016EA57FA588A999A957
:102B30000E9478AA4B015C01A70196016EA97FA9AA
:102B400088AD99AD0E9478AA9B01AC01C501B40182
:102B50000E9476AE6AAB7BAB8CAB9DAB59E15EAFAE
:102B60009201A3012A966CAD7DAD8EAD9FAD2A97E3
:102B70000E9477AE69837A838B839C832AA93BA9C1
:102B80004CA95DA96A966CAD7DAD8EAD9FAD6A977F
:102B90000E9477AE6D837E838F83988766962CAD77
:102BA0003DAD4EAD5FAD669769857A858B859C8519
:102BB0000E9477AE69877A878B879C87A2962CAD17
:102BC0003DAD4EAD5FADA2976D857E858F859889B1
:102BD0000E9477AE6D877E878F87988BCE01019696
:102BE0000E948593E090CE0C1AA21BA21CA21DA2EB
:102BF00089819A81AB81BC818E8B9F8BA88FB98F85
:102C00008D819E81AF81B8858A8F9B8FAC8FBD8F60
:102C100089859A85AB85BC858E8F9F8FA8A3B9A324
:102C2000AE01425E5F4FBE01665E7F4FCE014696AB
:102C30000E94A672CE0182966C018E01065D1F4F26
:102C40009E01235F3F4FAE01425E5F4FBE01665E55
:102C50007F4F0C970E942661811151C0E090CE0CED
:102C60001EA21FA218A619A68091180D9091190DE9
:102C7000A0911A0DB0911B0D8E8B9F8BA88FB98FD1
:102C800080911C0D90911D0DA0911E0DB0911F0DF6
:102C90008A8F9B8FAC8FBD8F8091200D9091210DDD
:102CA000A091220DB091230D8E8F9F8FA8A3B9A361
:102CB000AE01425E5F4FBE01665E7F4FCE0146961B
:102CC0000E94A672DE0196966D018E01065D1F4F71
:102CD00024E23DE0AE01425E5F4FBE01665E7F4F83
:102CE000CE0146960E94266180E1E8E1FDE0A1E187
:102CF000BEE001900D928A95E1F70C94F02824969D
:102D0000EEADFFAD249731962496FFAFEEAF24973A
:102D100063CEECE4FFE184918F010F5F1F4F8823A6
:102D200021F00E942774F801F6CFE9E0F2E08491E7
:102D30008F010F5F1F4F882311F40C94F0280E941D
:102D40002774F801F4CF0E9469470C94F02841E001
:102D500061E081E00E94102F81110C94F02880E541
:102D60000E94B933882321F00E940F33162F01C02F
:102D700010E083E50E94B933882321F00E940F33CD
:102D80005B0103C08CE0A82EB12C84E50E94B9330E
:102D900081110E940F3382E50E94B933882329F004
:102DA0000E943F332B013C0106C0412C512C00ED09
:102DB000602E00E4702E113011F40C94F0281230C3
:102DC00009F08DC03A2C80E090E0A4E3B2E489835E
:102DD0009A83AB83BC8380E090E0ACE2B3E48D8364
:102DE0009E83AF83B88780E090E0A0E0BFEB898747
:102DF0009A87AB87BC87AA2011F40C94F0281E8A0E
:102E00001F8A188E198EAE014A5E5F4F6A017C01DF
:102E10008D0120E030E04CE253E460E070E084E3B8
:102E200092E40E94CD2FF12C00E010E01E8A1F8A50
:102E3000188E198EB801012E000C880B990B0E9478
:102E400019AA2CE739ED40E25FE30E9478AA4B0112
:102E50005C010E9450AFA30192010E9478AA20E079
:102E600030E04CE253E40E9477AE6AA37BA38CA3CC
:102E70009DA3C501B4010E94D8B0A30192010E9494
:102E800078AA20E030E044E352E40E9477AE6EA3DB
:102E90007FA388A799A7AE014A5E5F4FBE016E5D12
:102EA0007F4FCE0186960E94AA300F5F1F4F0A30D7
:102EB000110509F0BBCFF394F31408F4B5CF1E8AC3
:102EC0001F8A188E198EAE014A5E5F4FBE016B5F7E
:102ED0007F4FCE0101960E94AA300C94F02880E02A
:102EE00090E0A6EEB2E489839A83AB83BC8340E092
:102EF00050E06CE273E44D835E836F83788780E0FB
:102F000090E0A0E0BFEB89879A87AB87BC8700E0A1
:102F100010E024E332E40E8B1F8B288F398F4A8F09
:102F20005B8F6C8F7D8F8E8F9F8FA8A3B9A31AA202
:102F30001BA21CA21DA2CE0182966C01E12CF12CD9
:102F400000E01FEB9A01AB0160E070E084E392E4E3
:102F50000E94CD2FBB24B594A79410E0812F90E060
:102F60008A159B0514F00C94F0281AA21BA21CA22F
:102F70001DA2AE014E5D5F4FBE016B5F7F4FCE0164
:102F800001960E94AA301AA21BA21CA21DA2AE0189
:102F90004E5D5F4FBE01665E7F4FCE0146960E943A
:102FA000AA301F5FDBCF209311020C94F02841E080
:102FB00061E081E00E94102F81110C94F02880E0E4
:102FC00090E0A0E2B1E489839A83AB83BC838DEC6B
:102FD0009CECACE2B3E48D839E83AF83B88780E042
:102FE00090E0A0EAB1E489879A87AB87BC8780E547
:102FF0000E94B933882319F00E940F3301C060E0AA
:103000006E8BBE016F5F7F4FCE0146960E9491731B
:103010000C94F0288091DE048770873071F48FE47F
:103020000E94B933882319F00E94303303C08FE423
:103030000E94723381110C94F0280E943A71C09062
:10304000510D80E00E941C490E94AE2F11E01093A8
:10305000DD0488E50E947233E82E89E50E94723310
:10306000082F8AE50E947233F82EE11004C0011186
:1030700004C0182705C0011102C010E001C0182FBC
:1030800080E1E1E1FEE0A8E1BDE001900D928A95CA
:10309000E1F7111102C0FF2019F082E00E94A78E13
:1030A00082E50E94B933882361F00E943F334B01CF
:1030B0005C0120E030E0A9010E9413AA882371F18D
:1030C00006C0812C912CF0E8AF2EF0E4BF2E111138
:1030D00004C0E11002C00023D9F18092200D90922B
:1030E000210DA092220DB092230D2091190E309146
:1030F0001A0E40911B0E50911C0EC501B4010E9486
:103100009DB018165CF419821A821B821C82BE01C3
:103110006F5F7F4F80E29DE00E94CB3011110CC0A9
:10312000EE2061F1011108C080E00E94A78E1123FA
:1031300011F40C94A62D09C00E9468461111F4CF19
:10314000E1100C94A32D002319F081E00E94A78EBA
:103150000E94B832D090DC041092DD041092DC049E
:10316000812C912CE0EAAE2EE0E4BE2E89829A8278
:10317000AB82BC82111118C00C94C62D0111E5CF91
:103180000E94B832D090DC041092DD041092DC046E
:1031900080E090E0A0EAB0E489839A83AB83BC83AB
:1031A000FF2011F40C94BC2D80E090E0ADE1B3E47D
:1031B0008E8B9F8BA88FB98FBE016F5F7F4FCE0123
:1031C00046960E94CB3080E090E0A0EAB0E489838C
:1031D0009A83AB83BC8311110BC0011109C080918C
:1031E000150E9091160EA091170EB091180E04C0F6
:1031F00080E090E0A1E3B3E48E8B9F8BA88FB98F22
:1032000011110BC0E11009C04091110E5091120E26
:103210006091130E7091140E04C040E050E060EA1B
:1032200070E44AA35BA36CA37DA3AE014F5F5F4F25
:10323000BE016A5E7F4FCE0182960E94AA30D09274
:10324000DD04D092DC048C2D0E941C490E94952F35
:103250000E94265E0C94F02880E00E941C4913E036
:1032600001E00093DF0424982C9A149A0E94A84944
:103270001092DF04249A2C9814988091510D882381
:1032800051F08091510D882369F08DE992E00E9400
:10329000DD8F0C94F0288DEC92E00E94DD8F1150B0
:1032A00001F7EFCFE4EBF2E084918F010F5F1F4F46
:1032B000882321F00E942774F801F6CF8EE292E075
:1032C0000E94DD8F8FE192E00E945790C090110E16
:1032D000D090120EE090130EF090140E88E50E942C
:1032E000B933811108C020E030E0A901C701B6015F
:1032F0000E9477AE02C00E943F336E8B7F8B888F17
:10330000998FC090150ED090160EE090170EF09089
:10331000180E89E50E94B933811108C020E030E021
:10332000A901C701B6010E9477AE02C00E943F33D7
:103330009B01AC0169837A838B839C836E897F892F
:10334000888D998D0E94898F882311F40C94F02820
:1033500080E00E941C490E94AE2F85E40E94B93390
:10336000882321F00E943033182F04C085E40E9486
:10337000723311E086E50E94B933882321F00E9460
:103380000F33262F01C021E0412FBE016F5F7F4F19
:10339000CE0146960E9484A36B017C019B01AC0187
:1033A0000E9423B181115FC08E889F88A88CB98C40
:1033B00020E030E0A901C501B4010E9413AA87FDF5
:1033C00005C027E137EB41E558E304C027E137EBBF
:1033D00041E558EBC501B4010E9477AEAB01BC01D9
:1033E00085E493E00E94AF4389809A80AB80BC80E3
:1033F00020E030E0A901C501B4010E9413AA87FDB5
:1034000005C027E137EB41E558E304C027E137EB7E
:1034100041E558EBC501B4010E9477AEAB01BC0198
:1034200080E493E00E94AF4320E030E0A901C701AF
:10343000B6010E9413AA87FD05C027E137EB41E5DD
:1034400058E304C027E137EB41E558EBC701B6016B
:103450000E9477AEAB01BC018BE393E00E94AF43C7
:103460008AE00E9427740E94952F0E94265E0C9489
:10347000F028209316030C94F028A0E0B3E0BFA737
:10348000AEA761E1E62E6EE0F62E78EFC72E7DE066
:10349000D72E312C00E010E0EEA5FFA58191FFA70B
:1034A000EEA70E94B9338823C1F10E943F332B015C
:1034B0003C01133049F0D6012D913D914D915C9125
:1034C0000E9476AE2B013C01F701208131814281BF
:1034D0005381C301B2010E9476AE4B015C012DEB1A
:1034E00037E346E855EB0E949DB087FD0AC02DEBFF
:1034F00037E346E855E3C501B4010E9413AA181644
:1035000064F4133011F001E002C033243394D70186
:103510004D925D926D927C9213971F5FB4E0EB0E1B
:10352000F11CE4E0CE0ED11C143009F0B5CF00231D
:1035300019F00E94B83257C0332009F454C0C0902B
:103540001D0ED0901E0EE0901F0EF090200E2091C8
:10355000A60D3091A70D4091A80D5091A90DC7015E
:10356000B6010E9478AA0E94A8B060938C0E709356
:103570008D0E80938E0E90938F0EC0927C0ED09203
:103580007D0EE0927E0EF0927F0E9091360E80912D
:10359000370E981719F00E94DC7025C00E943A710E
:1035A00080916F0081FB992790F981FF05C0809180
:1035B0006F008D7F80936F0040918C0E50918D0E27
:1035C00060918E0E70918F0E4093CF0D5093D00D61
:1035D0006093D10D7093D20D992329F080916F00E3
:1035E000826080936F000E94265E0C94F0280E94F7
:1035F000A7A50C94F0288091F30D9091F40D8B39D0
:10360000910509F49CC40CF0AEC08C35910509F409
:103610006DC50CF062C08C34910509F489C29CF52B
:103620008231910509F42DC594F497FF02C00C94E2
:10363000A728823091050CF454C1419711F00C94E5
:10364000A72817981698159814980C94F0288A3281
:10365000910509F4E2C18B34910509F41AC24F9720
:1036600011F00C94A7280E94F5386E8B7F8B888F01
:10367000998FBE016F5F7F4FCE0146960E94D9346D
:10368000EEEDFEE1B4C18235910509F4F1C4B4F464
:103690008E34910509F465C20CF45FC28135910541
:1036A00011F00C94A7280E94AB3F0E944A7110921F
:1036B0000D0410920C0400E010E0C3C484359105A1
:1036C00009F4DFC40CF4D8C48535910511F00C94CD
:1036D000A7280E94C8600C94F0288137910509F44E
:1036E000E7C3FCF48B36910509F4A7C464F489366A
:1036F000910509F409C40CF09CC48836910509F4BD
:1037000032C30C94A7288E36910509F44DC38F3629
:10371000910509F45CC38D36910511F00C94A7282E
:1037200035C48637910509F4EFC46CF483379105ED
:1037300009F4E6C40CF4DEC48537910511F40C9449
:10374000F0280C94A7288837910509F4F6C50CF4E5
:1037500028C58937910509F4F6C58C38910509F417
:1037600033C40C94A7288E35F1E09F0711F40C9414
:10377000E5260CF04BC0833D910509F4EAC614F52B
:103780008B3C910509F44CC674F4883C910509F40E
:10379000DFC5893C910509F421C68E3B910511F0E6
:1037A0000C94A7282FC48D3C910509F4CCC60CF4C9
:1037B00055C68E3C910511F00C94A7280E9402601A
:1037C0000C94F0288D3241E0940709F4D8C674F4C3
:1037D0008D3D910509F4CDC6823E910509F4CCC614
:1037E0008C3D910511F00C94A728B6C68F32A1E04C
:1037F0009A0709F4CAC60CF4C5C68033914011F08B
:103800000C94A7280E94AE5A0C94F028843FF1E053
:103810009F0711F40C947D279CF5813941E09407B2
:1038200011F40C94EE26ACF48336A1E09A0711F45F
:103830000C94E8268039B1E09B0711F40C94EB2638
:103840008F35914011F00C94A7280E94DB590C94FD
:10385000F028843AF1E09F0711F40C94F4268C3A96
:1038600021E0920709F472C68239914011F00C945C
:10387000A72880E00E9461490E94265E0C94F028EF
:10388000883F41E0940711F40C948F276CF4863F35
:10389000A1E09A0711F40C94802714F00C9483276C
:1038A0000E949D9C0C94F0288438E3E09E0711F45C
:1038B0000C9417283CF48335934011F40C94B127F1
:1038C0000C94A7288B3833E0930711F40C946E28DE
:1038D000873E934011F00C94A7280E94AD590C9498
:1038E000F0280091F10D1091F20D80E50E94B9339E
:1038F000882361F00E94FF326B017C01BB24B394EA
:10390000672B682B692B31F4B12C04C0B12CC12C6E
:10391000D12C760183E50E94B933882311F40C94ED
:1039200002290E943F3320E030E04AE754E40E943D
:1039300078AA0E94C0AF6B017C01B1100BC0672B4D
:10394000682B692B39F40115110521F0D8018C91F0
:10395000811102C0B12C02C0BB24B3940E943A7101
:10396000BB20C1F0EEEDFEE184915F01BFEFAB1A29
:10397000BB0A882321F00E942774F501F5CFF801D6
:1039800081918F01882319F00E942774F8CF8AE073
:103990000E94277483E08093D30C81E08093B30D61
:1039A000C114D104E104F104D9F00E94E938C60E33
:1039B000D71EE81EF91E0E94E938DC01CB018C19E4
:1039C0009D09AE09BF09B7FD04C01092B30D0C9458
:1039D000F0288091B30D8823C1F30E948790EBCF2C
:1039E0008091B30D882389F30E948790F9CF849149
:1039F0008F010F5F1F4F882321F00E942774F80169
:103A0000F6CFBE016F5F7F4F8DE493E00E94C64406
:103A10008AE00E9427740C94F02883E50E94B93351
:103A2000882311F40C94F0280E941F33E82E80E5BF
:103A30000E94B933811112C081E0E11001C080E021
:103A40008093DF04882329F024982C9A149A0C94EC
:103A5000F028249A2C9814980C94F02880E50E9461
:103A6000B933882339F00E941F33182F87FF03C012
:103A70000C94F0281DE0EAE5F3E08DE28E0F9491BE
:103A8000191711F40C94072931968E13F8CF0C9462
:103A90000A291091CA04113011F40C94F028123044
:103AA00059F40E94F5386093BE047093BF0480936C
:103AB000C0049093C10418C01092C6041092C704A9
:103AC0001092C8041092C9041092C2041092C30448
:103AD0001092C4041092C5041092BE041092BF0448
:103AE0001092C0041092C10481E08093CA040E9425
:103AF000E9386093C6047093C7048093C804909318
:103B0000C904123011F40C94F0288091CC049091E7
:103B1000CD0401969093CD048093CC041092EA0CCE
:103B20001092EB0C1092EC0C1092ED0C0C94F0280F
:103B30008091CA04813011F00C94F02882E08093C7
:103B4000CA040E94E9386093C2047093C30480934E
:103B5000C4049093C5040C94F0280E9428390C9456
:103B6000F02883E50E94B933811103C0E5EEF3E04C
:103B700009C00E940F336E347105C1F70E94C93429
:103B80000C94F02884918F010F5F1F4F882321F040
:103B90000E942774F801F6CFECEDF3E084918F01D9
:103BA0000F5F1F4F882321F00E942774F801F6CF82
:103BB0006091CC047091CD0480E090E04AE00E94D6
:103BC0005378EFECF3E084918F010F5F1F4F882350
:103BD00021F00E942774F801F6CF6091CE04709115
:103BE000CF0480E090E04AE00E945378E4ECF3E0F8
:103BF00084918F010F5F1F4F882321F00E9427744B
:103C0000F801F6CF6091CC047091CD048091CE0480
:103C10009091CF04681B790B8091CA04815021E0F8
:103C200030E0823010F020E030E0621B730B80E067
:103C300090E04AE00E9453788AE00E942774ECEBFF
:103C4000F3E084918F010F5F1F4F882321F00E94C2
:103C50002774F801F6CF8091D0049091D104A091FF
:103C6000D204B091D3048E8B9F8BA88FB98FBE01E5
:103C70006F5F7F4FCE0146960E94D934EFEAF3E0A2
:103C800084918F010F5F1F4F811106C09E012F5F2E
:103C90003F4F7901890104C00E942774F801F0CFD9
:103CA000D8018D918D01882319F00E942774F8CFD7
:103CB0008091D4049091D504A091D604B091D704FA
:103CC0008E8B9F8BA88FB98FBE016F5F7F4FCE0108
:103CD00046960E94D934EFE9F3E084918F010F5F9B
:103CE0001F4F882321F00E942774F801F6CFF701B7
:103CF00081917F01882319F00E942774F8CF8AE010
:103D00000E942774E7E9F3E084918F010F5F1F4F52
:103D1000882321F00E942774F801F6CFE7E8F3E04A
:103D200084918F010F5F1F4F882321F00E94277419
:103D3000F801F6CF20E030E04AE754E46091D8047F
:103D40007091D9048091DA049091DB040E9453AF02
:103D500042E00E94D3788DE60E9427748AE00E9498
:103D600027740C94F02888E690E00E94C5338111F6
:103D70000C94F0288091F10483FF02C00C94F02889
:103D800083E50E94B933882311F40C94F0280E9433
:103D90003F330E94BBAF709302046093010480E044
:103DA0000E94613F0C94F0288EE40E94B93388236E
:103DB00011F40C94F0280E940F336093270E709337
:103DC000280E8093290E90932A0E0C94F02883E5F8
:103DD0000E947233882359F083E50E94B933882307
:103DE00019F00E941F3301C080E08093F104EEEDD2
:103DF000FEE184918F010F5F1F4F882321F00E9405
:103E00002774F801F6CFEBEFF3E084918F010F5F99
:103E10001F4F882321F00E942774F801F6CF80916C
:103E2000F1048823A1F15DEEC52E53E0D52EE12CDF
:103E3000F12C20E08091F10490E00E2C02C09595C9
:103E400087950A94E2F780FF17C0BB24B394B20EA3
:103E5000222319F08CE20E942774F60125913491F7
:103E6000F901849189010F5F1F4F882321F00E947F
:103E700027749801F5CF2B2DFFEFEF1AFF0A32E0E0
:103E8000C30ED11C45E0E416F104A1F60CC0E7EF27
:103E9000F3E084918F010F5F1F4F882321F00E9470
:103EA0002774F801F6CF8AE00E9427740C94F0285A
:103EB00083E50E94B933882369F00E941F338D3354
:103EC00020F480934F020C94F0288CE380934F02EF
:103ED0000C94F028EEEDFEE184918F010F5F1F4FEF
:103EE000882321F00E942774F801F6CF40914F02F9
:103EF00050E060E070E082E094E00E9492438AE04B
:103F00000E9427740C94F02889E690E00E94C53343
:103F1000811111C0E9E0F4E084918F010F5F1F4F20
:103F2000882321F00E942774F801F6CF0E940344F1
:103F30008AE00E9427741092D30C0C94F02D83E534
:103F40000E94B933882311F40C94F0280E941F3387
:103F5000182F8D3308F01CE310930A0D0E94E938E6
:103F60006B017C01212F30E0A8EEB3E00E9467AE28
:103F7000C60ED71EE81EF91EC092060DD092070D80
:103F8000E092080DF092090D0C94F0288DE690E077
:103F90000E94C53381110C94F0288091F10483FFB5
:103FA00002C00C94F02883E50E94B93327968FAFA6
:103FB000279781110C941D2982E50E94B933811144
:103FC0000C941D290C94F0288091F10483FF02C009
:103FD0000C94F02883E50E94B933882311F40C94E3
:103FE000F0280E943F330E94BBAF6639710514F080
:103FF00066E970E0709300046093FF030E94173F2E
:104000000C94F0288091F10483FF02C00C94F028F6
:1040100083E50E94B93327968FAF279781110C94BF
:10402000862A82E50E94B93381110C94862A0C9469
:10403000F0280E94EF600C94F0280E94E0600C943D
:10404000F02862E370E080E090E00E94AF380E94C8
:104050002F420F5F1F4F0331110599F762E370E0A4
:1040600080E090E00E94AF380E942F420C94F0282C
:10407000109215030C94F02881E0809315030C94A2
:10408000F02883E50E94B9338823A1F00E943F33D2
:1040900020E030E04AE754E40E9478AA0E94C0AFD2
:1040A0006093500270935102809352029093530296
:1040B0000C94F02888E50E94723381110C94F92B3E
:1040C00089E50E94723381110C94F92B8AE50E94D4
:1040D000723381110C94F92B85E40E9472338111A3
:1040E0000C94F92B0E944A710C94F0280E942A60CB
:1040F0000C94F0280E943A710E94265E0C94F028DD
:104100000E94D75D0C94F0280091F10D1091F20DF2
:1041100083E0D12C40E08150E9F0D8019C91292F17
:104120002B7F2134C1F711962C912133A1F79134C3
:1041300021F0953421F441E002C0DD24D3949801AC
:104140002E5F3F4F89012F5F3F4FF80190819032E2
:10415000C9F3E1CF442369F0EEEDFEE184917F01E4
:104160002FEFE21AF20A882321F00E942774F70148
:10417000F5CFDD2069F0E4E1F4E084917F013FEFC9
:10418000E31AF30A882321F00E942774F701F5CF80
:10419000D8018D918D01882309F485CE0E94277462
:1041A000F7CF81E08093DF0424982C9A149AE8E4F6
:1041B000F4E084918F010F5F1F4F882321F00E944C
:1041C0002774F801F6CFE0E4F4E084918F010F5FEB
:1041D0001F4F882321F00E942774F801F6CF1E9B01
:1041E00003C005EE12E002C00AEE12E0F801819170
:1041F0008F01882319F00E942774F8CF8AE00E946B
:104200002774E8E3F4E084918F010F5F1F4F882348
:1042100021F00E942774F801F6CF379B03C005EE0A
:1042200012E002C00AEE12E0D8018D918D018823C0
:1042300019F00E942774F8CF8AE00E942774E0E307
:10424000F4E084918F010F5F1F4F882321F00E94BB
:104250002774F801F6CF1D9B03C005EE12E002C0E3
:104260000AEE12E0F80181918F01882319F00E9473
:104270002774F8CF8AE00E942774E8E2F4E0849182
:104280008F010F5F1F4F882321F00E942774F801D0
:10429000F6CF029B03C005EE12E002C00AEE12E068
:1042A000D8018D918D01882319F00E942774F8CFD1
:1042B0008AE00E942774E0E2F4E084918F010F5FAE
:1042C0001F4F882321F00E942774F801F6CF1C9B12
:1042D00003C005EE12E002C00AEE12E0F80181917F
:1042E0008F01882319F00E942774F8CF8AE00E947A
:1042F0002774E8E1F4E084918F010F5F1F4F88235A
:1043000021F00E942774F801F6CF019B03C005EE4F
:1043100012E002C00AEE12E0D8018D918D018823CF
:1043200019F00E942774F8CF8AE00E942774109237
:10433000DF04249A2C98149853C781E08093DD04FD
:104340008093DC044DC71092DD041092DC0448C752
:1043500088EC90E00E94C533811142C784E40E943A
:1043600072338823C1F10E943F3311E020E030E036
:10437000A9010E9413AA811101C010E01093AE0D93
:10438000112349F10E943F33E091FA03B4E0EB9F1F
:10439000F0011124E655F24F608371838283938389
:1043A00020E030E0A9016091AA0D7091AB0D8091E1
:1043B000AC0D9091AD0D0E9413AA81110CC080E04C
:1043C00090E0A0E4B0E48093AA0D9093AB0DA0938D
:1043D000AC0DB093AD0D0E942C7302C79AE7E92E85
:1043E0009DE0F92E00E013E024E0D22ED00EF8017B
:1043F00081918F010E947233882351F00E943F33D4
:104400000E94C0AFD7016D937D938D939C931397BA
:10441000B4E0EB0EF11CD012EACF0E94B08CE0C6E3
:104420001AE8E12E1DE0F12E00E013E084E0D82E22
:10443000D00EF80181918F010E947233882341F0E0
:104440000E943F33D7016D937D938D939C93139777
:10445000B4E0EB0EF11CD012ECCFC2C683E50E9493
:10446000B9338823A1F00E943F336093760D709397
:10447000770D8093780D9093790D60936E0D709306
:104480006F0D8093700D9093710D10E001C011E0DD
:1044900080E50E94B933882359F00E943F3360932E
:1044A000760D7093770D8093780D9093790D10E0D1
:1044B00082E50E94B933882359F00E943F3360930C
:1044C000720D7093730D8093740D9093750D10E0C1
:1044D00084E50E94B933882359F00E943F336093EA
:1044E0006E0D70936F0D8093700D9093710D78C663
:1044F000112309F475C64091760D5091770D6091A6
:10450000780D7091790D88E694E00E94AF43409158
:10451000720D5091730D6091740D7091750D85E65B
:1045200094E00E94AF4340916E0D50916F0D6091E9
:10453000700D7091710D82E694E00E94AF438AE0A5
:104540000E9427744DC60E946D5D4AC60E94135F8B
:1045500047C60E948F5C44C683E50E94B933882316
:1045600009F43EC60E940F3370934E0260934D02D1
:1045700037C60E941A5C34C60E94D05B31C60E94C6
:104580002D5B2EC60E94585A2BC685E40E94B93373
:10459000882321F00E940F337B0102C0E12CF12C13
:1045A00083E40E94B933882331F00E940F33AD9623
:1045B0006FAFAD9704C045E0AD964FAFAD9785E5C1
:1045C0000E94B933882319F00E94303303C085E577
:1045D0000E947233E9968FAFE997F7FC07C0812CF0
:1045E000912CB6E1AB2EB3E4BB2E06C0812C912CEE
:1045F000ACE8AA2EA2E4BA2E83E50E94B933882340
:1046000021F00E943F334B015C01E114F10411F4ED
:104610001092FA03EEA60E94E9382B013C015EA538
:1046200057FF0DC00CE310E080E090E0A0E0B1E4A3
:10463000ED968CAF9DAFAEAFBFAFED970CC004E170
:1046400010E020E030E040E551E4ED962CAF3DAFC6
:104650004EAF5FAFED9761E06E0D623068F0E1E163
:10466000F6E084918F010F5F1F4F882309F4B8C5CE
:104670000E942774F801F5CFEBE3F6E084917F0107
:104680003FEFE31AF30A882321F00E942774F70111
:10469000F5CF0E94AB3F4EA547FF04C08FE7809344
:1046A000F90308C05EA5E52F550FFF0BE850FC4F3E
:1046B0008FE78083C501B4010E94BBAF072E000CB9
:1046C000880B990B0E9419AA6AAF7EAF23968FAF11
:1046D000239727969FAF27979801A8EEB3E00E94F3
:1046E00067AEC358DF4F688379838A839B83CD5736
:1046F000D040DC01CB01840D951DA61DB71DC75709
:10470000DF4F88839983AA83BB83C958D04081E057
:1047100080935402E4964CAE5DAE6EAE7FAEE497ED
:10472000CF57DF4F488259826A827B82C158D0407E
:10473000E0961FAEE097CB57DF4F188219821A829E
:104740001B82C558D0406B961FAE6B9790E4639662
:104750009FAF6397ACE16F96AFAF6F97B6E4A39648
:10476000BFAFA397A7961FAEA797A8961FAEA8970F
:10477000A9961FAEA997AA961FAEAA9762961CAEDD
:104780001DAE1EAE1FAE62972E961CAE1DAE1EAEA7
:104790001FAE2E97C12CD12C76012FE730E040E0E0
:1047A00050E02EAB3FAB48AF59AFEFE78E2E912CC8
:1047B000A12CB12CE8961CAE1DAE1EAE1FAEE89724
:1047C00031E0AF963FAFAF9768961FAE1EAE6897C9
:1047D00010E0212C312C00E04EA5842F440F990BC2
:1047E000DC01A850BC4FC357DF4FB983A883CD5815
:1047F000D040880F991F880F991FFC01E15FFB4F84
:10480000AC96FFAFEEAFAC97AD962FADAD97022E45
:10481000000C330BAE963FAF2EAFAE978091540293
:10482000882309F41AC10E94E9386AAB7BAB8CABD0
:104830009DAB8091E703882309F4EFC00E94644098
:104840003EA537FF09C01091FB032090FC03309078
:10485000FD030091FE030DC0AC96AEADBFADAC97AD
:104860001C9111962C90119712963C9012971396CA
:104870000C91212F322D432D502FA7966FADA79766
:10488000A8967FADA897A9968FADA997AA969FAD38
:10489000AA970E9413AA87FF0CC0A7961FAFA797DD
:1048A000A8962FAEA897A9963FAEA997AA960FAF44
:1048B000AA97212F322D432D502F6B966FAD6B97FA
:1048C00063967FAD63976F968FAD6F97A3969FADFD
:1048D000A3970E949DB0181664F46B961FAF6B9758
:1048E00063962FAE63976F963FAE6F97A3960FAF09
:1048F000A397AF96BFADAF972AAD3EAD23964FAD10
:10490000239727965FAD2797612F722D832D902FC8
:10491000BB2309F468C00E949DB018160CF07DC03E
:104920002AA93BA94CA95DA92419350946095709AB
:10493000CE56DF4F288339834A835B83C259D040E8
:10494000DA01C90188589341A109B109B7FD65C0D1
:10495000D501C4012EA93FA948AD59AD821B930BC7
:10496000A40BB50B3EA5B595A7959795879537FFF1
:1049700003C08093F90307C0C357DF4FE881F98173
:10498000CD58D0408083CE56DF4F288139814A816F
:104990005B81C259D040E8962CAF3DAF4EAF5FAFC0
:1049A000E8973AADA7963FAFA7974EADA8964FAF01
:1049B000A89723965FAD2397A9965FAFA9972796EF
:1049C0008FAD2797AA968FAFAA972AA93BA94CA982
:1049D0005DA9E4962CAF3DAF4EAF5FAFE497AF96C5
:1049E0001FAEAF971AC00E9413AA87FF16C08AA9EC
:1049F0009BA9ACA9BDA9E4962CAD3DAD4EAD5FAD74
:104A0000E497821B930BA40BB50BAC01BD01485876
:104A100053416109710977FF14C720E030E040EA93
:104A200051E46AAD7EAD23968FAD239727969FAD57
:104A300027970E9477AE9B01AC01612F722D832DC9
:104A4000902F0E949DB018167CF4EDE9F5E084915A
:104A50008F010F5F1F4F811103C00E94AB3FC0C386
:104A60000E942774F801F3CF8AA99BA9ACA9BDA91C
:104A7000CF57DF4F288139814A815B81C158D040AF
:104A8000821B930BA40BB50BB7FDBAC00E94034465
:104A90008AE00E9427748AA99BA9ACA9BDA980536A
:104AA000984FAF4FBF4FCF57DF4F88839983AA836B
:104AB000BB83C158D040E0969FADE09791117BC079
:104AC000CB57DF4F288139814A815B81C558D0405F
:104AD000612F722D832D902F0E949DB018160CF01F
:104AE0004DC020E030E040E050E4612F722D832D76
:104AF000902F0E9477AECB57DF4F688379838A83EC
:104B00009B83C558D0402AA93BA94CA95DA9C3588D
:104B1000DF4F88819981AA81BB81CD57D040280F72
:104B2000391F4A1F5B1FC757DF4F288339834A83CA
:104B30005B83C958D040ED962CAD3DAD4EAD5FAD19
:104B4000ED976AAD7EAD23968FAD239727969FADE7
:104B500027970E9476AE9B01AC0191E0E0969FAF53
:104B6000E097612F722D832D902F0E949DB0181613
:104B70000CF446C0E0961FAEE09742C08AA99BA9FC
:104B8000ACA9BDA9C757DF4F288139814A815B8114
:104B9000C958D040821B930BA40BB50BB7FD30C096
:104BA0003EA53F3F19F049E655E002C04BE755E00E
:104BB0006EE875E022C020E030E040EA51E46AADE2
:104BC0007EAD23968FAD239727969FAD27970E94A2
:104BD00076AE9B01AC01612F722D832D902F0E9428
:104BE00013AA87FF0DC04EA54F3F19F042E355E0D1
:104BF00002C045E455E069E575E08EA50E9483405A
:104C00008AA99BA9ACA9BDA9880F991FAA1FBB1F80
:104C1000E4962CAD3DAD4EAD5FADE497821B930B9A
:104C2000A40BB50B84199509A609B70981389F44CF
:104C3000A241B10568F0E4E1F5E084918F010F5FD6
:104C40001F4F882309F409CF0E942774F801F5CF7C
:104C500068964EAD5FAD6897AE968EAD9FADAE9740
:104C6000841795070CF0DACDE7EBF4E084918F011F
:104C70000F5F1F4F882321F00E942774F801F6CFA1
:104C80009EA597FD03C00BEF12E002C004EF12E0F7
:104C9000B80186EA94E00E94C644B701A60182EA00
:104CA00094E00E94AF438AE00E942774B80181E932
:104CB00094E00E94C6442E964CAD5DAD6EAD7FADC6
:104CC0002E978DE894E00E94AF438AE00E942774FB
:104CD000B8018CE794E00E94C64462964CAD5DAD8D
:104CE0006EAD7FAD629788E794E00E94AF438AE0A3
:104CF0000E942774E996AFADE997AA2309F470C220
:104D0000BEA5B7FF31C0C092410DD092420DE092D6
:104D1000430DF092440D2CEA35EC47E25EE32E960B
:104D20006CAD7DAD8EAD9FAD2E970E9478AA60933D
:104D30003D0D70933E0D80933F0D9093400D2CEAF6
:104D400035EC47E25EE362966CAD7DAD8EAD9FAD16
:104D500062970E9453AF6093390D70933A0D809320
:104D60003B0D90933C0D3CC2C0924D0DD0924E0D28
:104D7000E0924F0DF092500D2CEA35EC47E25EE3E5
:104D80002E966CAD7DAD8EAD9FAD2E970E9478AA0C
:104D90006093490D70934A0D80934B0D90934C0D89
:104DA0002CEA35EC47E25EE362966CAD7DAD8EADEC
:104DB0009FAD62970E9453AF6093450D7093460D6F
:104DC0008093470D9093480D0BC20E94205A08C251
:104DD0000E94C05905C20E943A7102C281E00E943D
:104DE00061490E94265EFCC183E50E9472338823DC
:104DF00049F00E943033182F811106C080E00E94D4
:104E00001C4902C01091510D8091110E9091120E0B
:104E1000A091130EB091140E89839A83AB83BC8347
:104E20008091150E9091160EA091170EB091180E4C
:104E30008D839E83AF83B8878091190E90911A0E4F
:104E4000A0911B0EB0911C0E89879A87AB87BC87F7
:104E500086E50E947233882321F08CE796E00E9459
:104E600033A5812F0E941C49111103C0EEEDFEE114
:104E70001CC08091510D8111F9CFECE4FFE18491C8
:104E80008F010F5F1F4F882321F00E942774F801C4
:104E9000F6CFEDE5F6E084918F010F5F1F4F882379
:104EA00029F30E942774F801F6CF84918F010F5FD8
:104EB0001F4F882321F00E942774F801F6CF8091BC
:104EC000510D811103C06CEF72E002C068EF72E017
:104ED0008FE496E00E94C6448AE00E9427744CE06A
:104EE00050E061E17EE0CE0101960E9461B1892B24
:104EF00009F476C10E94265E73C10E94087F70C1CA
:104F00000E94309B6DC183E50E947233882321F09B
:104F10000E94303391E089270E94B69661C12093A8
:104F2000280D0E9477791092280D882309F458C122
:104F3000EEEDFEE184918F010F5F1F4F882321F07A
:104F40000E942774F801F6CFE9E9F6E084918F0119
:104F50000F5F1F4F882309F443C10E942774F80193
:104F6000F5CF8AE50E94B933882309F438C00E943E
:104F70003F336B017C0120E030E040E050EC0E94C8
:104F80009DB087FD13C020E030E040EA50E4C70147
:104F9000B6010E9413AA18164CF0C092210ED092AE
:104FA000220EE092230EF092240E1AC1ECE4FFE1EF
:104FB00084918F010F5F1F4F81110DC0E6EBF6E06A
:104FC00084918F010F5F1F4F882309F409C10E944C
:104FD0002774F801F5CF0E942774F801E9CFEEEDB0
:104FE000FEE184918F010F5F1F4F882321F00E9403
:104FF0002774F801F6CFE7EAF6E084918F010F5F9E
:105000001F4F882321F00E942774F801F6CF4091AA
:10501000210E5091220E6091230E7091240E84EA8D
:1050200096E00E94AF438AE00E942774D9C08BE4C7
:105030000E94B9338823B1F18BE40E94B9338823ED
:10504000B1F00E943F336B017C0120E030E0A90108
:105050000E949DB087FD19C020E030E040E251E49D
:10506000C701B6010E9413AA18167CF003C0C12C18
:10507000D12C76010E943A71C092350DD092360D36
:10508000E092370DF092380DABC0E1EDF6E084917F
:105090008F010F5F1F4F882309F4A2C00E9427745D
:1050A000F801F5CFEEEDFEE184918F010F5F1F4F08
:1050B000882321F00E942774F801F6CF4091350D26
:1050C0005091360D6091370D7091380D80EF96E05C
:1050D0000E94AF438AE00E94277482C088E50E9444
:1050E00072338823F1F00E940F338B01072E000CDE
:1050F000220B330B0093290D10932A0D20932B0DB7
:1051000030932C0DDB012FEF30E00E945BB120EDDE
:1051100037E040E050E00E9441AEB9018EE20E94CB
:10512000E8378AE50E947233882329F00E940F3302
:1051300081E00E94FC9F85E40E947233882309F479
:105140004FC00E940F3382E00E94FC9F49C00E9422
:10515000A7A546C0F090F30D0E943A71FF2029F1F7
:10516000EEEDFEE184918F010F5F1F4F882321F048
:105170000E942774F801F6CF84E50E9427746F2DF2
:1051800070E080E090E04AE00E94537880E20E9464
:105190002774EDE0F7E084918F010F5F1F4F8823A4
:1051A000F9F00E942774F801F6CF1092CE0CEEEDC4
:1051B000FEE184918F010F5F1F4F882321F00E9431
:1051C0002774F801F6CF6091CE0C70E08BEF96E07B
:1051D0000E94AD448AE00E94277402C00E94A7A5E5
:1051E0001092D30CC157DF4FE881CF58D040EE2347
:1051F00009F4F6C40E941995F3C40E94A5470E94C1
:10520000DA93EECFB1100C94AA1C0C94A31C0E944C
:105210000B61E6CF812F0E94D3A16E2D812F0E94BA
:105220001A37F12CB701812F0E94E8371830C1F6E8
:10523000F0920D04E0920C04D3CF0E943F330E9401
:10524000BBAF709302046093010480E00E94613F51
:1052500081E0809354021AAA1BAA1CAA1DAA6A966E
:105260001CAE1DAE1EAE1FAE6A971EA62B961FAEBD
:105270002B97FCE32F96FFAF2F972CE16B962FAF68
:105280006B9736E463963FAF6397C12CD12C90E8BF
:10529000E92E2FEBF22E812C912C54016091010408
:1052A00070910204072E000C880B990B0E9419AA1A
:1052B000262E172F082F392E262F372F482F592FFC
:1052C000B601C7010E9413AA8823E1F020910F04C0
:1052D000309110044091110450911204622D712FED
:1052E000802F932D0E9413AA881F8827881F8EA7BE
:1052F00027965FAD2797552349F0882339F0809191
:1053000054026ECF2C2C1D2D0E2D3F2C0E94E938FF
:105310006B017C01DC01CB016A962CAD3DAD4EAD3D
:105320005FAD6A97821B930BA40BB50BB7FD3DC015
:10533000D701C60188519C4FAF4FBF4F6A968CAFC3
:105340009DAFAEAFBFAF6A970E940344ECE0F4E0BC
:1053500084913F019FEF691A790A882321F00E9406
:105360002774F301F5CF81149104A104B104B9F0BD
:10537000D501C40188519C4FAF4FBF4FBC01CD0137
:105380006C197D098E099F0928EE33E040E050E05A
:105390000E941FAECA01B9010E94B97803C08FE311
:1053A0000E9427748AE00E9427740E9487900E94BE
:1053B000E9386093E20C7093E30C8093E40C9093D3
:1053C000E50CA0910F04AEABB0911004BAAFE09120
:1053D0001104EEAFF09112042396FFAF23979D01C5
:1053E000AF01622D712F802F932D0E9476AE2B017D
:1053F0003C0120E030E0A9010E949DB087FF04C07D
:1054000077FA709477F8709420E030E040E251E44D
:10541000C301B20181149104A104B10429F40E94D2
:1054200013AA87FF07C004C00E949DB0181614F489
:10543000460157012EA5222309F44CC08AA99BA935
:10544000ACA9BDA9892B8A2B8B2B61F0D701C60192
:105450002AA93BA94CA95DA9821B930BA40BB50BF0
:10546000B7FD38C02EA93AAD4EAD23965FAD239758
:105470002B966FAD2B972F967FAD2F976B968FAD99
:105480006B9763969FAD63970E9476AE20E030E005
:1054900040EC5FE30E9413AA87FD31CFD701C6011C
:1054A000805A9541AF4FBF4F8AAB9BABACABBDAB06
:1054B0009EA92B969FAF2B97AAAD2F96AFAF2F9794
:1054C000BEAD6B96BFAF6B972396EFAD23976396F8
:1054D000EFAF639780915402882309F410CF8114B1
:1054E0009104A104B10429F4C22CD12EE02EF32C96
:1054F000D5CEF8EECF1AF3E0DF0AE108F108C818BC
:10550000D908EA08FB08F7FEFACEEECF0E943F3337
:105510000E94BBAF663971050CF068C1709300043E
:105520006093FF030E94173F81E0809354028091B3
:10553000CE0C8093FA031AAA1BAA1CAA1DAA6A966B
:105540001CAE1DAE1EAE1FAE6A971EA62B961FAEDA
:105550002B972CE32F962FAF2F973CE16B963FAF05
:105560006B9746E463964FAF6397C12CD12C30E81C
:10557000E32E4FEBF42E812C912C54016091FF030C
:1055800070910004072E000C880B990B0E9419AA39
:10559000262E172F082F392E262F372F482F592F19
:1055A000B601C7010E9413AA8823E1F02091FB03F2
:1055B0003091FC034091FD035091FE03622D712F49
:1055C000802F932D0E9413AA881F8827881F8EA7DB
:1055D00027965FAD2797552349F0882339F08091AE
:1055E0005402FECD2C2C1D2D0E2D3F2C0E94E9388F
:1055F0006B017C01DC01CB016A962CAD3DAD4EAD5B
:105600005FAD6A97821B930BA40BB50BB7FD3DC032
:10561000D701C60188519C4FAF4FBF4F6A968CAFE0
:105620009DAFAEAFBFAF6A970E940344E0E1F4E0E4
:1056300084913F019FEF691A790A882321F00E9423
:105640002774F301F5CF81149104A104B104B9F0DA
:10565000D501C40188519C4FAF4FBF4FBC01CD0154
:105660006C197D098E099F0928EE33E040E050E077
:105670000E941FAECA01B9010E94B97803C08FE32E
:105680000E9427748AE00E9427740E9487900E94DB
:10569000E9386093E20C7093E30C8093E40C9093F0
:1056A000E50CA091FB03AEABB091FC03BAAFE09167
:1056B000FD03EEAFF091FE032396FFAF23979D010C
:1056C000AF01622D712F802F932D0E9476AE2B019A
:1056D0003C0120E030E0A9010E949DB087FF04C09A
:1056E00077FA709477F8709420E030E040EA50E464
:1056F000C301B20181149104A104B10429F40E94F0
:1057000013AA87FF07C004C00E949DB0181614F4A6
:10571000460157012EA5222309F44CC08AA99BA952
:10572000ACA9BDA9892B8A2B8B2B61F0D701C601AF
:105730002AA93BA94CA95DA9821B930BA40BB50B0D
:10574000B7FD38C02EA93AAD4EAD23965FAD239775
:105750002B966FAD2B972F967FAD2F976B968FADB6
:105760006B9763969FAD63970E9476AE20E030E022
:1057700040EC5FE30E9413AA87FD31CFD701C60139
:10578000805A9541AF4FBF4F8AAB9BABACABBDAB23
:105790009EA92B969FAF2B97AAAD2F96AFAF2F97B1
:1057A000BEAD6B96BFAF6B972396EFAD2397639615
:1057B000EFAF639780915402882309F410CF8114CE
:1057C0009104A104B10429F4C22CD12EE02EF32CB3
:1057D000D5CEF8EECF1AF3E0DF0AE108F108C818D9
:1057E000D908EA08FB08F7FEFACEEECF66E970E0CA
:1057F00095CE0E943A7188E575D7882331F0179AC3
:105800008091DE048E7F8093DE0489E56BD7882348
:1058100031F0169A8091DE048D7F8093DE048AE554
:1058200061D7882331F0159A8091DE048B7F8093B5
:10583000DE0485E457D7882309F4D2CC0E94429035
:10584000CFCC68964EAD5FAD6897452B09F43AC151
:10585000E8964CAC5DAC6EAC7FACE897480E591E38
:105860006A1E7B1EE8962CAD3DAD4EAD5FADE89750
:10587000281B390B4A0B5B0BCA01B9012EA93FA9A2
:1058800048AD59AD0E9410AEA30192010E9441AEF5
:10589000D501C401820F931FA41FB51F8431910548
:1058A000A105B105FCF04C015D018C3E9105A105FF
:1058B000B1052CF06BEE862E912CA12CB12C40E87A
:1058C00084169104A104B104DCF08EEF90E0A0E016
:1058D000B0E088199909AA09BB098EAB9FABA8AFA4
:1058E000B9AF12C054E1852E912CA12CB12C24E12A
:1058F00030E040E050E02EAB3FAB48AF59AF04C0C2
:105900008EAA9FAAA8AEB9AEB501A40189E096E01F
:105910000E9486444EA95FA968AD79AD84E096E007
:105920000E9486446B964FAD6B9763965FAD63970D
:105930006F966FAD6F97A3967FADA3978DEF95E0B0
:105940000E94AF43A7964FADA797A8965FADA897C3
:10595000A9966FADA997AA967FADAA9786EF95E015
:105960000E94AF4368964EAD5FAD689743305105D6
:105970000CF4A8C06EA97FA988AD99AD0E9419AAA0
:1059800020E030E040E850E40E9478AA6B017C01FE
:105990006B962FAD6B9763963FAD63976F964FAD48
:1059A0006F97A3965FADA397A7966FADA797A8969D
:1059B0007FADA897A9968FADA997AA969FADAA97F4
:1059C0000E9476AE2BED3FE049E450E40E9478AAB5
:1059D00020E030E040E05FE30E9478AA9B01AC0148
:1059E000C701B6010E9453AF6B017C01C301B20134
:1059F0000E9419AA2FE632E143E85AE30E9478AAEE
:105A00002B013C01B701A60180EF95E00E94AF4356
:105A1000B301A2018AEE95E00E94AF432AE939E979
:105A200049E15FE3C701B6010E9478AA6B017C01DE
:105A30009B01AC010E9477AEA30192010E9453AF7B
:105A40002E966CAF7DAF8EAF9FAF2E97A3019201C4
:105A5000C701B6010E9478AA20E030E040E05EE392
:105A60000E9478AA62966CAF7DAF8EAF9FAF6297AF
:105A7000EAEDF5E084913F015FEF651A750A88232E
:105A800021F00E942774F301F5CFB701A60184ED40
:105A900095E00E94AF432E964CAD5DAD6EAD7FADEF
:105AA0002E978EEC95E00E94AF4362964CAD5DADB3
:105AB0006EAD7FAD629788EC95E00E94AF438AE0BF
:105AC0000E9427748EA99FA9A8ADB9AD880D991D14
:105AD000AA1DBB1DEEA5B595A79597958795E7FFE0
:105AE00003C08093F90307C0C357DF4FE881F981F2
:105AF000CD58D040808368962EAD3FAD68972F5F1C
:105B00003F4F68963FAF2EAF68973AAD6B963FAF69
:105B10006B974EAD63964FAF639723965FAD239718
:105B20006F965FAF6F9727968FAD2797A3968FAF2E
:105B3000A3974AA85BA86CA87DA891E0AF969FAFF9
:105B4000AF970C940D2580E00E94A78E01110C9454
:105B5000A5180ED5D090DC041092DD041092DC0460
:105B6000812C912C80EAA82E80E4B82E89829A821A
:105B7000AB82BC82F11020C08091190E90911A0E58
:105B8000A0911B0EB0911C0E0C94D818FF20A1F30D
:105B900080E090E0ADE1B3E48E8B9F8BA88FB98F4E
:105BA000BE016F5F7F4FCE014696F5D289829A8201
:105BB000AB82BC820C94ED1880E090E0ADE1B3E4E0
:105BC0008E8B9F8BA88FB98FBE016F5F7F4FCE01E9
:105BD0004696E1D289829A82AB82BC820C94EF18FD
:105BE000CB56DF4F0FB6F894DEBF0FBECDBFDF91AF
:105BF000CF911F910F91FF90EF90DF90CF90BF90CA
:105C0000AF909F908F907F906F905F904F903F905C
:105C10002F900895089590E0FC013197E231F1054D
:105C200008F04EC08827EE58FF4F8F4F0C9453B1A9
:105C3000809180008F7703C0809180008F7D80935A
:105C40008000089580918000877FF9CF84B58F7799
:105C500002C084B58F7D84BD08958091B0008F7798
:105C600003C08091B0008F7D8093B0000895809133
:105C700090008F7707C0809190008F7D03C0809146
:105C80009000877F8093900008958091A0008F7787
:105C900007C08091A0008F7D03C08091A000877F06
:105CA0008093A0000895809120018F7707C0809194
:105CB00020018F7D03C080912001877F8093200188
:105CC00008953FB7F89480911C0390911D03A09113
:105CD0001E03B0911F0326B5A89B05C02F3F19F0E6
:105CE0000196A11DB11D3FBFBA2FA92F982F88275C
:105CF000820F911DA11DB11DBC01CD0142E0660FB7
:105D0000771F881F991F4A95D1F70895CF92DF9288
:105D1000EF920F931F93CF93DF93CDB7DEB76097CA
:105D20000FB6F894DEBF0FBECDBFE090CE0CE1E120
:105D3000FEE080859185A285B38544815581668189
:105D40007781008111812281338109831A832B831A
:105D50003C834D835E836F83788789879A87AB877F
:105D6000BC871D861E861F86188AAE01475F5F4F5F
:105D7000BE016B5F7F4FCE0101960E94A672CE01DD
:105D80000D966C0109E512E02DE13EE0AE01475FA2
:105D90005F4FBE016B5F7F4F0C970E94266160963C
:105DA0000FB6F894DEBF0FBECDBFDF91CF911F912C
:105DB0000F91EF90DF90CF900895FF920F931F9374
:105DC000CF93DF93FC0120812B3319F1D091D406BE
:105DD000D530F8F4F62EBC01C0912F030C2F10E043
:105DE000F0E6CF9FC00111248E509B4F0E9479B1E5
:105DF000F801E451FB4FF082CF5FC53018F4C09337
:105E00002F0302C010922F03DF5FD093D40681E0EE
:105E100001C080E0DF91CF911F910F91FF90089515
:105E2000EF92FF920F931F93CF93DF93882329F074
:105E3000D091170DD095D17001C0D0E0662341F00C
:105E40001091170D11FB882780F911E0182701C068
:105E500010E0442341F0C091170DC2FB882780F960
:105E6000C1E0C82701C0C0E0D11102C0112319F060
:105E7000EEEDFEE103C0C111FBCF4FC084917F0165
:105E80009FEFE91AF90A882321F00E942774F7018D
:105E9000F5CFE2ECF8E084917F019FEFE91AF90A6F
:105EA000882321F00E942774F701F5CFDD2369F0E4
:105EB000E0ECF8E084917F019FEFE91AF90A88236A
:105EC00021F00E942774F701F5CF112361F0EEEB6A
:105ED000F8E084918F010F5F1F4F882321F00E940B
:105EE0002774F801F6CFC11103C0E4EBF8E00BC052
:105EF000ECEBF8E08491EF0121968823B1F30E9446
:105F00002774FE01F7CF8491EF012196882321F0B9
:105F10000E942774FE01F7CFC1E08C2FDF91CF9153
:105F20001F910F91FF90EF900895809197039091AA
:105F30009803A0919903B0919A038093590290938A
:105F40005A02A0935B02B0935C02809195039091FA
:105F5000960390934E0280934D02089580915902CA
:105F600090915A02A0915B02B0915C0280939703DA
:105F700090939803A0939903B0939A0380914D0254
:105F800090914E02909396038093950384E690E05F
:105F900090934E0280934D0208954F925F926F92BC
:105FA0007F928F929F92AF92BF92CF92DF92EF92A9
:105FB000FF920F931F93CF93DF93CDB7DEB72C974C
:105FC0000FB6F894DEBF0FBECDBF6D837E838F8387
:105FD000988729873A874B875C87470158013601A4
:105FE0008091590290915A02A0915B02B0915C029B
:105FF00089839A83AB83BC83D601CD90DD90ED90ED
:10600000FC9020E030E0A901C701B6010E9413AA6C
:10601000811106C0ECE5FBE1C590D590E590F490C8
:10602000A50194016091190E70911A0E80911B0EBA
:1060300090911C0E0E9413AA87FF11C0C0925902B2
:10604000D0925A02E0925B02F0925C028092190EAA
:1060500090921A0EA0921B0EB0921C0E57DEF30106
:10606000408051806280738020E030E0A901C3014C
:10607000B2010E9413AA811108C0409055025090AD
:106080005602609057027090580240925902509206
:106090005A0260925B0270925C028D819E81AF8198
:1060A000B8858093110E9093120EA093130EB093A7
:1060B000140E89859A85AB85BC858093150E9093C7
:1060C000160EA093170EB093180E20DEA5019401B2
:1060D0006091190E70911A0E80911B0E90911C0EFA
:1060E0000E949DB018168CF4C0925902D0925A02A8
:1060F000E0925B02F0925C028092190E90921A0E6E
:10610000A0921B0EB0921C0E01DE0E943A71898192
:106110009A81AB81BC818093590290935A02A093DB
:106120005B02B0935C022C960FB6F894DEBF0FBEF4
:10613000CDBFDF91CF911F910F91FF90EF90DF9036
:10614000CF90BF90AF909F908F907F906F905F9017
:106150004F900895CF92DF92EF92FF920F931F938B
:106160006A01E090190EF0901A0E00911B0E10912A
:106170001C0EFB012081318142815381FC01608131
:1061800071818281938109DF1F910F91FF90EF90C0
:10619000DF90CF900895CF92DF92EF92FF920F930E
:1061A0001F936B01FC01E080F18002811381E1E12A
:1061B000FEE0248135814681578160817181828131
:1061C0009381EBDE1F910F91FF90EF90DF90CF90C6
:1061D00008950F931F93CF93DF9394E0899FE0017D
:1061E00011248E010850124FFE01E052FB4FDE01D8
:1061F000A55FB24F2D913D914D915C916081718170
:10620000828193810E9477AEF801608371838283DB
:106210009383FE01E456F74F85919591A591B49132
:10622000FE01E95EFD4F80839183A283B383FE016B
:10623000E855F74F85919591A591B491C05CDD4FDC
:1062400088839983AA83BB83DF91CF911F910F919C
:106250000895CF92DF92EF92FF920F931F93CF9307
:10626000DF938091D406853008F003C10E94447901
:10627000AC0197FDFEC0982F2091250E3091260E7F
:106280008A3019F09D3009F0C2C010929403211594
:10629000310519F40E942F42E4CFF901EC5CFC4F68
:1062A00010821092260E1092250E24E333E0E901AD
:1062B00088812F5F3F4F8032D1F37E018E3409F009
:1062C00081C0209709F47EC064E878E0CE010E9486
:1062D000CAA911E0892B11F410E009C06EE470E046
:1062E000CE0104960E946EB1009709F07C014AE04D
:1062F00050E060E070E0C70101960E942BA7609318
:106300003003709331038093320390933303C09032
:10631000270ED090280EE090290EF0902A0E2FEF35
:10632000C21AD20AE20AF20A6C157D058E059F0593
:1063300029F0111103C081E997E02AC06AE270E0F8
:10634000CE010E948EB19C01009701F1982F9C1BF9
:1063500010E0992339F09150FE01E90FF11D808181
:106360001827F7CF4AE050E060E070E0C9010196DD
:106370000E942BA7012F10E020E030E0601771078A
:106380008207930779F085E698E002C08BE398E0F6
:10639000DF91CF911F910F91FF90EF90DF90CF9001
:1063A0000C94BFA28091300390913103A0913203ED
:1063B000B09133038093270E9093280EA093290E5B
:1063C000B0932A0E8091110281111CC067E470E025
:1063D000CE010E946EB10097A9F04AE050E060E063
:1063E00070E001960E942BA76430710558F4E4EC2C
:1063F000F7E08491EF012196882321F00E94277411
:10640000FE01F7CF61E084E393E0D7DC2ACF2F359C
:1064100031050CF026CF9C35C1F40E94447997FDDC
:1064200020CF2091940321111CCF2091250E309173
:10643000260EA9014F5F5F4F5093260E4093250E05
:10644000F901EC5CFC4F80830CCF9B3319F481E0A5
:106450008093940380919403811103CFC901019625
:106460009093260E8093250EF901EC5CFC4F40833F
:10647000F8CEDF91CF911F910F91FF90EF90DF90B9
:10648000CF900895BF92CF92DF92EF92FF920F9339
:106490001F93CF93DF93CDB7DEB76E970FB6F89407
:1064A000DEBF0FBECDBF60912D0370912E0361152D
:1064B000710561F14DE150E0CE0101967C010E9431
:1064C000BBA91E8EF7018F010E191F09B190BB20C9
:1064D00031F19AE0B912F7CF22C0B70184E897E012
:1064E0000E94C64482E20E9427748AE00E942774B8
:1064F000BB2059F10F5F1F4F80912D0390912E0308
:10650000080F191F10932E0300932D0381E0209193
:106510002D0330912E03232BD9F480E019C0F7010D
:10652000E00FF11F108260E0C70147DC882371F3A0
:10653000EEEDFEE184916F019FEFC91AD90A88231D
:1065400061F20E942774F601F5CF00E010E0DACF87
:106550006E960FB6F894DEBF0FBECDBFDF91CF9120
:106560001F910F91FF90EF90DF90CF90BF90089513
:106570000F931F93CF93DF93CDB7DEB72C970FB652
:10658000F894DEBF0FBECDBFE1E1FEE080859185CE
:10659000A285B3854481558166817781008111810F
:1065A0002281338109831A832B833C834D835E834D
:1065B0006F83788789879A87AB87BC87AE01475FEF
:1065C0005F4FBE016B5F7F4FCE0101960E94A672A6
:1065D0002DE13EE0AE01475F5F4FBE016B5F7F4F35
:1065E000CE0101960E941A8D2C960FB6F894DEBF4C
:1065F0000FBECDBFDF91CF911F910F910895809174
:106600002B0390912C03009731F04AE050E060E0BA
:1066100070E00C9453A860E070E0CB010895809185
:106620002B0390912C03009731F04AE050E060E09A
:1066300070E00C942BA760E070E0CB010895EFDFD1
:1066400097FD0AC0ECDF6F3F71058105910509F0E8
:106650002CF4E5DF862F089580E008958FEF0895EC
:1066600080912B0390912C03892B31F0E8DF91E08E
:10667000811103C090E001C091E0892F08950F932C
:106680001F93CF9380912B0390912C030097F1F0EF
:10669000FC018F01C1912C2F2F7D89F0C53411F0A1
:1066A000C536B9F7F801108260E070E00E94C4A519
:1066B000F801C083562F472F382F292F0BC060E0D9
:1066C00070E0CF911F910F910C94C4A550E040E071
:1066D00030E020E0652F742F832F922FCF911F91F0
:1066E0000F91089581548A3108F041C0A82FB0E07D
:1066F0004091ED0D5091EE0D6091EF0D7091F00D08
:1067000004C076956795579547958A95D2F740FFCF
:106710002EC0E091F60DF091F70DAD52B24F8C9175
:106720008823E9F0E80FF11D808190ED980F9A30F1
:1067300098F08E3211F481810CC08D3211F08B32C1
:1067400071F4818190ED980F9A3030F08E3239F4E7
:10675000828180538A3018F49E2F8F2F02C090E0E0
:1067600080E090932B0380932C0381E0089580E0D8
:106770000895B8DF882341F081E020912B03309108
:106780002C03232B09F480E00895EF92FF920F93DE
:106790001F93CF93DF937C0184E5EBDFD82F882311
:1067A00041F14DDFC82F181604F5EEEDFEE184919E
:1067B0008F010F5F1F4F882321F00E942774F8017B
:1067C000F6CF8DE40E942774B70180E090E04AE0A4
:1067D0000E9453786C2FCC0F770B89E898E00E94C9
:1067E000AD448AE00E94277408C08093FA03D0E089
:1067F00004C08091CE0C8093FA038D2FDF91CF914E
:106800001F910F91FF90EF90089580912A031E9998
:1068100002C0816001C08E7F80932A0380912A0389
:10682000379902C0806101C08F7E80932A038091D6
:106830002A031D9902C0826001C08D7F80932A03C4
:1068400080912A03029902C0806201C08F7D8093EB
:106850002A0380912A031C9902C0846001C08B7FA7
:1068600080932A0380912A03019902C0806401C0A9
:106870008F7B80932A039091290380912A03981794
:1068800031F097E0909328038093290309C0809109
:106890002803882329F0815080932803882349F016
:1068A0008091DD04811108C08091DF04811104C052
:1068B000089590932703F4CF8091C10C80FF16C0F8
:1068C0009091800C8091270390FF06C080FF0EC03E
:1068D0008091100E816005C084FF08C08091100E69
:1068E00080618093100E80E00E94A8A08091C10C6E
:1068F00081FF16C09091800C8091270391FF06C004
:1069000081FF0EC08091100E826005C085FF08C017
:106910008091100E80628093100E81E00E94A8A0EA
:106920008091C10C82FF1CC08091800C82FF0CC042
:106930008091DF048823A1F08091270382FF10C09B
:106940008091100E846007C08091270386FF08C0E5
:106950008091100E80648093100E82E00C94A8A0A9
:1069600008958091100E882319F01092100E08954A
:1069700086E797E00E9457908091CB04882341F0EE
:1069800040E150E063E370E08CEC94E00C94E1AD06
:10699000089581E08093CB04ECECF4E080E1DF012A
:1069A0001D928A95E9F7E8DF66E182E390E00C94B6
:1069B00002AE4F925F926F927F92AF92BF92CF9250
:1069C000DF92EF92FF92CF93DF93EB01FC016081A6
:1069D0007181828193812CE3C22ED12CE12CF12C88
:1069E000A70196010E941FAEB62EA72ECA01B901BB
:1069F000A70196010E941FAE6B017C01CA01B9017B
:106A000028E130E040E050E00E941FAE2B013C0145
:106A1000C9016DE671E00E943FB161157105D9F0C1
:106A2000AF92BF92DF92CF925F924F929F938F93DC
:106A30007F936F9382E697E09F938F93DF93CF933B
:106A40000E94E4A98DB79EB70E960FB6F8949EBF2C
:106A50000FBE8DBF61C00097C9F0AF92BF92DF92A9
:106A6000CF925F924F929F938F9382E597E09F938F
:106A70008F93DF93CF930E94E4A9EDB7FEB73C96C6
:106A80000FB6F894FEBF0FBEEDBF46C041145104CF
:106A900061047104B9F0AF92BF92DF92CF925F921E
:106AA0004F9286E497E09F938F93DF93CF930E945A
:106AB000E4A98DB79EB70A960FB6F8949EBF0FBE95
:106AC0008DBF2AC0C114D104E104F104A9F0AF9232
:106AD000BF92DF92CF928EE397E09F938F93DF93E5
:106AE000CF930E94E4A9EDB7FEB738960FB6F8949D
:106AF000FEBF0FBEEDBF10C0AF92BF928AE397E01A
:106B00009F938F93DF93CF930E94E4A90F900F90F0
:106B10000F900F900F900F90DF91CF91FF90EF901B
:106B2000DF90CF90BF90AF907F906F905F904F902D
:106B300008951F920F920FB60F9211240BB60F9269
:106B40002F933F934F935F936F937F938F939F9375
:106B5000AF93BF93EF93FF93E0910E02F0910F027A
:106B60001995FF91EF91BF91AF919F918F917F9177
:106B70006F915F914F913F912F910F900BBE0F90AE
:106B80000FBE0F901F9018951F920F920FB60F9285
:106B900011240BB60F922F933F934F935F936F93F4
:106BA0007F938F939F93AF93BF93EF93FF93E09166
:106BB0000C02F0910D021995FF91EF91BF91AF91E9
:106BC0009F918F917F916F915F914F913F912F9105
:106BD0000F900BBE0F900FBE0F901F9018951F9235
:106BE0000F920FB60F9211240BB60F922F933F9373
:106BF0004F935F936F937F938F939F93AF93BF93C5
:106C0000EF93FF93E0910202F09103021995FF9137
:106C1000EF91BF91AF919F918F917F916F915F9114
:106C20004F913F912F910F900BBE0F900FBE0F9081
:106C30001F9018951F920F920FB60F9211240BB64A
:106C40000F922F933F934F935F936F937F938F9305
:106C50009F93AF93BF93EF93FF93E0910002F09166
:106C600001021995FF91EF91BF91AF919F918F9183
:106C70007F916F915F914F913F912F910F900BBE3C
:106C80000F900FBE0F901F9018951F920F920FB686
:106C90000F9211240BB60F922F933F934F935F9354
:106CA0006F937F938F939F93AF93BF93EF93FF93D4
:106CB000E0910A02F0910B021995FF91EF91BF91BB
:106CC000AF919F918F917F916F915F914F913F9184
:106CD0002F910F900BBE0F900FBE0F901F90189525
:106CE0001F920F920FB60F9211240BB60F922F9393
:106CF0003F934F935F936F937F938F939F93AF9344
:106D0000BF93EF93FF93E0910802F0910902199568
:106D1000FF91EF91BF91AF919F918F917F916F9173
:106D20005F914F913F912F910F900BBE0F900FBE2F
:106D30000F901F9018951F920F920FB60F9211246B
:106D40000BB60F922F933F934F935F936F937F9365
:106D50008F939F93AF93BF93EF93FF93E0910602BE
:106D6000F09107021995FF91EF91BF91AF919F911B
:106D70008F917F916F915F914F913F912F910F90E4
:106D80000BBE0F900FBE0F901F9018951F920F9281
:106D90000FB60F9211240BB60F922F933F934F9380
:106DA0005F936F937F938F939F93AF93BF93EF9373
:106DB000FF93E0910402F09105021995FF91EF9184
:106DC000BF91AF919F918F917F916F915F914F9103
:106DD0003F912F910F900BBE0F900FBE0F901F9001
:106DE0001895CF93DF93282F30E0F901EC51F14E45
:106DF0008491F901EC5FFF4DD491F901E254F04E1A
:106E0000C491CC2391F081110E940B2EEC2FF0E065
:106E1000EE0FFF1FE15EF84FA591B491EC91ED23C9
:106E200081E090E021F480E002C080E090E0DF911A
:106E3000CF9108951F93CF93DF93282F30E0F9016E
:106E4000EC51F14E8491F901EC5FFF4DD491F901C1
:106E5000E254F04EC491CC23C9F0162F81110E9448
:106E60000B2EEC2FF0E0EE0FFF1FE657F04EA59132
:106E7000B4918FB7F894111105C09C91ED2FE09556
:106E8000E92302C0EC91ED2BEC938FBFDF91CF9102
:106E90001F9108951F920F920FB60F9211240BB6F7
:106EA0000F922F933F934F935F936F937F938F93A3
:106EB0009F93AF93BF93EF93FF93809123039091A0
:106EC0002403A0912503B0912603892B8A2B8B2BB9
:106ED00059F180912203E0912003F09121039081E8
:106EE000892780838091230390912403A091250317
:106EF000B0912603181619061A061B060CF055C089
:106F00008091230390912403A0912503B09126033F
:106F10000197A109B1098093230390932403A093BF
:106F20002503B093260341C080911002E9E3F7E006
:106F3000E4919FEF90931002E230C9F050F4EE23F9
:106F400099F0E13081F590916F009D7F90936F00F3
:106F50002AC0E43019F1E0F0E53029F59091730092
:106F60009D7F909373001FC010926E001CC0909183
:106F700070009D7F9093700091E09093B00090918D
:106F8000B100987F94609093B1001092B3000BC051
:106F9000909171009D7F9093710005C09091720057
:106FA0009D7F9093720060E045DFFF91EF91BF916C
:106FB000AF919F918F917F916F915F914F913F9191
:106FC0002F910F900BBE0F900FBE0F901F90189532
:106FD0001F93CF93DF93182FEB010E94D3A120972B
:106FE00011F460E004C0CF3FD10531F461E0812F9E
:106FF000DF91CF911F911ECFE12FF0E0EC51F14EC8
:10700000E4914E2F50E0FA013197E231F10508F09A
:107010009DC08827EC57FF4F8F4F0C9453B184B518
:10702000806884BDC7BD97C084B5806284BDC8BD7B
:1070300092C080918000806880938000D093890006
:10704000C093880088C08091800080628093800017
:10705000D0938B00C0938A007EC0809180008860AE
:1070600080938000D0938D00C0938C0074C0809179
:10707000B00080688093B000C093B3006CC0809172
:10708000B00080628093B000C093B40064C080916F
:107090009000806880939000D0939900C0939800EE
:1070A0005AC080919000806280939000D0939B00A2
:1070B000C0939A0050C080919000886080939000A7
:1070C000D0939D00C0939C0046C08091A000806832
:1070D0008093A0008091A0008F7B8093A000D0932C
:1070E000A900C093A80037C08091A000806280935F
:1070F000A000D093AB00C093AA002DC08091A00047
:1071000088608093A000D093AD00C093AC0023C0F2
:1071100080912001806880932001D0932901C09341
:10712000280119C080912001806280932001D093B2
:107130002B01C0932A010FC08091200188608093A9
:107140002001D0932D01C0932C0105C0C038D1057A
:107150000CF04CCF46CFDF91CF911F9108958F92C5
:107160009F92AF92BF92CF92DF92EF92FF926B010C
:107170007C010E94612E4B015C01C114D104E10429
:10718000F104F1F00E94612EDC01CB01881999090C
:10719000AA09BB09883E9340A105B10570F321E01F
:1071A000C21AD108E108F10888EE880E83E0981E23
:1071B000A11CB11CC114D104E104F10419F7DDCF05
:1071C000FF90EF90DF90CF90BF90AF909F908F9007
:1071D00008952FB7F8946091180370911903809166
:1071E0001A0390911B032FBF08950F931F93809153
:1071F000CA04813011F4EDDF08C06091C2047091BF
:10720000C3048091C4049091C5040091C6041091F8
:10721000C7042091C8043091C904601B710B820B14
:10722000930B28EE33E040E050E00E941FAE8091C7
:10723000BE049091BF04A091C004B091C104BC01F0
:10724000CD01620F731F841F951F1F910F91089529
:10725000CF92DF92EF92FF920F931F938091CA0417
:107260008150823010F080E058C01092CA04B1DF23
:107270006093C2047093C3048093C4049093C504C4
:107280008091CE049091CF0401969093CF04809387
:10729000CE04C090EA0CD090EB0CE090EC0CF09097
:1072A000ED0CA3DF6093EA0C7093EB0C8093EC0C75
:1072B0009093ED0C0091D0041091D1042091D20450
:1072C0003091D3040C191D092E093F09DC01CB01B3
:1072D000800F911FA21FB31F8093D0049093D104FD
:1072E000A093D204B093D30480DF0091D404109112
:1072F000D5042091D6043091D70406171707280724
:10730000390748F472DF6093D4047093D5048093F6
:10731000D6049093D70430DB81E01F910F91FF904A
:10732000EF90DF90CF9008951F920F920FB60F92BB
:1073300011242F933F938F939F93AF93BF9380918B
:10734000180390911903A0911A03B0911B03309177
:10735000170323E0230F2D3720F40196A11DB11D43
:1073600005C026E8230F0296A11DB11D2093170327
:107370008093180390931903A0931A03B0931B03EF
:1073800080911C0390911D03A0911E03B0911F03D7
:107390000196A11DB11D80931C0390931D03A09322
:1073A0001E03B0931F03BF91AF919F918F913F91A7
:1073B0002F910F900FBE0F901F9018954F925F92D4
:1073C0006F927F928F929F92AF92BF92CF92DF92F5
:1073D000EF92FF92CF93DF93CDB7DEB72C970FB626
:1073E000F894DEBF0FBECDBF8091FB039091FC03EC
:1073F000A091FD03B091FE0389839A83AB83BC8384
:107400006091FF0370910004072E000C880B990B0C
:107410000E9419AA29813A814B815C810E9476AE33
:107420006B017C016093C9037093CA038093CB0303
:107430009093CC032091410D3091420D4091430D2A
:107440005091440D0E9478AA6D837E838F83988724
:107450006093C5037093C6038093C7039093C803DA
:107460002091C1033091C2034091C3035091C403E2
:10747000C701B6010E9477AE4B015C016093C10366
:107480007093C2038093C3039093C40320913D0D76
:1074900030913E0D40913F0D5091400D0E9478AAD1
:1074A00069877A878B879C876093BD037093BE033F
:1074B0008093BF039093C00320ED3CEC4CE45DE36C
:1074C0006091390D70913A0D80913B0D90913C0D7A
:1074D0000E9478AA2B013C012091B9033091BA0394
:1074E0004091BB035091BC0369817A818B819C815F
:1074F0000E9476AE9B01AC01C301B2010E9478AA42
:107500002B013C0123E333E343E75FE36091B503E1
:107510007091B6038091B7039091B8030E9478AA46
:107520009B01AC01C301B2010E9477AE2B013C016B
:107530006093B5037093B6038093B7039093B80339
:1075400089819A81AB81BC818093B9039093BA03FE
:10755000A093BB03B093BC0329853A854B855C851A
:107560006D817E818F8198850E9477AEA301920103
:107570000E9476AE2B013C0120E030E04FE753E45F
:107580000E949DB020E030E0A9011816ACF4C701BC
:10759000B6010E949DB018166CF5A7019601C501B1
:1075A000B4010E9476AE6093C1037093C2038093CE
:1075B000C3039093C4031EC0C301B2010E9413AA67
:1075C00087FF22C020E030E0A901C701B6010E9478
:1075D00013AA87FF16C0A7019601C501B4010E9436
:1075E00076AE6093C1037093C2038093C3039093FC
:1075F000C40307C0412C512C8FE7682E83E4782EFA
:1076000003C0412C512C3201C301B2012C960FB69C
:10761000F894DEBF0FBECDBFDF91CF91FF90EF900A
:10762000DF90CF90BF90AF909F908F907F906F90A2
:107630005F904F9008952F923F924F925F926F927A
:107640007F928F929F92AF92BF92CF92DF92EF92F2
:10765000FF92CF93DF9300D01F92CDB7DEB760903B
:1076600001047090020480900F0490901004A09088
:107670001104B0901204B301072C000C880B990B75
:107680000E9419AAA50194010E9476AE6B017C01AB
:107690006093B1037093B2038093B3039093B403E8
:1076A00020ED3CEC4CE45DE36091450D7091460D9E
:1076B0008091470D9091480D0E9478AA1B012C01E2
:1076C0002091AD033091AE034091AF035091B003D0
:1076D000C501B4010E9476AE9B01AC01C201B101AB
:1076E0000E9478AA1B012C0123E333E343E75FE305
:1076F0006091A9037091AA038091AB039091AC03B0
:107700000E9478AA9B01AC01C201B1010E9477AE30
:1077100069837A838B839C836093A9037093AA0304
:107720008093AB039093AC038092AD039092AE0331
:10773000A092AF03B092B00320E030E040E251E409
:10774000C701B6010E949DB0181624F481E0809311
:10775000A80389C020E030E040E251ECC701B60147
:107760000E9413AA87FD02C0672821F481E080935C
:10777000A8039DC08091A803882351F01092A40310
:107780001092A5031092A6031092A7031092A803CB
:1077900020914D0D30914E0D40914F0D5091500D57
:1077A000C701B6010E9478AA2B013C016093A00397
:1077B0007093A1038093A2039093A3032091A40349
:1077C0003091A5034091A6035091A703C701B601CC
:1077D0000E9477AE4B015C016093A4037093A503F4
:1077E0008093A6039093A7032091490D30914A0DF1
:1077F00040914B0D50914C0D0E9478AA9B01AC0119
:1078000060939C0370939D0380939E0390939F03CA
:10781000C301B2010E9477AE29813A814B815C811C
:107820000E9476AE2B013C0120E030E04FE753E4AC
:107830000E949DB020E030E0A9011816DCF4C701D9
:10784000B6010E949DB0181674F4A7019601C501F7
:10785000B4010E9476AE6093A4037093A503809355
:10786000A6039093A703412C512C8FE7682E83E445
:10787000782E20C0C301B2010E9413AA87FF1AC04C
:1078800020E030E0A901C701B6010E9413AA87FFDA
:107890000EC0A7019601C501B4010E9476AE6093A7
:1078A000A4037093A5038093A6039093A703412C90
:1078B000512C3201C301B2010F900F900F900F9025
:1078C000DF91CF91FF90EF90DF90CF90BF90AF907E
:1078D0009F908F907F906F905F904F903F902F90F0
:1078E00008954F925F926F927F928F929F92AF9284
:1078F000BF92CF92DF92EF92FF920F931F93CF939D
:10790000DF93CDB7DEB768970FB6F894DEBF0FBE32
:10791000CDBF8C015B014A01FC01EE5BFF4F608132
:107920007181828193810E9417AA6B017C01D5012C
:107930002D913D914D915C910E9478AA0E943DAF9E
:107940000E94C0AF69877A878B879C87F40120816A
:10795000318142815381C701B6010E9478AA0E94F9
:107960003DAF0E94C0AF6D877E878F87988B29853A
:107970003A854B855C85283731054105510540F432
:1079800088E790E0A0E0B0E089879A87AB87BC8762
:107990002D853E854F85588928373105410551058C
:1079A00040F488E790E0A0E0B0E08D879E87AF8745
:1079B000B88B9801225B3F4FD9018D919D910D901D
:1079C000BC91A02D89839A83AB83BC83BC01CD017C
:1079D0000E9419AA2B013C0169857A858B859C85BB
:1079E0000E9417AA698B7A8B8B8B9C8B20E030E0EE
:1079F000A901C301B2010E9413AA882329F1A7019A
:107A00009601C701B6010E9478AA4B015C01298941
:107A10003A894B895C89CA01B9010E9478AA9B0105
:107A2000AC01C501B4010E9476AE4B015C01A3011B
:107A30009201C301B2010E9477AE9B01AC01C50166
:107A4000B4010E9453AF03C060E070E0CB010E941C
:107A50003DAF0E94C0AF6D837E838F83988769811D
:107A60007A818B819C8190958095709561957F4FEF
:107A70008F4F9F4F0E9419AA4B015C016D857E8537
:107A80008F8598890E9417AA69837A838B839C8348
:107A900020E030E0A901C501B4010E9413AA8823A7
:107AA00049F129813A814B815C81CA01B9010E9467
:107AB00078AA6D8B7E8B8F8B988FA7019601C7015B
:107AC000B6010E9478AA9B01AC016D897E898F89DD
:107AD000988D0E9476AE6B017C01A5019401C501D1
:107AE000B4010E9477AE9B01AC01C701B6010E94B0
:107AF00053AF03C060E070E0CB010E94ECAFF8012F
:107B000085A096A0A7A0B0A4750164012D813E8137
:107B10004F815885C21AD30AE40AF50A0E94C0AF01
:107B2000C61AD70AE80AF90AF7FE73C020E030E067
:107B3000A901C301B2010E9413AA882309F443C01A
:107B4000A3019201C301B2010E9477AE6B017C01D7
:107B5000C501B4010E9417AA9B01AC01C701B6017F
:107B60000E9478AA6B017C0129893A894B895C893A
:107B7000CA01B9010E9478AA9B01AC01C701B601F4
:107B80000E9476AE6B017C0129813A814B815C8138
:107B9000CA01B9010E9478AA9B01AC01C701B601D4
:107BA0000E9477AE6B017C0120E030E040E850E4B9
:107BB000C301B2010E9478AA9B01AC01C701B601C2
:107BC0000E9453AF03C060E070E0CB010E943DAF64
:107BD0007B016C0120E030E0A9010E949DB01816E5
:107BE00024F0E12CF12CC12CD12CB701C6010E944C
:107BF000C0AF6D837E838F83988786169706A8060D
:107C0000B90620F48D829E82AF82B886C12CD12C19
:107C100076018D819E81AF81B885F80182A793A7F7
:107C2000A4A7B5A7C80ED91EEA1EFB1EC6A6D7A6D6
:107C3000E0AAF1AAEA5BFF4F29853A854B855C856E
:107C4000208331834283538334968D859E85AF850F
:107C5000B88980839183A283B38368960FB6F89422
:107C6000DEBF0FBECDBFDF91CF911F910F91FF906F
:107C7000EF90DF90CF90BF90AF909F908F907F90CC
:107C80006F905F904F9008954F925F926F927F92A6
:107C90008F929F92AF92BF92CF92DF92EF92FF921C
:107CA0000F931F93CF93DF933C01B0E2A0E06A2FC4
:107CB00070E0AB014B0F511D559547954A1711F0D8
:107CC0004B130BC0E6E4F9E065917491072E000CAC
:107CD000880B990B0E9419AA62C0CA010197880FEC
:107CE000991F880F991FFC01E853F74F05911491D4
:107CF0009A01220F331F220F331FF901E853F74F68
:107D0000C591D4916016710614F4B42FD2CFA42F6C
:107D1000C615D7050CF4CBCF8653974FFC01E590E1
:107D2000F490F901E653F74FC590D490B7010F2CAA
:107D3000000C880B990B0E9419AA4B015C01B3013E
:107D4000601B710B072E000C880B990B0E9419AA5F
:107D50002B013C01B6016E197F09072E000C880B20
:107D6000990B0E9419AA9B01AC01C301B2010E94A8
:107D700078AA6B017C01C01BD10BBE01DD0F880B03
:107D8000990B0E9419AA9B01AC01C701B6010E9480
:107D900053AF9B01AC01C501B4010E9477AEDF91E6
:107DA000CF911F910F91FF90EF90DF90CF90BF90F8
:107DB000AF909F908F907F906F905F904F900895BD
:107DC0000F930FB70F9300916E000B7F00936E001F
:107DD00078940F930BB70F930CB70F921F922F93BA
:107DE0003F934F935F936F937F938F939F93AF9343
:107DF000BF93EF93FF93112406D2FF91EF91BF91B0
:107E0000AF919F918F917F916F915F914F913F9132
:107E10002F911F900F900CBF0F910BBF0F9104601B
:107E2000F89400936E000F910FBF0F911895CF92A9
:107E3000DF92EF92FF92C090FB03D090FC03E090A2
:107E4000FD03F090FE038091FF03909100040897DA
:107E5000BC01990F880B990B0E9419AA9B01AC01D8
:107E6000C701B6010E9413AA87FF1EC020E030E0C0
:107E700040E050E4C701B6010E9477AE0E94C0AF57
:107E80007093E2036093E103A4D9DC01CB01805A33
:107E90009541AF4FBF4F8093DD039093DE03A093D6
:107EA000DF03B093E00308C01092DD031092DE03FD
:107EB0001092DF031092E003FF90EF90DF90CF90DD
:107EC0000895CF92DF92EF92FF92C0900F04D0906E
:107ED0001004E0901104F09012048091010490913C
:107EE00002040D97BC01990F880B990B0E9419AAE7
:107EF0009B01AC01C701B6010E9413AA87FF1EC0F7
:107F000020E030E040E050E4C701B6010E9477AEC7
:107F10000E94C0AF7093DC036093DB035AD9DC018D
:107F2000CB01805E914BAF4FBF4F8093D7039093AF
:107F3000D803A093D903B093DA0308C01092D703F3
:107F40001092D8031092D9031092DA03FF90EF90A9
:107F5000DF90CF900895109202041092010480E007
:107F6000B0DF109200041092FF0361DF71D910920C
:107F700002041092010480E0A4DF1092F8037598C7
:107F8000109200041092FF031092F903A59808952F
:107F90004F925F926F927F928F929F92AF92BF9219
:107FA000CF92DF92EF92FF920F931F93CF93DF93C5
:107FB0003C01BAE3A0E06A2F70E0AB014B0F511D0A
:107FC000559547954A1711F04B130BC0EDE9FAE0B0
:107FD00065917491072E000C880B990B0E9419AAC9
:107FE00062C0CA010197880F991F880F991FFC0171
:107FF000E954F64F059114919A01220F331F220F75
:10800000331FF901E954F64FC591D49160167106FA
:1080100014F4B42FD2CFA42FC615D7050CF4CBCFB0
:108020008754964FFC01E590F490F901E754F64F20
:10803000C590D490B7010F2C000C880B990B0E94AF
:1080400019AA4B015C01B301601B710B072E000CD8
:10805000880B990B0E9419AA2B013C01B6016E19DD
:108060007F09072E000C880B990B0E9419AA9B010F
:10807000AC01C301B2010E9478AA6B017C01C01B54
:10808000D10BBE01DD0F880B990B0E9419AA9B0131
:10809000AC01C701B6010E9453AF9B01AC01C50101
:1080A000B4010E9477AEDF91CF911F910F91FF90A5
:1080B000EF90DF90CF90BF90AF909F908F907F9088
:1080C0006F905F904F90089560E08091E5039091EC
:1080D000E603DADD60930F047093100480931104BB
:1080E000909312048091E3039091E40351DF609335
:1080F000FB037093FC038093FD039093FE03A8950C
:108100001092E7030895CF92DF92FF920F931F938F
:10811000CF93DF931F921F92CDB7DEB7F82E8A015F
:1081200080911102882309F444C0ECE4FFE18491BA
:108130006F019FEFC91AD90A882341F069837A83B6
:108140000E942774F60169817A81F1CFFB01849145
:108150006F019FEFC91AD90A882321F00E94277462
:10816000F601F5CFEDE4F9E084916F019FEFC91AB4
:10817000D90A882321F00E942774F601F5CFF7FC75
:108180000BC06F2DFF0C770B880B990B0E94B978F1
:108190008AE00E9427740DC0E8E4F9E084916F0141
:1081A0009FEFC91AD90A882321F00E942774F6018B
:1081B000F5CF80919B03811108C01092110281E0DC
:1081C00080939B03C8010E9457900F900F90DF91FE
:1081D000CF911F910F91FF90DF90CF90BCCE8F3F3A
:1081E00019F042ED5AE002C042EE5AE063EF7AE045
:1081F0008ACF8F3F19F04FE95AE002C04FEA5AE0A8
:1082000060EC7AE080CF0F931F93CF93DF93809140
:1082100016028F3790F08F579091F8039093F703E1
:10822000992311F0759A01C075989091F903909374
:10823000F603992359F0A59A0AC09091F70389177C
:1082400008F075989091F603891708F0A5988F5F4C
:10825000809316029091F50381E089278093F503BE
:1082600080911502853018F4C1E0C80F01C0C0E04C
:10827000823009F4ACC048F48823F9F0813009F069
:10828000DAC010927B0080E4B8C0843009F4BDC02D
:1082900008F4B0C0853009F0CEC09091F40391117C
:1082A00002C08093F4038091F40381508093F4031F
:1082B000882309F4C0C0C5E0BEC0809114028F5F5E
:1082C00080311CF480931402B6C010921402809185
:1082D000E703811113C08091EA039091EB0390931F
:1082E000E6038093E5038091E8039091E90390937E
:1082F000E4038093E30381E08093E7038AE0EAEEFE
:10830000F3E0DF011D928A95E9F71092E9031092DC
:10831000E8030091E5031091E60311950195110919
:10832000D1E08091F803811101C0D0E08091BA04BE
:108330009091BB049195819591098017910744F420
:10834000DD2331F04FE95AE060EC7AE080E0DBDEDB
:1083500080912D0290912E02919581959109081797
:10836000190744F4DD2331F042ED5AE063EF7AE07F
:1083700080E0C9DE11E08091F903811101C010E0B5
:108380002091E3033091E4038091B8049091B90403
:108390008217930744F0112331F04FEA5AE060EC62
:1083A0007AE08FEFB0DE20912B0230912C02809189
:1083B000E3039091E40382179307ECF11123D9F1C1
:1083C00042EE5AE063EF7AE08FEF9DDE34C0809199
:1083D0007A0086FD2DC080917800909179002091DF
:1083E000EA033091EB03820F931F9093EB0380938A
:1083F000EA0321C010927B0082E480937C0080918C
:108400007A00806480937A0016C080917A0086FD9D
:1084100011C080917800909179002091E80330910B
:10842000E903820F931F9093E9038093E80303C04D
:10843000C2E001C0C4E0C09315020E9405348091DF
:10844000B00D9091B10D009729F001979093B10D67
:108450008093B00DDF91CF911F910F9108958F926E
:108460009F92AF92BF92CF92DF92EF92FF920F93C3
:10847000CF93DF9300D01F92CDB7DEB78091B20DBE
:108480008111F2C08091E703811110C00F900F900D
:108490000F900F90DF91CF910F91FF90EF90DF90B1
:1084A000CF90BF90AF909F908F9008950DDE0E9467
:1084B000E9384B015C018091120290911302181669
:1084C00019060CF000C101979093130280931202D9
:1084D0006091010470910204072E000C880B990B27
:1084E0000E9419AA69837A838B839C833EE1E32EE1
:1084F000F12C00E09E012F5F3F4F4FE054E063ED11
:1085000073E082ED93E00E94F2A1C0900F04D0903E
:108510001004E0901104F09012048091BC0490913A
:10852000BD04BC01990F880B990B0E9419AA9B01ED
:10853000AC01C701B6010E949DB018160CF4A9C089
:1085400060E06093F8038091D7039091D803A091E5
:10855000D903B091DA030097A105B10521F1A50176
:108560009401281B390B4A0B5B0B57FD1CC0609113
:10857000DB037091DC0380E090E00E9417AA9B016E
:10858000AC0160910F0470911004809111049091DE
:1085900012040E9413AA87FFB7C04DE859E06FE9A3
:1085A00079E080E0B0DD8091DD039091DE03A09161
:1085B000DF03B091E0030097A105B10511F1881A1E
:1085C000990AAA0ABB0AB7FC1CC06091E10370912A
:1085D000E20380E090E00E9417AA9B01AC01609149
:1085E000FB037091FC038091FD039091FE030E94B8
:1085F00013AA87FF87C04BE659E06EE779E08FEF5B
:1086000082DD6091FF0370910004072E000C880B3F
:10861000990B0E9419AA69837A838B839C839AE0C1
:10862000E92EF12C0FEF9E012F5F3F4F4BEF53E0F0
:108630006DEC73E081ED93E00E94F2A18090FB036A
:108640009090FC03A090FD03B090FE0320E030E08A
:1086500040EA50E4C501B4010E949DB087FF08C004
:1086600060E06093F90312CF8EEA99E00E94579080
:1086700020E030E046E153E4C501B4010E9413AAB2
:10868000181674F30E94DE390E94BBAF759567958A
:10869000E8CF60912F0270913002072E000C880BFA
:1086A000990B0E9419AA9B01AC01C701B6010E9457
:1086B00013AA87FF45CF80E00E941B3B0E94BBAFFF
:1086C000759567953ECFC0900F04D0901004E09050
:1086D0001104F090120420E030E848E953E4C701A7
:1086E000B6010E949DB0181694F020E030E040EAF8
:1086F00050E4C701B6010E9413AA87FFE9CE80E0CB
:108700006EDDE6CE94DB7DCF80E0DBDB4CCF80E01E
:1087100070DDC0900F04D0901004E0901104F09030
:108720001204E3CFCF92DF92EF92FF92CF93DF93C9
:108730006A017B01FC018491EF012196882321F0DD
:108740000E942774FE01F7CF4AE0C701B601DF910E
:10875000CF91FF90EF90DF90CF900C945378CF9211
:10876000DF92EF92FF92CF93DF936A017B01FC01CE
:108770008491EF012196882321F00E942774FE0145
:10878000F7CF42E0C701B601DF91CF91FF90EF90A4
:10879000DF90CF900C94D378EF92FF920F931F93BA
:1087A000CF93DF931F92CDB7DEB78C017B0180E2C0
:1087B00049830E94277449814F3F11F084E501C02D
:1087C00082E40E9427748AE30E942774F801608182
:1087D00071818281938142E00E94D378F7014081C8
:1087E00051816281738185E09BE0B9DF62E070E0D6
:1087F00080E090E00F90DF91CF911F910F91FF905B
:10880000EF900C94AF380F931F93CF93DF93CDB7B6
:10881000DEB728970FB6F894DEBF0FBECDBF6091CC
:10882000010470910204072E000C880B990B0E9422
:1088300019AA6D837E838F83988780910F0490910E
:108840001004A0911104B091120489839A83AB8320
:10885000BC834DEFBE016B5F7F4FCE0101969CDF65
:108860006091FF0370910004072E000C880B990B98
:108870000E9419AA6D837E838F8398878091FB0362
:108880009091FC03A091FD03B091FE0389839A832C
:10889000AB83BC834FEFBE016B5F7F4FCE01019670
:1088A0007BDFEDE0FBE084918F010F5F1F4F88239A
:1088B00021F00E942774F801F6CFE091FA03F0E06E
:1088C000E850FC4F608170E080E090E00E94B97851
:1088D000E8E0FBE084918F010F5F1F4F882321F0B8
:1088E0000E942774F801F6CF6091F90370E080E0F0
:1088F00090E00E94B97828960FB6F894DEBF0FBEBC
:10890000CDBFDF91CF911F910F9108950F931F93CA
:10891000CF93DF9300D01F92CDB7DEB7FC018491D7
:108920008F010F5F1F4F882361F049835A836B8348
:108930007C830E942774F80149815A816B817C8174
:10894000EECFCB01BA010F900F900F900F90DF91F7
:10895000CF911F910F910C94B9780F931F93CF93E0
:10896000DF938B01FC018491EF012196882321F094
:108970000E942774FE01F7CFB801110F880B990BE5
:10898000DF91CF911F910F910C94B9780F931F93A2
:10899000CF93DF931F921F92CDB7DEB7FC01849176
:1089A0008F010F5F1F4F811102C08B0108C06983C7
:1089B0007A830E942774F80169817A81F0CFF801E7
:1089C00081918F01882319F00E942774F8CF0F90AE
:1089D0000F90DF91CF911F910F9108954F925F9269
:1089E0006F927F928F929F92AF92BF92CF92DF92BF
:1089F000EF92FF92CF93DF93CDB7DEB728970FB6F4
:108A0000F894DEBF0FBECDBF2496AEADBFAD2497A8
:108A10008D919D910D90BC91A02D89839A83AB83FC
:108A2000BC832296EEADFFAD2297C080D180E2805C
:108A3000F380AEADBFAD8D909D90AD90BC902E8D6E
:108A40003F8D48A159A1C501B4010E9478AA2B010C
:108A50003C012AA53BA54CA55DA5C701B6010E9416
:108A600078AA9B01AC01C301B2010E9477AE2B0131
:108A70003C012EA93FA948AD59AD69817A818B810E
:108A80009C810E9478AA9B01AC01C301B2010E94A3
:108A900077AE6D837E838F8398872AA13BA14CA1FB
:108AA0005DA1C501B4010E9478AA2B013C012EA54D
:108AB0003FA548A959A9C701B6010E9478AA9B0100
:108AC000AC01C301B2010E9477AE2B013C012AAD7B
:108AD0003BAD4CAD5DAD69817A818B819C810E94FB
:108AE00078AA9B01AC01C301B2010E9477AE2B01B1
:108AF0003C012A8D3B8D4C8D5D8DC501B4010E94DA
:108B000078AA4B015C012EA13FA148A559A5C70138
:108B1000B6010E9478AA9B01AC01C501B4010E9474
:108B200077AE6B017C012AA93BA94CA95DA969819B
:108B30007A818B819C810E9478AA9B01AC01C7013C
:108B4000B6010E9477AEEEADFFAD60837183828384
:108B500093838D819E81AF81B8852296EEADFFAD66
:108B6000229780839183A283B3832496AEADBFAD59
:108B700024974D925D926D927C92139728960FB632
:108B8000F894DEBF0FBECDBFDF91CF91FF90EF9085
:108B9000DF90CF90BF90AF909F908F907F906F901D
:108BA0005F904F9008954F925F926F927F928F9255
:108BB0009F92AF92BF92CF92DF92EF92FF920F936C
:108BC0001F93CF93DF9300D01F92CDB7DEB78C01F8
:108BD000DC014D905D906D907C90139714968D9074
:108BE0009D90AD90BC90179718968D919D910D908A
:108BF000BC91A02D89839A83AB83BC83A30192018E
:108C0000C301B2010E9478AA6B017C01A501940105
:108C1000C501B4010E9478AA9B01AC01C701B6014D
:108C20000E9477AE6B017C0129813A814B815C8186
:108C3000CA01B9010E9478AA9B01AC01C701B60123
:108C40000E9477AE0E94E2B09B01AC0160E070E050
:108C500080E89FE30E9453AF6B017C019B01AC0154
:108C6000C301B2010E9478AAF801608371838283F4
:108C70009383A7019601C501B4010E9478AAD80187
:108C800014966D937D938D939C931797A7019601EE
:108C900069817A818B819C810E9478AAF801608722
:108CA0007187828793870F900F900F900F90DF91BD
:108CB000CF911F910F91FF90EF90DF90CF90BF90D9
:108CC000AF909F908F907F906F905F904F9008959E
:108CD0002F923F924F925F926F927F928F929F92CC
:108CE000AF92BF92CF92DF92EF92FF920F931F93BA
:108CF000CF93DF93CDB7DEB765970FB6F894DEBF9D
:108D00000FBECDBF1092150E1092160E1092170EB8
:108D10001092180E1092110E1092120E1092130E45
:108D20001092140E0E94B832E1EAFBE124912D8BDF
:108D3000E5E9FBE185909590A590B490E9E9FBE128
:108D4000C590D590E590F490A7019601C501B401B6
:108D50000E949DB018162CF4A5019401C701B6011C
:108D600004C0A7019601C501B4010E9453AF2B01B5
:108D70003C01E8E5FBE185919591A591B4918D8742
:108D80009E87AF87B88BE4E5FBE185919591A5912E
:108D9000B491898B9A8BAB8BBC8B2D853E854F858F
:108DA0005889BC01CD010E9413AA87FD05C01D850D
:108DB0000E853F84288804C019890A893B882C883D
:108DC000A3019201C301B2010E9478AA20E030E021
:108DD00040E85FE30E9477AE0E94E2B09B01AC01E5
:108DE000612F702F832D922D0E9478AA69837A8338
:108DF0008B839C83E2EAFBE1149120E030E040ECBD
:108E00005FE3C701B6010E9478AA6B017C01612F64
:108E1000110F770B880B990B0E9419AA9B01AC01CB
:108E2000C701B6010E9478AA69877A878B879C87D9
:108E300020E030E040EC5FE3C501B4010E9478AA75
:108E40006B017C01AD896A2FAA0F770B880B990BF8
:108E50000E9419AA9B01AC01C701B6010E9478AA21
:108E60006D837E838F839887AE014F5F5F4FBE0116
:108E7000675F7F4FCE0105960E94AA300E94B134F1
:108E80001092150E1092160E1092170E1092180EC8
:108E90001092110E1092120E1092130E1092140EC8
:108EA00065960FB6F894DEBF0FBECDBFDF91CF91B0
:108EB0001F910F91FF90EF90DF90CF90BF90AF90F8
:108EC0009F908F907F906F905F904F903F902F90EA
:108ED0000895CF92DF92EF92FF9280E50E94B9331E
:108EE000882329F00E94FF326B017C0103C0C12C52
:108EF000D12C760183E50E94B933882361F00E946A
:108F00003F3320E030E04AE754E40E9478AA0E9410
:108F1000C0AF6B017C010E943A710E94E938C60E15
:108F2000D71EE81EF91E0E94E938DC01CB018C191E
:108F30009D09AE09BF09B7FF03C00E948790F3CF18
:108F4000FF90EF90DF90CF900895AF92BF92CF92B5
:108F5000DF92EF92FF920F931F93CF93DF9380E006
:108F6000A82E83E0B82E98E1E92E9DE0F92E01E1CC
:108F70001EE028EFC22E2DE0D22EC0E0D0E0F50199
:108F800081915F010E947233882321F10E943F3357
:108F9000FE01EE5EFC4F2081211104C020911603DA
:108FA000222341F0F80120813181428153810E94C6
:108FB00077AE0AC0C330D10539F0F6012081318186
:108FC000428153810E9476AEF70160837183828370
:108FD00093830AC0F80180819181A281B381F70156
:108FE00080839183A283B3832196F4E0EF0EF11C7A
:108FF0000C5F1F4F84E0C80ED11CC430D10509F0AE
:10900000BECF86E40E94B9338823C9F00E943F3363
:1090100020E030E0A9010E949DB0181684F40E945F
:109020003F3320E030E040E752E40E9453AF6093CA
:10903000590270935A0280935B0290935C02809174
:10904000F10483FD2AC06091240D7091250D80915B
:10905000260D9091270D20911D0E30911E0E4091EE
:109060001F0E5091200EE091CB04EE23B1F00E9430
:1090700076AE9B01AC016091D8047091D9048091C7
:10908000DA049091DB040E9477AE6093D804709369
:10909000D9048093DA049093DB04DF91CF911F9180
:1090A0000F91FF90EF90DF90CF90BF90AF90089519
:1090B0002F923F924F925F926F927F929F92AF92C8
:1090C000BF92CF92DF92EF92FF920F931F93CF93B5
:1090D000DF93CDB7DEB764970FB6F894DEBF0FBE4F
:1090E000CDBF2A013B01902EA12E6901082F10E06F
:1090F000F801EF55F44EE491BB24B3941E160CF422
:10910000B12CFF24F39420E030E0A901C301B201A7
:109110000E949DB018160CF0F12C000F111F000FCB
:10912000111FC8018F5E914F1C01FC01108211823A
:10913000128213820E94B832F1014082518262820F
:109140007382E090CE0C20E030E0A901692D7A2DE9
:10915000C6010E9413AA811108C0F801EC5AF44E0E
:1091600085919591A591B49103C0892D9A2DD60131
:10917000898B9A8BAB8BBC8B8091190E90911A0EB8
:10918000A0911B0EB0911C0E4091150E5091160E21
:109190006091170E7091180E0091110E1091120E21
:1091A0002091130E3091140E09831A832B833C8374
:1091B0004D835E836F83788789879A87AB87BC8767
:1091C0001D861E861F86188AAE01475F5F4FBE014F
:1091D0006B5F7F4FCE0101960E94A672CE010D9665
:1091E0006C018E010F5E1F4F2DE13EE0AE01475F27
:1091F0005F4FBE016B5F7F4F0C970E9426610E94FC
:109200003A71BF100E94B13464960FB6F894DEBF75
:109210000FBECDBFDF91CF911F910F91FF90EF90C7
:10922000DF90CF90BF90AF909F907F906F905F90B6
:109230004F903F902F9008959091510D891799F07C
:109240008093510D811109C00E94489384E09EE0F3
:109250000E9488710E949D8E04C081E19EE00E9460
:1092600088710C94B832089580E0E6DFE8E3FEE010
:1092700080E090E0A0E8BFE380839183A283B38382
:109280001482158216821782108611861286138622
:109290001486158616861786808B918BA28BB38BCE
:1092A000148A158A168A178A108E118E128E138EC2
:1092B000148E158E168E178E80A391A3A2A3B3A32E
:1092C0000895BF92CF92DF92EF92FF920F931F9378
:1092D000CF93DF9300D01F92CDB7DEB79091DF041C
:1092E000981739F1B82E81110E9416A36091110EC2
:1092F0007091120E8091130E9091140E2091150E04
:109300003091160E4091170E5091180E19821A8244
:109310001B821C82E090190EF0901A0E00911B0E19
:1093200010911C0EFE0131966F010E94CD2FB0925C
:10933000DF0480E00F900F900F900F90DF91CF919E
:109340001F910F91FF90EF90DF90CF90BF90089505
:109350002F923F924F925F926F927F928F929F9245
:10936000AF92BF92CF92DF92EF92FF920F931F9333
:10937000CF93DF93CDB7DEB7C650D1400FB6F89488
:10938000DEBF0FBECDBF41E061E081E00E94102F43
:1093900081110C944F598091510D882371F08FE405
:1093A0000E94B933882319F00E94303303C08FE440
:1093B0000E94723381110C944F59FE0131968CE357
:1093C000DF011D928A95E9F73090510D8AE40E94E1
:1093D0007233882319F048DF0C944F5986E50E94B8
:1093E000B933882349F00E940F33C153DF4F79838B
:1093F0006883CF5CD04006C0C153DF4F198218820A
:10940000CF5CD040C153DF4F08811981CF5CD04081
:109410000530110570F0E0E1FDE084918F010F5FF0
:109420001F4F882311F40C944F590E942774F801A0
:10943000F4CF84E40E94B933882319F00E943033BA
:1094400003C084E40E947233C251DF4F8883CE5E32
:10945000D040C153DF4F08811981CF5CD040033029
:1094600011058CF484E50E94B933882319F00E9419
:10947000303303C084E50E947233CD50DF4F8883C0
:10948000C35FD04006C011E0CD50DF4F1883C35FEB
:10949000D04088E50E94B933882321F00E940F3321
:1094A000162F01C012E089E50E94B933882321F00C
:1094B0000E940F33062F01C002E080E50E94B933FD
:1094C000811102C0612F03C00E940F33062F62304A
:1094D00071F0E7EEFCE084918F010F5F1F4F88234E
:1094E00011F40C944F590E942774F801F4CF023004
:1094F00071F0EEEBFCE084918F010F5F1F4F88232A
:1095000011F40C944F590E942774F801F4CF83E5AD
:109510000E94B933882319F00E943F3304C060E0F1
:1095200070E88BEB95E420E030E040E752E40E94E5
:1095300053AF6093550270935602809357029093F5
:1095400058028CE40E94B933882381F00E943F3393
:109550002091F80D3091F90D4091FA0D5091FB0DCD
:109560000E9476AE0E94BBAF5B0104C01DEFA12E2E
:10957000BB24BA9482E50E94B933882381F00E940B
:109580003F332091F80D3091F90D4091FA0D509133
:10959000FB0D0E9476AE0E94BBAF7B0103C0B1EA17
:1095A000EB2EF12C86E40E94B933882381F00E94CF
:1095B0003F332091FC0D3091FD0D4091FE0D5091F7
:1095C000FF0D0E9476AE0E94BBAF6B0104C0A9EFF5
:1095D000CA2EDD24DA9482E40E94B933882381F014
:1095E0000E943F332091FC0D3091FD0D4091FE0D06
:1095F0005091FF0D0E9476AE0E94BBAF8B0102C05E
:1096000001EA10E0B6010D2C000C880B990B0E94AA
:1096100019AAC751DF4F688379838A839B83C95E08
:10962000D040B5010B2C000C880B990B0E9419AA95
:10963000C151DF4F688379838A839B83CF5ED0409B
:10964000C751DF4F288139814A815B81C95ED04093
:109650000E94898F811103C0E2EAFCE042C0B80198
:10966000012E000C880B990B0E9419AA9B01AC01DA
:10967000B7010F2C000C880B990BCB5FDE4F2883B2
:10968000C550D140CA5FDE4F3883C650D140CD5F50
:10969000DE4F4883C350D140CC5FDE4F5883C45067
:1096A000D1400E9419AACB5FDE4F2881C550D1401E
:1096B000CA5FDE4F3881C650D140CD5FDE4F488152
:1096C000C350D140CC5FDE4F5881C450D1400E947E
:1096D000898FCC50DF4F8883C45FD04081110DC08B
:1096E000BBCF84918F010F5F1F4F882311F40C941F
:1096F0004F590E942774F801F4CFB7016A197B090A
:10970000072E000C880B990B0E9419AACB50DF4F33
:10971000688379838A839B83C55FD040B8016C19C5
:109720007D09072E000C880B990B0E9419AAC750BF
:10973000DF4F688379838A839B83C95FD040C1539D
:10974000DF4F08811981CF5CD040012B11F1ECE88B
:10975000FCE084918F010F5F1F4F882321F00E944E
:109760002774F801F6CFC251DF4F0881CE5ED0409A
:10977000002361F0E2E8FCE084918F010F5F1F4F4E
:10978000882321F00E942774F801F6CF8AE00E9416
:1097900027740E943A7180E04FDD81E092DD8823DA
:1097A00021F0832D49DD0C944F590E94AE2F85E4A2
:1097B0000E94B933882359F00E943033882359F02E
:1097C00011E0CB51DF4F1883C55ED0400AC085E45D
:1097D0000E947233F3CF02E0CB51DF4F0883C55EA6
:1097E000D040CD53DF4F19821882C35CD040C9539B
:1097F000DF4F188219821A821B82C75CD040CF5279
:10980000DF4F1882C15DD0400FEF1FEFC954DF4F0B
:1098100019830883C75BD040CB52DF4F188219826F
:109820001A821B82C55DD0401FEFC752DF4F1883DD
:10983000C95DD040C553DF4F0883CB5CD04011E0F9
:109840002CE0C954DF4F48815981C75BD040249F29
:10985000C001259F900D1124DC01A057B14FC554C4
:10986000DF4FB983A883CB5BD040440F551F440F13
:10987000551FCF51DF4F59834883C15ED040EDE380
:10988000F0E0EC0FFD1FE40FF51FC154DF4FF9832B
:10989000E883CF5BD040C352DF4F19821882CD5D81
:1098A000D040CD53DF4F28813981C35CD040032E97
:1098B000000C440B550BC350DF4F288339834A8378
:1098C0005B83CD5FD040CD53DF4F48815981C35C6E
:1098D000D040440F551FCF5FDE4F59834883C1509E
:1098E000D140C553DF4F0881CB5CD040101709F43D
:1098F00095C2C350DF4F688179818A819B81CD5F9A
:10990000D0400E9419AA9B01AC01CB50DF4F688167
:1099100079818A819B81C55FD0400E9478AA9B0192
:10992000AC01C151DF4F688179818A819B81CF5E13
:10993000D0400E9477AE4B015C01612F012E000CDC
:10994000770B880B990B0E9419AA9B01AC01C75099
:10995000DF4F688179818A819B81C95FD0400E94F5
:1099600078AA9B01AC01C751DF4F688179818A8158
:109970009B81C95ED0400E9477AE6B017C0120E0E4
:1099800030E0A901C501B4010E9413AA87FD05C0FA
:1099900020E030E040E05FE303C020E030E0A901D8
:1099A000C501B4010E9477AE0E94ECAFC355DF4FF2
:1099B000688379838A839B83CD5AD04020E030E04E
:1099C000A901C701B6010E9413AA87FD05C020E0C6
:1099D00030E040E05FE303C020E030E0A901C701D0
:1099E000B6010E9477AE0E94ECAFC755DF4F688387
:1099F00079838A839B83C95AD040C954DF4F8881B9
:109A00009981C75BD0400196C954DF4F9983888301
:109A1000C75BD040CF5FDE4FE881F981C150D140B4
:109A2000E10FF11D17FDFA95EE0FFF1FA1EAB0E05F
:109A3000AC0FBD1FEA0FFB1F91838083C153DF4F23
:109A40002881CF5CD040CB51DF4F4881C55ED040EC
:109A5000BE0167557F4FCE0183559F4F0E9484A35F
:109A6000C953DF4F688379838A839B83C75CD04067
:109A70009B01AC010E9423B1882319F0832DDCDB0C
:109A8000E6C1C953DF4F288139814A815B81C75CB8
:109A9000D040CB52DF4F688179818A819B81C55D3F
:109AA000D0400E9477AECB52DF4F688379838A83A0
:109AB0009B83C55DD040C352DF4FE881F981CD5D06
:109AC000D040CF51DF4F28813981C15ED040E20FB5
:109AD000F31F4DE650E04C0F5D1FE40FF51FC95317
:109AE000DF4F88819981AA81BB81C75CD040848384
:109AF0009583A683B783C355DF4FC880D980EA809A
:109B0000FB80CD5AD040C154DF4FA881B981CF5BD3
:109B1000D0401496CD92DD92ED92FC921797C755E6
:109B2000DF4F288039804A805B80C95AD040FD01D0
:109B3000248A358A468A578A20E030E040E85FE38D
:109B400094962D933D934D935C939797A70196011F
:109B500069817A818B819C810E9477AE69837A8347
:109B60008B839C83A20191016D817E818F81988579
:109B70000E9477AE6D837E838F839887C953DF4FB2
:109B8000288139814A815B81C75CD04069857A85AB
:109B90008B859C850E9477AE69877A878B879C87A7
:109BA000A7019601C701B6010E9478AA9B01AC01EA
:109BB0006D857E858F8598890E9477AE6D877E87BB
:109BC0008F87988BA2019101C201B1010E9478AAEE
:109BD0009B01AC0169897A898B899C890E9477AE47
:109BE000698B7A8B8B8B9C8BC953DF4F2881398192
:109BF0004A815B81C75CD040CA01B9010E9478AA42
:109C00009B01AC016D897E898F89988D0E9477AE0A
:109C10006D8B7E8B8F8B988FA2019101C701B6014E
:109C20000E9478AA9B01AC01698D7A8D8B8D9C8DE9
:109C30000E9477AE698F7A8F8B8F9C8FC953DF4FCD
:109C4000288139814A815B81C75CD040C701B60158
:109C50000E9478AA9B01AC016D8D7E8D8F8D98A19D
:109C60000E9477AE6D8F7E8F8F8F98A3C953DF4F81
:109C7000288139814A815B81C75CD040C201B10132
:109C80000E9478AA9B01AC0169A17AA18BA19CA139
:109C90000E9477AE69A37AA38BA39CA36DA07EA03C
:109CA0000FA1B8A5C351DF4FB883CD5ED04020E0EF
:109CB00030E0A901C701B6010E949DB046015701DD
:109CC00087FF04C0B7FAB094B7F8B0949301402F5F
:109CD000C351DF4F5881CD5ED040C501B4010E9411
:109CE0009DB018163CF04301A02EC351DF4FB88041
:109CF000CD5ED0408DA29EA2AFA2B8A669A47AA4E0
:109D00000BA5ECA5C351DF4FE883CD5ED04020E02A
:109D100030E0A901C201B1010E949DB05201410190
:109D200087FF04C0B7FAB094B7F8B0949301402FFE
:109D3000C351DF4F5881CD5ED040C501B4010E94B0
:109D40009DB018163CF04301A02EC351DF4FB880E0
:109D5000CD5ED04089A69AA6ABA6BCA620E030E096
:109D600040E85FE369AD7AAD8BAD9CAD0E9477AE04
:109D700069AF7AAF8BAF9CAFC554DF4FA881B98173
:109D8000CB5BD0401C96CD92DD92ED92FC921F975A
:109D9000FD01208A318A428A538AC953DF4F2881C4
:109DA00039814A815B81C75CD04054962D933D93A5
:109DB0004D935C9357970E948790C752DF4F08815D
:109DC000C95DD040100FC554DF4F28813981CB5B6E
:109DD000D040245F3F4FC554DF4F39832883CB5B8E
:109DE000D040C352DF4F48815981CD5DD0404C5F98
:109DF0005F4FC352DF4F59834883CD5DD040C1547C
:109E0000DF4F88819981CF5BD0400496C154DF4FEA
:109E100099838883CF5BD040312C63CDCD53DF4F06
:109E200008811981C35CD0400130110581F0C9530C
:109E3000DF4F288139814A815B81C75CD040CA01EC
:109E4000B9010E9423B1882311F40C941C5980E0BD
:109E500038DA882321F0832DEFD90C941059C95397
:109E6000DF4F288139814A815B81C75CD040CA01BC
:109E7000B9010E9423B181110C94105989AC9AAC9C
:109E8000ABACBCAC20E030E0A901C501B4010E943C
:109E900013AA882309F411C2A501940169817A816A
:109EA0008B819C810E9453AFC954DF4F68837983B3
:109EB0008A839B83C75BD04069837A838B839C832F
:109EC000A50194016D817E818F8198850E9453AF99
:109ED000C554DF4F688379838A839B83CB5BD040F3
:109EE0006D837E838F839887A501940169857A8528
:109EF0008B859C850E9453AFC154DF4F6883798363
:109F00008A839B83CF5BD04069877A878B879C87C6
:109F1000A50194016D857E858F8598890E9453AF38
:109F20006B017C01C954DF4F288139814A815B81F3
:109F3000C75BD040CA01B9010E9478AA9B01AC015D
:109F4000C701B6010E9476AEC553DF4F688379839F
:109F50008A839B83CB5CD0406D877E878F87988B6D
:109F6000A501940169897A898B899C890E9453AFE4
:109F70006B017C01C554DF4F288139814A815B81A7
:109F8000CB5BD040CA01B9010E9478AA9B01AC0109
:109F9000C701B6010E9476AEC752DF4F688379834E
:109FA0008A839B83C95DD040698B7A8B8B8B9C8B1A
:109FB000A50194016D897E898F89988D0E9453AF88
:109FC0006B017C01C154DF4F288139814A815B815B
:109FD000CF5BD040CA01B9010E9478AA9B01AC01B5
:109FE000C701B6010E9476AE6D8B7E8B8F8B988FEA
:109FF000A5019401698D7A8D8B8D9C8D0E9453AF44
:10A000006B017C01C554DF4F288139814A815B8116
:10A01000CB5BD040C954DF4F688179818A819B81B5
:10A02000C75BD0400E9478AA9B01AC01C701B60172
:10A030000E9476AECD53DF4F688379838A839B83FA
:10A04000C35CD040698F7A8F8B8F9C8FA501940160
:10A0500069A17AA18BA19CA10E9453AF6B017C01E5
:10A06000C154DF4F288139814A815B81CF5BD04069
:10A07000C554DF4F688179818A819B81CB5BD04059
:10A080000E9478AA9B01AC01C701B6010E9476AE7E
:10A09000CF52DF4F688379838A839B83C15DD04031
:10A0A00069A37AA38BA39CA3A50194016D8D7E8DDA
:10A0B0008F8D98A10E9453AF4B015C01C154DF4FBB
:10A0C000288139814A815B81CF5BD040C954DF4F01
:10A0D000688179818A819B81C75BD0400E9478AA80
:10A0E0009B01AC01C501B4010E9476AE4B015C013D
:10A0F0006D8F7E8F8F8F98A3C752DF4F2881398154
:10A100004A815B81C95DD040C553DF4F6881798149
:10A110008A819B81CB5CD0400E9478AA2B013C01B4
:10A12000CD53DF4F288139814A815B81C35CD040A8
:10A13000CA01B9010E9478AA9B01AC01C301B20116
:10A140000E9476AE6B017C0120E030E0A9010E9404
:10A150009DB02601370187FF04C077FA709477F825
:10A16000709429A53AA54BA55CA56DA17EA18FA1F0
:10A1700098A50E9477AE2FEF36EE4BED5EE20E947F
:10A1800078AA9B01AC01C301B2010E9413AA181660
:10A190000CF093C0CD53DF4F288139814A815B8118
:10A1A000C35CD040CF52DF4F688179818A819B8127
:10A1B000C15DD0400E9478AA2B013C01C752DF4FFD
:10A1C000288139814A815B81C95DD040C501B401D4
:10A1D0000E9478AA9B01AC01C301B2010E9476AE35
:10A1E000A70196010E9453AF2B013C016DA77EA7EA
:10A1F0008FA798ABCD53DF4F288139814A815B818E
:10A20000C35CD040C501B4010E9478AA4B015C0137
:10A21000C553DF4F288139814A815B81CB5CD040B7
:10A22000CF52DF4F688179818A819B81C15DD040A7
:10A230000E9478AA9B01AC01C501B4010E9476AED0
:10A24000A70196010E9453AF6B017C0169AB7AAB09
:10A250008BAB9CABC954DF4F288139814A815B812C
:10A26000C75BD040C301B2010E9478AA9B01AC0138
:10A27000C154DF4F688179818A819B81CF5BD04057
:10A280000E9477AE4B015C01C554DF4F28813981B4
:10A290004A815B81CB5BD040C701B6010E9478AA9E
:10A2A0009B01AC01C501B4010E9477AEDC01CB017A
:10A2B000B0588DAB9EABAFABB8AF2DA53EA54FA5AB
:10A2C00058A9C554DF4F288339834A835B83CB5B0E
:10A2D000D0405058C154DF4F288339834A835B8371
:10A2E000CF5BD04089A99AA9ABA9BCA9CD53DF4FB8
:10A2F00088839983AA83BB83C35CD0400DA91EA920
:10A300002FA938ADC151DF4F088319832A833B83BE
:10A31000CF5ED04020E030E040E85EE3CB52DF4F3C
:10A32000688179818A819B81C55DD0400E9478AA2D
:10A33000C752DF4F688379838A839B83C95DD0408E
:10A34000C153DF4F08811981CF5CD040012B09F444
:10A350006CC24090A40E5090A50E6090A60E709016
:10A36000A70E2091B00E3091B10E4091B20E5091D7
:10A37000B30EC301B2010E9476AEC352DF4F6883B1
:10A3800079838A839B83CD5DD040C090A00ED0900E
:10A39000A10EE090A20EF090A30E2091AC0E309191
:10A3A000AD0E4091AE0E5091AF0EC701B6010E94A6
:10A3B00076AECF51DF4F688379838A839B83C15EFA
:10A3C000D04080909C0E90909D0EA0909E0EB090DC
:10A3D0009F0E2091A80E3091A90E4091AA0E509187
:10A3E000AB0EC501B4010E9476AECB51DF4F68833E
:10A3F00079838A839B83C55ED0402091980E3091EB
:10A40000990E40919A0E50919B0EC553DF4F2883B1
:10A4100039834A835B83CB5CD040A3019201C5534F
:10A42000DF4F688179818A819B81CB5CD0400E941B
:10A4300076AEC751DF4F688379838A839B83C95E79
:10A44000D0408091940E9091950EA091960EB0916F
:10A45000970ECB52DF4F88839983AA83BB83C55D58
:10A46000D040A7019601BC01CD010E9476AE6B01E0
:10A470007C010091900E1091910E2091920E3091DE
:10A48000930ECF52DF4F088319832A833B83C15D2C
:10A49000D040A5019401CF52DF4F688179818A8134
:10A4A0009B81C15DD0400E9476AE4B015C01CF51D3
:10A4B000DF4F288139814A815B81C15ED0400E9493
:10A4C00078AA2B013C01CB51DF4F288139814A8189
:10A4D0005B81C55ED040C701B6010E9478AA9B018E
:10A4E000AC01C301B2010E9476AEC954DF4F68834C
:10A4F00079838A839B83C75BD040CB51DF4F288110
:10A5000039814A815B81C55ED040C751DF4F688188
:10A5100079818A819B81C95ED0400E9478AA2B01F3
:10A520003C01C352DF4F288139814A815B81CD5D77
:10A53000D040C501B4010E9478AA9B01AC01C301BF
:10A54000B2010E9476AE2B013C01C352DF4F28813D
:10A5500039814A815B81CD5DD040C701B6010E943F
:10A5600078AA6B017C01CF51DF4F288139814A8164
:10A570005B81C15ED040C751DF4F688179818A819C
:10A580009B81C95ED0400E9478AA9B01AC01C701A3
:10A59000B6010E9476AE6B017C012091B40E309121
:10A5A000B50E4091B60E5091B70E0E9478AA4B019D
:10A5B0005C012091B80E3091B90E4091BA0E5091C5
:10A5C000BB0EC301B2010E9478AA9B01AC01C50178
:10A5D000B4010E9477AE4B015C012091BC0E30911A
:10A5E000BD0E4091BE0E5091BF0EC954DF4F688121
:10A5F00079818A819B81C75BD0400E9478AA9B01A8
:10A60000AC01C501B4010E9477AE4B015C01CF5291
:10A61000DF4F688179818A819B81C15DD0409058EC
:10A62000A70196010E9478AACF52DF4F68837983F1
:10A630008A839B83C15DD040A3019201CB52DF4F3F
:10A64000688179818A819B81C55DD0400E9478AA0A
:10A650009B01AC01CF52DF4F688179818A819B8158
:10A66000C15DD0400E9476AECB52DF4F68837983C4
:10A670008A839B83C55DD040C954DF4F28813981CF
:10A680004A815B81C75BD040C553DF4F68817981C8
:10A690008A819B81CB5CD0400E9478AA9B01AC014F
:10A6A000CB52DF4F688179818A819B81C55DD04023
:10A6B0000E9476AE9B01AC01C501B4010E9477AE49
:10A6C0004B015C0120E030E0A9010E949DB018160A
:10A6D00024F0B7FAB094B7F8B094A7019601C70177
:10A6E000B6010E9478AA6B017C01A3019201C3010B
:10A6F000B2010E9478AA9B01AC01C701B6010E9479
:10A7000077AE6B017C01C954DF4F288139814A81C2
:10A710005B81C75BD040CA01B9010E9478AA9B0146
:10A72000AC01C701B6010E9477AE0E94E2B09B0166
:10A73000AC01C501B4010E9453AFAB01BC018BE574
:10A740009CE00E94AF438AE00E9427748AE00E9446
:10A750002774E5E4FCE084918F010F5F1F4F88238D
:10A7600021F00E942774F801F6CF48E0C154DF4F72
:10A77000688179818A819B81CF5BD0400E94D378A8
:10A78000E0E4FCE084918F010F5F1F4F882321F0EC
:10A790000E942774F801F6CF48E0CD53DF4F68815F
:10A7A00079818A819B81C35CD04090580E94D37884
:10A7B000EBE3FCE084918F010F5F1F4F882321F0B2
:10A7C0000E942774F801F6CFC151DF4F688179816B
:10A7D0008A819B81CF5ED040905848E00E94D37818
:10A7E0008AE00E942774C153DF4F08811981CF5C32
:10A7F000D04003301105CCF002E21CE0F801849156
:10A80000882329F00F5F1F4F0E942774F7CF48E07D
:10A81000C752DF4F688179818A819B81C95DD040B1
:10A820000E94D3788AE00E942774C251DF4F0881CA
:10A83000CE5ED0400111E9C1C554DF4F2881398176
:10A840004A815B81CB5BD040CB56DF4F2883398375
:10A850004A835B83C559D040CD53DF4F88819981AE
:10A86000AA81BB81C35CD040C756DF4F88839983E0
:10A87000AA83BB83C959D040C12CD12C60E8E62EF5
:10A880006FE3F62EC356DF4FC882D982EA82FB827D
:10A89000CD59D040CE018B569F4F0E94D345C7570C
:10A8A000DF4FC882D982EA82FB82C958D040C357A1
:10A8B000DF4F188219821A821B82CD58D040C154B2
:10A8C000DF4F088119812A813B81CF5BD040CF5671
:10A8D000DF4F088319832A833B83C159D040CE01BF
:10A8E00087579F4F0E94D345CB56DF4F2881398130
:10A8F0004A815B81C559D040C954DF4F28833983D1
:10A900004A835B83C75BD040C756DF4F488059807E
:10A910006A807B80C959D040C356DF4F88809980B8
:10A92000AA80BB80CD59D040C757DF4F888199811D
:10A93000AA81BB81C958D040C554DF4F8883998311
:10A94000AA83BB83CB5BD040C357DF4F08811981FB
:10A950002A813B81CD58D040C154DF4F08831983F1
:10A960002A833B83CF5BD040CF56DF4FC880D9804E
:10A97000EA80FB80C159D040A7019601C301B20112
:10A980000E9478AACD53DF4F688379838A839B83A3
:10A99000C35CD040C154DF4F288139814A815B813B
:10A9A000CF5BD040C501B4010E9478AA9B01AC01E5
:10A9B000CD53DF4F688179818A819B81C35CD04010
:10A9C0000E9476AEC358DF4F688379838A839B8366
:10A9D000CD57D040C554DF4F288139814A815B81F2
:10A9E000CB5BD040C501B4010E9478AA4B015C0149
:10A9F000A7019601C954DF4F688179818A819B81C3
:10AA0000C75BD0400E9478AA9B01AC01C501B4018C
:10AA10000E9476AECF57DF4F688379838A839B830A
:10AA2000C158D040C154DF4F288139814A815B81B0
:10AA3000CF5BD040C954DF4F688179818A819B8187
:10AA4000C75BD0400E9478AA6B017C01C554DF4FE0
:10AA5000288139814A815B81CB5BD040C301B2013F
:10AA60000E9478AA9B01AC01C701B6010E9476AE94
:10AA7000CB57DF4F688379838A839B83C558D04047
:10AA8000CE0183589F4F0E94D345C757DF4F08819F
:10AA900019812A813B81C958D040C357DF4F488074
:10AAA00059806A807B80CD58D040CF56DF4F888058
:10AAB0009980AA80BB80C159D040C358DF4F88819C
:10AAC0009981AA81BB81CD57D040C954DF4F88837B
:10AAD0009983AA83BB83C75BD040CF57DF4F888160
:10AAE0009981AA81BB81C158D040C554DF4F88836A
:10AAF0009983AA83BB83CB5BD040CB57DF4F888140
:10AB00009981AA81BB81C558D040C154DF4F888349
:10AB10009983AA83BB83CF5BD040CB56DF4FC880DD
:10AB2000D980EA80FB80C559D040C756DF4F4881A5
:10AB300059816A817B81C959D040C356DF4F8881D2
:10AB40009981AA81BB81CD59D0400093380E1093D2
:10AB5000390E20933A0E30933B0E40923C0E5092A9
:10AB60003D0E60923E0E70923F0E8092400E90928B
:10AB7000410EA092420EB092430EC954DF4F08819D
:10AB800019812A813B81C75BD0400093440E10930A
:10AB9000450E2093460E3093470EC554DF4F088173
:10ABA00019812A813B81CB5BD0400093480E1093E2
:10ABB000490E20934A0E30934B0EC154DF4F08814B
:10ABC00019812A813B81CF5BD04000934C0E1093BA
:10ABD0004D0E20934E0E30934F0EC092500ED092D9
:10ABE000510EE092520EF092530E4093540E509339
:10ABF000550E6093560E7093570E8093580E909397
:10AC0000590EA0935A0EB0935B0ECD50DF4F1881B2
:10AC1000C35FD040112309F460C2EFE5FBE08491EB
:10AC20008F010F5F1F4F81113DC06E0123EAC20EDD
:10AC3000D11CC554DF4FD982C882CB5BD04002E023
:10AC4000CB52DF4F0883C55DD040212C10ECC1549E
:10AC5000DF4F1883CF5BD04009E7CD53DF4F088328
:10AC6000C35CD04014E4C553DF4F1883CB5CD040A5
:10AC70008E010B561F4FCF54DF4F19830883C15BE2
:10AC8000D0400C501109CD54DF4F19830883C35BAA
:10AC9000D0400C501109CB54DF4F19830883C55B9A
:10ACA000D0403CC00E942774F801B9CF80E20E94D6
:10ACB000277445E0C501B4010E94D378C954DF4F21
:10ACC00008811981C75BD0400C5F1F4FC954DF4F0B
:10ACD00019830883C75BD0400830110529F58AE045
:10ACE0000E942774C554DF4F08811981CB5BD04087
:10ACF00002501109C554DF4F19830883CB5BD04044
:10AD0000CB52DF4F1881C55DD040113009F4F2C03D
:10AD100001E0CB52DF4F0883C55DD040C954DF4FFF
:10AD200019821882C75BD040C554DF4FE881F98192
:10AD3000CB5BD040C954DF4F08811981C75BD0403D
:10AD4000E00FF11F008111817801EE0CFF1CEE0C69
:10AD5000FF1CEDE6F0E0EC0FFD1FEE0DFF1D408047
:10AD6000518062807380C752DF4F288139814A81C8
:10AD70005B81C95DD040C301B2010E9476AE4B0138
:10AD80005C01E1E0F0E0EC0FFD1FEE0DFF1D84AD76
:10AD900095ADA6ADB7ADCB56DF4F88839983AA8317
:10ADA000BB83C559D040F8013496EE0FFF1FEE0F5C
:10ADB000FF1F21E030E02C0F3D1FE20FF31F84AD99
:10ADC00095ADA6ADB7ADC757DF4F88839983AA83EA
:10ADD000BB83C958D040C358DF4F188219821A82EA
:10ADE0001B82CD57D040CA54DF4F3881C65BD0405C
:10ADF0003F93CB54DF4F4881C55BD0404F93CC5439
:10AE0000DF4F5881C45BD0405F93CD54DF4F8881C2
:10AE1000C35BD0408F93CE54DF4F9881C25BD0404C
:10AE20009F93CF54DF4FA881C15BD040AF93EDB764
:10AE3000FEB7B4970FB6F894FEBF0FBEEDBFADB727
:10AE4000BEB71196E8E3FEE084E201900D928A9588
:10AE5000E1F70E94EE44C358DF4F288139814A81CF
:10AE60005B81CD57D040C301B2010E9476AE7B0119
:10AE70008C010FB6F894DEBF0FBECDBF9B01AC01B5
:10AE8000622DC154DF4F7881CF5BD040CD53DF4F6F
:10AE90008881C35CD040C553DF4F9881CB5CD040E4
:10AEA0000E949DB0181684F42E2CC154DF4FF882F6
:10AEB000CF5BD040CD53DF4F0883C35CD040C55338
:10AEC000DF4F1883CB5CD04020E030E0A901C50102
:10AED000B4010E949DB087FDE9CEECE5FBE08491D2
:10AEE0008F010F5F1F4F882309F4E3CE0E94277460
:10AEF000F801F5CF8AE00E942774C153DF4F088123
:10AF00001981CF5CD0400430110509F0E6C0E3E3BD
:10AF1000FBE084918F010F5F1F4F882321F00E9477
:10AF20002774F801F6CF02E0C153DF4F0883CF5CEE
:10AF3000D0404E0115E9810E911C5E0129E8A20E58
:10AF4000B11C7E013DE7E30EF11C00E010E0F601CC
:10AF5000E00FF11F808191813C01660C771C660C2B
:10AF6000771CE1E0F0E0EC0FFD1FE60DF71D44ADAE
:10AF700055AD66AD77ADD4014D935D936D937C93E4
:10AF80001397FC013496EE0FFF1FEE0FFF1F21E019
:10AF900030E02C0F3D1FE20FF31F84AD95ADA6AD41
:10AFA000B7ADF50180839183A283B383D7011D924E
:10AFB0001D921D921C921397FF92EF92BF92AF9237
:10AFC0009F928F92EDB7FEB7B4970FB6F894FEBF7D
:10AFD0000FBEEDBFADB7BEB71196E8E3FEE084E269
:10AFE00001900D928A95E1F70E94EE44EDE6F0E0C3
:10AFF000EC0FFD1FE60DF71DD7012D913D914D91F1
:10B000005C9160817181828193810E9476AE222D54
:10B01000C154DF4F3881CF5BD040CD53DF4F4881E3
:10B02000C35CD040C553DF4F5881CB5CD0400E94F9
:10B0300076AE2B013C010FB6F894DEBF0FBECDBF3C
:10B0400020E030E0A9010E949DB087FD20C0E0E330
:10B05000FBE084919F012F5F3F4F8823D9F0CB5FA6
:10B06000DE4F2883C550D140CA5FDE4F3883C650BB
:10B07000D1400E942774CB5FDE4F2881C550D1405C
:10B08000CA5FDE4F3881C650D140F901E2CF80E27D
:10B090000E94277445E0C301B2010E94D3780C5F7F
:10B0A0001F4F0830110509F052CF8AE00E94277423
:10B0B000F2E0CF1AD108C153DF4F0881CF5CD040F6
:10B0C000013039F011E0C153DF4F1883CF5CD0401D
:10B0D0003CCF8AE00E94277408C0C153DF4F08812B
:10B0E0001981CF5CD040012B21F081E19BE00E94CF
:10B0F00033A5C251DF4F1881CE5ED040111184C0FC
:10B100008CE0E1E1FEE0DE01A358BF4F01900D921B
:10B110008A95E1F781E08093510DCE0183589F4FCE
:10B120000E948871C355DF4F288139814A815B8134
:10B13000CD5AD0406091110E7091120E8091130E75
:10B140009091140E0E9476AE6B017C012DEB37E3DB
:10B1500046E855EB0E949DB087FD4BC02DEB37E3D1
:10B1600046E855E3C701B6010E9413AA18160CF46D
:10B1700040C0C755DF4F288139814A815B81C95A58
:10B18000D0406091150E7091160E8091170E90911F
:10B19000180E0E9476AE6B017C012DEB37E346E87A
:10B1A00055EB0E949DB087FD24C02DEB37E346E8A8
:10B1B00055E3C701B6010E9413AA1816D4F0C9536B
:10B1C000DF4F288139814A815B81C75CD040609123
:10B1D000190E70911A0E80911B0E90911C0E0E94F8
:10B1E00076AECB57DF4F688379838A839B83C558BC
:10B1F000D0408CE0FE01E358FF4FA1E1BEE001909A
:10B200000D928A95E1F705C0CC50DF4F3882C45FBC
:10B21000D040CC50DF4F0881C45FD0400093510D27
:10B220000E94952F81E08093D30C8091510D811164
:10B230000E94B8320BD533C081E0CF52DF4F188166
:10B24000C15DD0401827CF52DF4F1883C15DD04079
:10B25000111117C01FEFC752DF4F1883C95DD040CF
:10B260000FEFC553DF4F0883CB5CD04011E021E0E6
:10B2700030E0CD53DF4F39832883C35CD0400C943A
:10B28000204C01E0C752DF4F0883C95DD04012E077
:10B29000C553DF4F1883CB5CD04010E0E8CFCA5FC6
:10B2A000DE4F0FB6F894DEBF0FBECDBFDF91CF915A
:10B2B0001F910F91FF90EF90DF90CF90BF90AF90D4
:10B2C0009F908F907F906F905F904F903F902F90C6
:10B2D0000895EF92FF920F931F93CF93DF931F92E6
:10B2E000CDB7DEB7082F162FEAE6FDE084917F0187
:10B2F0002FEFE21AF20A882331F099830E94277413
:10B30000F7019981F3CFE02FF92F84917F019FEF0F
:10B31000E91AF90A882321F00E942774F701F5CF72
:10B32000E8E6FDE084917F012FEFE21AF20A88231C
:10B3300021F00E942774F701F5CF612F70E080E0C3
:10B3400090E00E94B9788AE00F90DF91CF911F9131
:10B350000F91FF90EF900C94277481E0809311027D
:10B3600083E50E94B933882331F00E943033811184
:10B3700006C00C94859583E50E947233F8CF08953A
:10B38000CF93DF93ECE4FFE18491EF0121968823D2
:10B3900021F00E942774FE01F7CFEBEFFFE08491CC
:10B3A000EF012196882321F00E942774FE01F7CF38
:10B3B000DF91CF9108950F931F93CF9383E50E9460
:10B3C000B9338823C1F10E941F33813031F08230BC
:10B3D00091F500E013E0C0E01FC000E013E0C0E022
:10B3E000F80181918F010E94B933882339F00E94BE
:10B3F0001F334FEF682F8C2F0E94749FCF5FC43094
:10B4000079F782E40E94B9338823A9F00E941F33A0
:10B4100012C0CF5FC430A9F3F80181918F010E945F
:10B42000B9338823B1F30E941F33482F6FEF8C2F5D
:10B430000E94749FEECFCF911F910F910C94DD9ECF
:10B440000F931F93CF9383E50E947233811104C041
:10B4500000E013E0C0E00EC0C0E00E941F33682F80
:10B460008C2F0E94C99FCF5FC530B9F7F1CFCF5F56
:10B47000C43071F0F80181918F010E9472338823EA
:10B48000B1F30E941F33682F8C2F0E94C99FEFCF0A
:10B4900082E40E947233882331F00E941F33682FA8
:10B4A00084E00E94C99FCF911F910F910C94DD9E63
:10B4B000CF93DF9383E50E947233C82F882371F006
:10B4C0000E943F330E94BBAF70932A02609329020F
:10B4D00021E0672B09F020E020930E0480E50E9414
:10B4E0007233882359F02091290230912A02232BAC
:10B4F00011F00E94303380930E042DC0C1112BC077
:10B50000EEEDFEE18491EF012196882321F00E9467
:10B510002774FE01F7CF80910E04811103C064E00F
:10B5200073E002C067EE72E08AEC9FE00E94C644BE
:10B530006091290270912A0289EB9FE00E94AD443C
:10B54000E5EBFFE08491EF012196882321F00E9432
:10B550002774FE01F7CFDF91CF910895CF93DF934A
:10B5600080E50E947233882351F00E943F3360933C
:10B57000410D7093420D8093430D9093440D89E4E7
:10B580000E947233882381F00E943F332CEA35EC0D
:10B5900047E25EE30E9478AA60933D0D70933E0DF2
:10B5A00080933F0D9093400D84E40E947233882372
:10B5B00081F00E943F332CEA35EC47E25EE30E94C3
:10B5C00053AF6093390D70933A0D80933B0D909378
:10B5D0003C0DEEEDFEE18491EF012196882321F0F0
:10B5E0000E942774FE01F7CF4091410D5091420D0A
:10B5F0006091430D7091440D81EB9FE00E94AF4339
:10B600002CEA35EC47E25EE360913D0D70913E0D12
:10B6100080913F0D9091400D0E9453AFAB01BC0152
:10B620008DEA9FE00E94AF432CEA35EC47E25EE3EF
:10B630006091390D70913A0D80913B0D90913C0DC8
:10B640000E9478AAAB01BC0189EA9FE00E94AF4347
:10B650008AE0DF91CF910C942774CF93DF9385E438
:10B660000E94B933811110C080E50E947233882393
:10B6700091F00E943F3360934D0D70934E0D809377
:10B680004F0D9093500D07C00E941F33882361F324
:10B69000ECE4FFE16EC089E40E947233882381F0FC
:10B6A0000E943F332CEA35EC47E25EE30E9478AA21
:10B6B0006093490D70934A0D80934B0D90934C0D00
:10B6C00084E40E947233882381F00E943F332CEA85
:10B6D00035EC47E25EE30E9453AF6093450D7093F3
:10B6E000460D8093470D9093480DEEEDFEE1849159
:10B6F000EF012196882321F00E942774FE01F7CFE5
:10B7000040914D0D50914E0D60914F0D7091500D27
:10B7100083E99FE00E94AF432CEA35EC47E25EE309
:10B720006091490D70914A0D80914B0D90914C0D97
:10B730000E9453AFAB01BC018FE89FE00E94AF4372
:10B740002CEA35EC47E25EE36091450D7091460DC1
:10B750008091470D9091480D0E9478AAAB01BC01E1
:10B760008BE89FE00E94AF438AE0DF91CF910C9479
:10B7700027748491EF012196882321F00E94277479
:10B78000FE01F7CFE7E9FFE08491EF0121968823DE
:10B7900021F00E942774FE01F7CFDF91CF91089529
:10B7A000CF92DF92EF92FF92CF93DF9380E50E94DA
:10B7B00072338823C1F10E940F336B017C0183E552
:10B7C0000E94B933882321F00E940F33EB0102C09D
:10B7D000CFEFDFEF9E012F5F3F4F2330310518F58C
:10B7E000D7FC21C00E943A71CF3F8FEFD80729F0D4
:10B7F000219771F4C1E0D0E00DC08C2D0E94F1368C
:10B8000031E020E0892B09F030E0C32FD22F02C0B5
:10B81000C0E0D0E08C2D0E94F1368C179D0719F006
:10B820000E948790F7CFDF91CF91FF90EF90DF904C
:10B83000CF9008950F931F93CF93DF938DED90E0FA
:10B840000E94C533811166C083E50E94B933882305
:10B85000B9F1C091FA03D0E00E940F33CC0FDD1F85
:10B86000CD5DDD4F798368838091FA0390E0EC0130
:10B87000CC0FDD1FCC0FDD1F8E010B5D1D4F880F20
:10B88000991FFC01ED5DFD4F60817181072E000C59
:10B89000880B990B0E9419AA2AE037ED43E25CE37A
:10B8A0000E9478AACD5FDB4F288139814A815B8174
:10B8B0000E9478AAF80160837183828393832AC0EF
:10B8C000EEEDFEE18491EF012196882321F00E94A4
:10B8D0002774FE01F7CF85E40E9427748091FA0354
:10B8E000805D0E942774E091FA03F0E0EE0FFF1FE5
:10B8F000ED5DFD4F6081718183E89FE00E94AD4462
:10B9000085E20E9427748AE0DF91CF911F910F9109
:10B910000C942774DF91CF911F910F910895CF93CD
:10B92000DF93EEEDFEE18491EF012196882321F073
:10B930000E942774FE01F7CF83E50E9472338823AB
:10B9400021F00E94303380934C02E3E7FFE08491C2
:10B95000EF012196882321F00E942774FE01F7CF82
:10B9600080914C02811103C0EFE6FFE002C0EBE6DC
:10B97000FFE08491EF012196882321F00E94277433
:10B98000FE01F7CFE3E6FFE08491EF0121968823E3
:10B9900021F00E942774FE01F7CF2091F80D30911D
:10B9A000F90D4091FA0D5091FB0D609117027091C5
:10B9B00018028091190290911A020E9477AEAB0191
:10B9C000BC0181E69FE00E94AF432091FC0D3091C5
:10B9D000FD0D4091FE0D5091FF0D60911B02709185
:10B9E0001C0280911D0290911E020E9477AEAB0155
:10B9F000BC018EE59FE00E94AF432091000E309184
:10BA0000010E4091020E5091030E60911F02709141
:10BA1000200280912102909122020E9477AEAB0118
:10BA2000BC018BE59FE00E94AF43E3E5FFE084911A
:10BA3000EF012196882321F00E942774FE01F7CFA1
:10BA40002091F80D3091F90D4091FA0D5091FB0DB8
:10BA500060914002709141028091420290914302B4
:10BA60000E9477AEAB01BC0181E59FE00E94AF432D
:10BA70002091FC0D3091FD0D4091FE0D5091FF0D78
:10BA80006091440270914502809146029091470274
:10BA90000E9477AEAB01BC018EE49FE00E94AF43F1
:10BAA0002091000E3091010E4091020E5091030E34
:10BAB000609148027091490280914A0290914B0234
:10BAC0000E9477AEAB01BC018BE49FE00E94AF43C4
:10BAD0008AE0DF91CF910C94277482E40E94723344
:10BAE000882351F00E94FF3260936A0D70936B0DB2
:10BAF00080936C0D90936D0D83E50E9472338823C3
:10BB000051F00E943F336093660D7093670D8093F0
:10BB1000680D9093690D84E50E947233882351F07B
:10BB20000E943F336093620D7093630D8093640DA8
:10BB30009093650D88E50E947233882351F00E942E
:10BB40003F336093520D7093530D8093540D909337
:10BB5000550D89E50E947233882351F00E943F33CE
:10BB60006093560D7093570D8093580D9093590D17
:10BB70008AE50E947233882351F00E943F3360931C
:10BB80005A0D70935B0D80935C0D90935D0D85E471
:10BB90000E947233882351F00E943F3360935E0D00
:10BBA00070935F0D8093600D9093610D0895CF9316
:10BBB000DF93EEE4FEE08491EF012196882321F0EB
:10BBC0000E942774FE01F7CF60E08EE39EE081DBE8
:10BBD00061E087E39EE07DDB61E08CE29EE079DB63
:10BBE00061E08CE19EE075DB60E083E19EE071DB6B
:10BBF00061E089E09EE06DDB61E08FEF9DE069DB55
:10BC000061E087EF9DE065DB61E089EE9DE061DB4F
:10BC100060E08BED9DE05DDB60E08CEC9DE059DB4E
:10BC200060E08EEB9DE055DB60E088EA9DE051DB53
:10BC300061E087E99DE04DDB60E082E89DE049DB63
:10BC400061E08FE69DE0DF91CF9143CB4F925F9211
:10BC50006F927F928F929F92AF92BF92CF92DF921C
:10BC6000EF92FF92CF93DF93E5E6FDE08491EF0141
:10BC70002196882321F00E942774FE01F7CF20919E
:10BC8000F80D3091F90D4091FA0D5091FB0D609136
:10BC9000110E7091120E8091130E9091140E0E944D
:10BCA00077AE42E00E94D378E1E6FDE08491EF01B7
:10BCB0002196882321F00E942774FE01F7CF20915E
:10BCC000FC0D3091FD0D4091FE0D5091FF0D6091E6
:10BCD000150E7091160E8091170E9091180E0E94FD
:10BCE00077AE42E00E94D378EDE5FDE08491EF016C
:10BCF0002196882321F00E942774FE01F7CF20911E
:10BD0000000E3091010E4091020E5091030E609191
:10BD1000190E70911A0E80911B0E90911C0E0E94AC
:10BD200077AE42E00E94D378E9E5FDE08491EF012F
:10BD30002196882321F00E942774FE01F7CF60919D
:10BD40001D0E70911E0E80911F0E9091200E42E0EC
:10BD50000E94D37880916F0081FB992790F981FF31
:10BD600005C080916F008D7F80936F004090C30D60
:10BD70005090C40D6090C50D7090C60D8090C70D99
:10BD80009090C80DA090C90DB090CA0DC090CB0D79
:10BD9000D090CC0DE090CD0DF090CE0D992329F0F0
:10BDA00080916F00826080936F00EFE4FDE08491EA
:10BDB000EF012196882321F00E942774FE01F7CF1E
:10BDC000C301B2010E94B978EBE4FDE08491EF0178
:10BDD0002196882321F00E942774FE01F7CFC50128
:10BDE000B4010E94B978E7E4FDE08491EF01219667
:10BDF000882321F00E942774FE01F7CFC701B60106
:10BE00000E94B9788AE0DF91CF91FF90EF90DF90A8
:10BE1000CF90BF90AF909F908F907F906F905F90EA
:10BE20004F900C9427742F923F924F925F926F9293
:10BE30007F928F929F92AF92BF92CF92DF92EF92BA
:10BE4000FF920F931F93CF93DF93CDB7DEB72F975A
:10BE50000FB6F894DEBF0FBECDBF41E061E081E0D8
:10BE60000E94102F8111B5C098E4892E9BE1992E74
:10BE700081E19EE09E878D87FE0131965F0101EA98
:10BE80001BE11F01F3E0F00FFF87F401659175914D
:10BE900085919491ED85FE85C190D190E190F190CE
:10BEA000FE87ED87A70196010E9476AE2B013C012B
:10BEB00020E030E040EA51EC0E949DB087FD10C0C8
:10BEC00020E030E040EA51E4C301B2010E9413AA2D
:10BED000181634F0F10140825182628273820DC0E3
:10BEE000F80184911816B4F7F7FAF094F7F8F09483
:10BEF000F101C082D182E282F382F101C190D1903E
:10BF0000E190F1901F0120E030E040EA51ECC701E0
:10BF1000B6010E949DB087FF03C0ECE4FFE10BC0B7
:10BF200020E030E040EA51E4C701B6010E9413AAC4
:10BF30001816BCF4F2CF84918F010F5F1F4F882336
:10BF400021F00E942774F801F6CFEDEDFFE0849117
:10BF50008F010F5F1F4F8823E1F10E942774F801C2
:10BF6000F6CFF4E08F0E911C0F5F1F4F8F8580136B
:10BF70008CCF80EEE82E84E0F82E10E0F501819160
:10BF80009191A191B1915F01F70181939193A19357
:10BF9000B1937F01812F0E94E9301F5F133071F749
:10BFA0002F960FB6F894DEBF0FBECDBFDF91CF91B5
:10BFB0001F910F91FF90EF90DF90CF90BF90AF90C7
:10BFC0009F908F907F906F905F904F903F902F90B9
:10BFD0003DCE2F960FB6F894DEBF0FBECDBFDF91DA
:10BFE000CF911F910F91FF90EF90DF90CF90BF9076
:10BFF000AF909F908F907F906F905F904F903F9009
:10C000002F900895EF92FF920F931F93CF9380E0AC
:10C01000E82E83E0F82E00EE14E0C0E0F7018191F5
:10C020007F010E947233882351F00E943F33F80150
:10C0300060837183828393838C2F0E94E930CF5F6A
:10C040000C5F1F4FC33051F7CF911F910F91FF909D
:10C05000EF90FCCD4F925F926F927F92AF92BF9222
:10C06000CF92DF92EF92FF920F931F93CF9380E0D6
:10C07000A82E83E0B82E0AE91DE0C0E0F501819109
:10C080005F010E947233882309F46DC0C33009F048
:10C0900063C00E943F336B017C0120E030E040EA46
:10C0A00051E40E9413AA87FF4EC0A7019601609138
:10C0B000A60D7091A70D8091A80D9091A90D0E94D9
:10C0C00053AF2B013C019B01AC0160915E0D70915F
:10C0D0005F0D8091600D9091610D0E9478AA609330
:10C0E0005E0D70935F0D8093600D9093610DA301C1
:10C0F00092016091960D7091970D8091980D90919D
:10C10000990D0E9478AA6093960D7093970D809375
:10C11000980D9093990D6091E6067091E7068091D5
:10C12000E8069091E9060E9417AAA30192010E94D5
:10C1300078AA0E94C0AF6093E6067093E7068093EA
:10C14000E8069093E906C092A60DD092A70DE09262
:10C15000A80DF092A90D07C00E943F33F80160833B
:10C16000718382839383CF5F0C5F1F4FC43009F0CC
:10C1700085CFCF911F910F91FF90EF90DF90CF90DF
:10C18000BF90AF907F906F905F904F900C942C8EEB
:10C1900083E50E947233882391F00E943F3320E0B0
:10C1A00030E04AE754E40E9478AA0E94C0AF60934E
:10C1B000E60C7093E70C8093E80C9093E90C0895DB
:10C1C00080E50E94B933811105C010920D041092D0
:10C1D0000C0408950E940F33672BB9F3089580E58E
:10C1E0000E94B933811106C083E50E94B9338823C8
:10C1F00059F005C00E941F3381110CC0F5CF0E9479
:10C200000F336F3F710510F06FEF70E070930D0406
:10C2100060930C040895CF93DF93ECE4FFE18491E5
:10C22000EF012196882321F00E942774FE01F7CFA9
:10C23000E8E3FDE08491EF012196882321F00E943C
:10C240002774FE01F7CFDF91CF9108952F923F928F
:10C250004F925F926F927F928F929F92AF92BF9216
:10C26000CF92DF92EF92FF920F931F93CF93DF93C2
:10C27000CDB7DEB7C957D1090FB6F894DEBF0FBEF0
:10C28000CDBFE091B00DF091B10DEF2B09F09CC73F
:10C290002896DFAECEAE28972E2C79016A015B017D
:10C2A000FC012081318142815381A4962CAF3DAFA6
:10C2B0004EAF5FAFA49720919A0D30919B0D4091A6
:10C2C0009C0D50919D0DA4966CAD7DAD8EAD9FAD36
:10C2D000A4970E9478AA0E94A8B0E0966CAF7DAFA8
:10C2E0008EAF9FAFE097D5018D919D910D90BC9140
:10C2F000A02DA8968CAF9DAFAEAFBFAFA8972091F1
:10C300009E0D30919F0D4091A00D5091A10DBC014B
:10C31000CD010E9478AA0E94A8B0E4966CAF7DAFD0
:10C320008EAF9FAFE497D6012D913D914D915C91D9
:10C33000AC962CAF3DAF4EAF5FAFAC972091A20D46
:10C340003091A30D4091A40D5091A50DAC966CAD0C
:10C350007DAD8EAD9FADAC970E9478AA0E94A8B02B
:10C36000E8966CAF7DAF8EAF9FAFE897D7012D9168
:10C370003D914D915C9122962CAF3DAF4EAF5FAF9A
:10C3800022972091A60D3091A70D4091A80D5091B4
:10C39000A90D22966CAD7DAD8EAD9FAD22970E940A
:10C3A00078AA0E94A8B060966CAF7DAF8EAF9FAFA9
:10C3B00060978091F10483FF1CC060962CAD3DAD69
:10C3C0004EAD5FAD609720938C0E30938D0E4093F1
:10C3D0008E0E50938F0E22968CAD9DADAEADBFAD3F
:10C3E000229780937C0E90937D0EA0937E0EB09347
:10C3F0007F0ED801BC91BDA3F801F181F9ABD80142
:10C400001296BC91BAABF801F381FAAF8091360E67
:10C410009091370E891B8F708F3019F40E9487908E
:10C42000F5CF0091360EE9960FAFE9978091360E61
:10C43000082F10E01CA30BA38091800E9091810E19
:10C44000A091820EB091830EE0964CAC5DAC6EACC8
:10C450007FACE097481A590A6A0A7B0A8091840ED9
:10C460009091850EA091860EB091870EE4962CAD2A
:10C470003DAD4EAD5FADE497281B390B4A0B5B0B0E
:10C480002DA73EA74FA758AB8091880E9091890E9B
:10C49000A0918A0EB0918B0EE8968CAC9DACAEACA0
:10C4A000BFACE897881A990AAA0ABB0A80918C0E39
:10C4B00090918D0EA0918E0EB0918F0E60960CAD66
:10C4C0001DAD2EAD3FAD6097081B190B2A0B3B0B22
:10C4D00009A71AA72BA73CA7012B022B032B09F4B2
:10C4E000BAC060910F047091100480911104909172
:10C4F000120420910E04211141C00E94BBAF209173
:10C50000290230912A0262177307C4F560962CAD98
:10C510003DAD4EAD5FAD609720938C0E30938D0E88
:10C5200040938E0E50938F0E22968CAD9DADAEAD86
:10C53000BFAD229780937C0E90937D0EA0937E0ECC
:10C54000B0937F0EEEEDFEE184918F010F5F1F4FE0
:10C55000882321F00E942774F801F6CFE9E2F0E188
:10C5600084918F010F5F1F4F882321F00E94277451
:10C57000F801F6CF19A61AA61BA61CA669A57AA5CE
:10C580008BA59CA50E9419AAA4E02A9EF001112463
:10C59000EB5DFD4F20813181428153810E9478AA59
:10C5A0006B017C0120E030E0A9010E949DB087FF73
:10C5B00004C0F7FAF094F7F8F0946091A60D70912A
:10C5C000A70D8091A80D9091A90D0E94BBAF9B0172
:10C5D000AC01A8ECB0E00E945DAE0E9419AA9B01DC
:10C5E000AC01C701B6010E949DB01816C4F5609653
:10C5F0000CAD1DAD2EAD3FAD609700938C0E10932A
:10C600008D0E20938E0E30938F0E22962CAD3DAD65
:10C610004EAD5FAD229720937C0E30937D0E4093FC
:10C620007E0E50937F0EEEEDFEE184918F010F5F41
:10C630001F4F882321F00E942774F801F6CFEAE00B
:10C64000F0E184918F010F5F1F4F882321F00E943A
:10C650002774F801F6CF19A61AA61BA61CA6D301AB
:10C66000C2018827B7FD83959927AA27BB27182FD2
:10C670002DA53EA54FA558A957FD1260B7FC146023
:10C6800089A59AA5ABA5BCA5B7FD186069A57AA533
:10C690008BA59CA50E9419AAA4E02A9EF001112452
:10C6A000EB5DFD4F20813181428153810E9478AA48
:10C6B0006B017C0120E030E0A9010E949DB087FF62
:10C6C00004C0C701B601905802C0C701B60120E0FE
:10C6D00030E040E05FE30E9477AE0E94C0AF6EABF7
:10C6E0007FAB88AF99AF88E52BA13CA1829FF00179
:10C6F000839FF00D1124E650F94F108216ABB30161
:10C70000A20177FE07C044275527BA0144195509ED
:10C710006609770988E50BA11CA1809FF001819F24
:10C72000F00D1124E650F94F458B568B678B708FB7
:10C730008DA59EA5AFA5B8A926968CAF9DAFAEAF2F
:10C74000BFAF2697B7FF0DC0B095A0959095819586
:10C750009F4FAF4FBF4F26968CAF9DAFAEAFBFAFD1
:10C76000269728E50BA11CA1209FF001219FF00D29
:10C770001124E650F94F26968CAD9DADAEADBFAD00
:10C780002697818F928FA38FB48F95018401B7FE76
:10C7900007C0002711279801081919092A093B0920
:10C7A000E8E53E2EABA1BCA13A9EC0013B9E900D98
:10C7B0001124FC01E650F94F058F168F278F30A307
:10C7C0008EA99FA9A8ADB9AD81A392A3A3A3B4A339
:10C7D00026968CAD9DADAEADBFAD2697841795075F
:10C7E000A607B70710F4DB01CA0180179107A2075B
:10C7F000B30710F4D901C8010EA91FA928AD39AD9E
:10C8000080179107A207B30710F4D901C80128E5E2
:10C810000BA11CA1209FF001219FF00D1124E650D7
:10C82000F94F85A396A3A7A3B0A70697A105B105C5
:10C8300008F4C3C4DF01AE5ABF4F80910C0490913D
:10C840000D048D939C9321A6452B462B472B09F075
:10C85000179888E50BA11CA1809FF001819FF00D26
:10C860001124E650F94F818D928DA38DB48D892BC3
:10C870008A2B8B2B09F0169888E50BA11CA1809FB1
:10C88000F001819FF00D1124E650F94F858D968DB2
:10C89000A78DB0A1892B8A2B8B2B09F015982EA977
:10C8A0003FA948AD59AD232B242B252B09F48EC469
:10C8B00080910B04882319F0815080930B04211080
:10C8C00004C0149880E280930B042090660D309091
:10C8D000670D0091680D1091690D9101A8016DA17E
:10C8E00079A98AA99AAD0E9413AA87FF04C02DA234
:10C8F00039AA0AAB1AAFC301B2010E9419AA20914A
:10C90000EA063091EB064091EC065091ED060E944C
:10C9100078AA26966CAF7DAF8EAF9FAF2697698BB6
:10C920007A8B8B8B9C8B6DA57EA58FA598A90E9479
:10C9300019AA2091EE063091EF064091F006509131
:10C94000F1060E9478AA2B013C016D8B7E8B8F8BA8
:10C95000988FC501B4010E9419AA2091F206309166
:10C96000F3064091F4065091F5060E9478AA4B0117
:10C970005C01698F7A8F8B8F9C8F2091F6063091A6
:10C98000F7064091F8065091F906C701B6010E94DA
:10C9900078AA6B017C016D8F7E8F8F8F98A388E5BD
:10C9A0000BA11CA1809FF001819FF00D1124E65086
:10C9B000F94F258936894789508D2DA73EA74FA766
:10C9C00058AB263031054105510508F408C42896B6
:10C9D000AEADBFAD2897CD90DD90ED90FC9020E0FE
:10C9E00030E0A901C701B6010E9413AA811116C443
:10C9F00026962CAD3DAD4EAD5FAD2697CA01B9016F
:10CA00000E9478AA6B017C01A3019201C301B201CB
:10CA10000E9478AA9B01AC01C701B6010E9477AEC3
:10CA20006B017C01A5019401C501B4010E9478AAA3
:10CA30009B01AC01C701B6010E9477AE0E94E2B033
:10CA400028E50BA11CA1209FF001219FF00D1124CE
:10CA5000E650F94F658776878787908B88E50BA12D
:10CA60001CA1809FF001819FF00D1124E650F94F29
:10CA700085849684A784B088A501940160E070E065
:10CA800080E89FE30E9453AF66966CAF7DAF8EAF98
:10CA90009FAF66979B01AC016DA179A98AA99AAD58
:10CAA0000E9478AA2B013C018091360E9091340EA1
:10CAB000891B8F7027968FAF2797A301920160E0A3
:10CAC00074E284E799E40E9453AF0E94A8B06B011E
:10CAD0007C0127968FAD27978250863008F4ADC32E
:10CAE000A3019201C501B4010E9478AA9B01AC0187
:10CAF0000E9478AA6A966CAF7DAF8EAF9FAF6A979F
:10CB000088E5ABA1BCA18A9F80018B9F100D1124E9
:10CB10000650194F6A962CAD3DAD4EAD5FAD6A978C
:10CB2000D80111962D933D934D935C931497959650
:10CB30002D913D914D915C9198972AAB3BAB4CABBD
:10CB40005DABCA01B9010E9417AA6AAF7BAF8CAF77
:10CB50009DAFA30192010E9478AA0E943DAF0E945E
:10CB6000C0AF4B015C01F801EE5BFF4F6083718346
:10CB7000828393838E010F5E1F4F2A961FAF0EAFE5
:10CB80002A970051110924961FAF0EAF24970AE887
:10CB90001DE0A0961FAF0EAFA0978E010F5D1F4F37
:10CBA0001AA309A324960EAD1FAD249762961FAF5A
:10CBB0000EAF6297312C212C10E81DA30FE309ABB7
:10CBC0002A96AEADBFAD2A976D917D918D919D91C5
:10CBD0002A96BFAFAEAF2A97A30192010E9478AA0E
:10CBE0006B017C016296EEADFFAD6297619371932C
:10CBF000819391936296FFAFEEAF629720E030E0B1
:10CC0000A9010E949DB087FF04C0F7FAF094F7F8DD
:10CC1000F094A096AEADBFADA0970D911D912D9152
:10CC20003D91A096BFAFAEAFA0976E960CAF1DAF73
:10CC30002EAF3FAF6E97A9019801C701B6010E94C0
:10CC40009DB018160CF433C32A960EAD1FAD2A976B
:10CC500029A13AA10217130709F0B2CF20E030E072
:10CC600040E85FE3632D722D8DA199A90E9413AA5C
:10CC700087FF56C07E0131E1E30EF11C24960EAD14
:10CC80001FAD2497232D322D4DA159A9D8016D91A7
:10CC90007D918D919C910E9478AAF8016193719386
:10CCA000819391938F01EE15FF0561F728E50BA1A4
:10CCB0001CA1209FC001219F900D11249C01265092
:10CCC000394F790189010E5B1F4FC501B4010E94E4
:10CCD00017AA232D322D4DA159A90E9478AA0E948E
:10CCE000C0AFD8016D937D938D939C931397232DA3
:10CCF000322D4DA159A9632D722D8DA199A90E94A4
:10CD000078AA9B01AC016A966CAD7DAD8EAD9FADEE
:10CD10006A970E9478AAF701618372838383948360
:10CD200066962CAD3DAD4EAD5FAD66976AAD7BAD01
:10CD30008CAD9DAD0E9478AA6DA37EA38FA398A70A
:10CD40000DA51EA52FA538A9012B022B032B09F039
:10CD5000CAC288E52BA13CA1829F8001839F100D50
:10CD600011240650194FF801818D928DA38DB48D39
:10CD7000892B8A2B8B2B09F0B6C2858D968DA78DBA
:10CD8000B0A1892B8A2B8B2B09F0ADC22091720D9B
:10CD90003091730D4091740D5091750D6DA17EA170
:10CDA0008FA198A50E9478AA0E943DAF0E94C0AFB3
:10CDB0002B013C01D801D7961C9288E52BA13CA100
:10CDC000829F8001839F100D11240650194FF80196
:10CDD000E25BFF4F4082518262827382C301B201E3
:10CDE0000E9417AA6B017C012DA13EA14FA158A55D
:10CDF0000E9453AF6AAF7BAF8CAF9DAFD801519605
:10CE00006D937D938D939C9354972DEB37E346E080
:10CE100051E4C701B6010E9478AA0E94C0AFF80190
:10CE200062AB73AB84AB95AB87A9882371F1FE9697
:10CE300020813181428153816091350D7091360D91
:10CE40008091370D9091380D0E9478AA2AAD3BADA4
:10CE50004CAD5DAD0E9478AA2091A60D3091A70D32
:10CE60004091A80D5091A90D0E9478AA9B01AC0198
:10CE700060E074E284EF99E40E9453AF0E94C0AF77
:10CE8000D801D9967C936E93D89788E50BA11CA105
:10CE9000809FF001819FF00D1124E650F94F218110
:10CEA0003281438154812C962CAF3DAF4EAF5FAFA2
:10CEB0002C97CA01B9010E94E2B0162F072F382E15
:10CEC000292E42E55DE062965FAF4EAF62973E016C
:10CED00051E1650E711C82E59DE09BAB8AAB249607
:10CEE0004EAC5FAC249719A70DA73DA229AA1EAA94
:10CEF000D201CD90DD90ED90FD902D0120E030E04D
:10CF0000A901C701B6010E949DB087FF04C0F7FACE
:10CF1000F094F7F8F094EAA9FBA981909190A19080
:10CF2000B190FBABEAABA5019401C701B6010E9429
:10CF30009DB018160CF4F6C446145704C9F659A54A
:10CF400067965FAF67978DA56B968FAF6B979DA127
:10CF50006F969FAF6F97A9A9EA96AFAFEA9727960A
:10CF6000BFAD2797B1111EC567968FAD67976B96BA
:10CF70009FAD6B976F96AFAD6F97EA96BFADEA978F
:10CF80008093070490930804A0930904B0930A04C3
:10CF900088E54BA15CA1849F8001859F100D112421
:10CFA0000650194F29A53DA54DA159A969A57DA5F3
:10CFB0008DA199A90E9478AAD80119966D937D93A5
:10CFC0008D939C931C976AAD7BAD8CAD9DAD9058B5
:10CFD0009B01AC010E9477AEF80125853685478517
:10CFE00050890E9478AA9B01AC016BE077ED83E247
:10CFF0009BE30E9476AE9B01AC018BE097EDA3E230
:10D00000BBE3F80185839683A783B08710812C96B4
:10D010006CAD7DAD8EAD9FAD2C970E9413AA1816F6
:10D020000CF0FEC581E0182B88E52BA13CA1829F66
:10D03000F001839FF00D1124E650F94F108380E139
:10D04000FE013196A0E6BEE001900D928A95E1F7CF
:10D050002C968CAD9DADAEADBFAD2C9780935C0E84
:10D0600090935D0EA0935E0EB0935F0EE0960CADB4
:10D070001DAD2EAD3FADE0970093800E1093810E55
:10D080002093820E3093830EE4962CAD3DAD4EADD1
:10D090005FADE4972093840E3093850E4093860E07
:10D0A0005093870EE8968CAD9DADAEADBFADE897C1
:10D0B0008093880E9093890EA0938A0EB0938B0E66
:10D0C00060960CAD1DAD2EAD3FAD609700938C0EFC
:10D0D00010938D0E20938E0E30938F0EA4962CAD50
:10D0E0003DAD4EAD5FADA4972093700E3093710EA1
:10D0F0004093720E5093730EA8968CAD9DADAEAD5D
:10D10000BFADA8978093740E9093750EA093760E82
:10D11000B093770EAC960CAD1DAD2EAD3FADAC9778
:10D120000093780E1093790E20937A0E30937B0E35
:10D1300022962CAD3DAD4EAD5FAD229720937C0E77
:10D1400030937D0E40937E0E50937F0E9091360E5D
:10D150008091370E981303C084E68093330EE996CE
:10D160008FADE9978F5F8F708093360E8091360E6A
:10D170009091350E81508F70891354C50091370EF0
:10D180000BA31091360E19A798E509A51BA1011351
:10D19000D2C5812C912CA12CB12C1DA61DA219AA9F
:10D1A0001EAE212C312C00E010E0FBA129A5F213CA
:10D1B000CFC52114310409F080C680916F008260D0
:10D1C00080936F0081E0DEC780E0DCC72090620DB5
:10D1D0003090630D0091640D1091650D7ECB818DB3
:10D1E000928DA38DB48D0697A105B10508F0EFCB04
:10D1F000858D968DA78DB0A10697A105B10508F084
:10D20000E6CB20E030E0A901C701B6010E949DB045
:10D2100087FF04C0F7FAF094F7F8F09488E50BA1C3
:10D220001CA1809FF001819FF00D1124E650F94F61
:10D23000C586D686E786F08A11CC80916A0D9091DA
:10D240006B0DA0916C0DB0916D0DC816D906EA0654
:10D25000FB0608F045CC8C199D09AE09BF09BC013D
:10D26000CD01660F771F881F991F27964FAD27970F
:10D27000042F10E020E030E0A90198010E941FAEC9
:10D28000CA01B9010E9417AA0E94A8B06C0D7D1DA9
:10D290008E1D9F1D0E9417AA9B01AC0160E074E2E5
:10D2A00084E799E40E9453AF2B013C0119CCA701FC
:10D2B00096016E966CAD7DAD8EAD9FAD6E970E9462
:10D2C00053AF7B018C019B01AC01632D722D8DA1AD
:10D2D00099A90E949DB018160CF0B6CC3E2C2F2CAC
:10D2E0000DA319ABB1CC0EA91FA928AD39AD012BE7
:10D2F000022B032B49F06091760D7091770D809190
:10D30000780D9091790D08C060916E0D70916F0D40
:10D310008091700D9091710D2DA13EA14FA158A546
:10D320000E9478AA0E943DAF0E94C0AF2B013C0131
:10D330002EA93FA948AD59AD232B242B252BC9F08D
:10D3400020E030E0A9016091350D7091360D80919B
:10D35000370D9091380D0E9413AA882351F081E077
:10D3600009A51AA52BA53CA5101611061206130631
:10D370000CF080E098E52BA13CA1929F8001939F47
:10D38000100D11240650194FD801D7968C9388237D
:10D3900009F4B2C02091700E3091710E4091720E5E
:10D3A0005091730EA4966CAD7DAD8EAD9FADA497DC
:10D3B0000E9476AE69A77AA78BA79CA72091740ECE
:10D3C0003091750E4091760E5091770EA8966CAD07
:10D3D0007DAD8EAD9FADA8970E9476AE4B015C01EE
:10D3E0002091780E3091790E40917A0E50917B0EFB
:10D3F000AC966CAD7DAD8EAD9FADAC970E9476AE18
:10D400006B017C0129A53AA54BA55CA5CA01B90110
:10D410000E9478AA69A77AA78BA79CA7A501940167
:10D42000C501B4010E9478AA9B01AC0169A57AA547
:10D430008BA59CA50E9477AE4B015C01A7019601CC
:10D44000C701B6010E9478AA9B01AC01C501B401D5
:10D450000E9477AE0E94E2B06B017C0120917C0EAD
:10D4600030917D0E40917E0E50917F0E22966CADD4
:10D470007DAD8EAD9FAD22970E9476AEA70196013D
:10D480000E9453AF6B017C01F801FE9660837183AB
:10D490008283938320E030E040E450E40E949DB01A
:10D4A00018161CF4F80117AA27C02091350D3091E9
:10D4B000360D4091370D5091380DC701B6010E94CD
:10D4C00078AA9B01AC0160915E0D70915F0D809117
:10D4D000600D9091610D0E9453AF2DA13EA14FA10F
:10D4E00058A50E9478AA0E94C0AF641575058605EC
:10D4F000970510F42B013C018091D6069091D70638
:10D50000A091D806B091D9060AA91BA92CA93DA9BA
:10D5100080179107A207B30708F4E9C02DA53EA51F
:10D520004FA558A9232B242B252B61F12091DA0636
:10D530003091DB064091DC065091DD06241535055F
:10D5400046055705F8F46AA97BA98CA99DA90E94F4
:10D5500010AE6B017C01A30192016DA57EA58FA584
:10D5600098A90E9410AEC616D706E806F90650F430
:10D57000C701B6012DA53EA54FA558A90E941FAE13
:10D5800029013A0188E50BA11CA1809FF001819F30
:10D59000F00D1124E650F94FC18CD28CE38CF48C41
:10D5A000C114D104E104F10441F12091DE0630916F
:10D5B000DF064091E0065091E10624153505460549
:10D5C0005705D8F46AA97BA98CA99DA90E9410AE21
:10D5D0004B015C01A3019201C701B6010E9410AE8C
:10D5E00086169706A806B90640F4C501B401A7013E
:10D5F00096010E941FAE29013A0188E50BA11CA1EA
:10D60000809FF001819FF00D1124E650F94FC58CE9
:10D61000D68CE78CF0A0C114D104E104F10441F1EF
:10D620002091E2063091E3064091E4065091E50630
:10D630002415350546055705D8F46AA97BA98CA998
:10D640009DA90E9410AE4B015C01A3019201C7018C
:10D65000B6010E9410AE86169706A806B90640F4D9
:10D66000C501B401A70196010E941FAE29013A012C
:10D6700088E50BA11CA1809FF001819FF00D112472
:10D68000E650F94FC1A0D2A0E3A0F4A0C114D10488
:10D69000E104F10409F491CB2091E6063091E7060C
:10D6A0004091E8065091E9062415350546055705D1
:10D6B00008F083CB6AA97BA98CA99DA90E9410AE12
:10D6C0004B015C01A3019201C701B6010E9410AE9B
:10D6D00086169706A806B90608F06FCBC501B401F7
:10D6E000A70196010E941FAE29013A0166CB2DA524
:10D6F0003EA54FA558A9232B242B252BB9F16091CA
:10D70000DA067091DB068091DC069091DD066415E7
:10D7100075058605970550F50E9417AA2AAD3BAD01
:10D720004CAD5DAD0E9478AA6B017C016DA57EA514
:10D730008FA598A90E9417AA4B015C01C301B201F1
:10D740000E9417AAA50194010E9478AAA701960138
:10D750000E949DB0181654F4A5019401C701B601AA
:10D760000E9453AF0E94C0AF2B013C0188E50BA182
:10D770001CA1809FF001819FF00D1124E650F94F0C
:10D78000818C928CA38CB48C81149104A104B1047B
:10D79000A9F16091DE067091DF068091E00690911C
:10D7A000E106641575058605970540F50E9417AAE0
:10D7B0002AAD3BAD4CAD5DAD0E9478AA6B017C01FA
:10D7C000C501B4010E9417AA4B015C01C301B2015B
:10D7D0000E9417AAA50194010E9478AAA7019601A8
:10D7E0000E949DB0181654F4A5019401C701B6011A
:10D7F0000E9453AF0E94C0AF2B013C0188E50BA1F2
:10D800001CA1809FF001819FF00D1124E650F94F7B
:10D81000858C968CA78CB0A081149104A104B104CE
:10D82000A9F16091E2067091E3068091E40690917F
:10D83000E506641575058605970540F50E9417AA4B
:10D840002AAD3BAD4CAD5DAD0E9478AA6B017C0169
:10D85000C501B4010E9417AA4B015C01C301B201CA
:10D860000E9417AAA50194010E9478AAA701960117
:10D870000E949DB0181654F4A5019401C701B60189
:10D880000E9453AF0E94C0AF2B013C0188E50BA161
:10D890001CA1809FF001819FF00D1124E650F94FEB
:10D8A000C1A0D2A0E3A0F4A0C114D104E104F1040A
:10D8B00009F483CA6091E6067091E7068091E80654
:10D8C0009091E906641575058605970508F075CAF7
:10D8D0000E9417AA2AAD3BAD4CAD5DAD0E9478AA5F
:10D8E0004B015C01C701B6010E9417AA6B017C01C4
:10D8F000C301B2010E9417AAA70196010E9478AA4B
:10D90000A50194010E949DB018160CF056CAA701FB
:10D910009601C501B4010E9453AF0E94C0AF2B0114
:10D920003C014BCAFEA9FF2329F1A5019401612FF7
:10D93000702F832D922D0E9478AA4B015C0129A59E
:10D940003DA54DA159A9C701B6010E9478AAA5011C
:10D9500094010E949DB0181614F5A7019601C50107
:10D96000B4010E9453AF69A77DA78DA399AB21E0B5
:10D970002EABE2CAA7019601C501B4010E9453AFC4
:10D980009B01AC0169A57DA58DA199A90E9478AAEA
:10D9900069A77DA78DA399AB31E03EABCDCA41E02D
:10D9A0004EABCACAC0905C0ED0905D0EE0905E0E89
:10D9B000F0905F0E2DEB37E346E855E3C701B60163
:10D9C0000E9413AA87FDD0CAC701B6010E94E2B027
:10D9D0006B017C019B01AC01612F702F832D922D77
:10D9E0000E9413AA87FD04C01C2D0D2D3E2C2F2C48
:10D9F0009601A701612F702F832D922D0E9453AFA6
:10DA000066966CAF7DAF8EAF9FAF6697E0E6FEE0A7
:10DA10002896FFAFEEAF289720E030E040E85FE3C4
:10DA20002EAB3FAB48AF59AF1AAA2896AEADBFADEB
:10DA300028976D917D918D919D912896BFAFAEAF46
:10DA4000289766962CAD3DAD4EAD5FAD66970E94B2
:10DA500078AA6B017C012496EEADFFAD24978190EE
:10DA60009190A190B1902496FFAFEEAF2497FAA9C0
:10DA7000FF2391F02EA93FA948AD59AD0E9478AA85
:10DA80006B017C012EA93FA948AD59ADC501B40178
:10DA90000E9478AA4B015C01A5019401C701B6015F
:10DAA0000E949DB020E030E0A90118162CF5C501B8
:10DAB000B4010E949DB018164CF020E030E0A9019E
:10DAC000C701B6010E9413AA87FF05C0A5019401F2
:10DAD000C701B60124C02401350177FA709477F8A4
:10DAE0007094A3019201C701B6010E949DB018165F
:10DAF0005CF52601370128C0C501B4010E9413AAB4
:10DB000087FD09C020E030E0A901C701B6010E94ED
:10DB10009DB018164CF4A7019601C501B4010E94EE
:10DB200076AE2B013C0110C02601370177FA7094C4
:10DB300077F87094A5019401C301B2010E949DB0D1
:10DB4000181614F0240135016296AEADBFAD629790
:10DB5000CD90DD90ED90FD906296BFAFAEAF629735
:10DB6000A7019601C301B2010E949DB01816ACF442
:10DB7000A3019201C701B6010E9453AF9B01AC0102
:10DB80006EA97FA988AD99AD0E9478AA6EAB7FABD4
:10DB900088AF99AFBAA9BF5FBAAB2896EEADFFAD1B
:10DBA0002897E057FE4009F040CF3AA9332371F09F
:10DBB0002EA93FA948AD59AD612F702F832D922D0D
:10DBC0000E9478AA162F072F382E292E24EA30E734
:10DBD0004DE75FE3612F702F832D922D0E9478AA6D
:10DBE0006B017C019B01AC016091070470910804FA
:10DBF0008091090490910A040E949DB018165CF46B
:10DC0000A701960169A57DA58DA199A90E949DB046
:10DC100018160CF4A9C919A70DA73DA229AAA4C9D1
:10DC200083E001CAF090360E8FEF8F0D8F708BA3BB
:10DC3000B090350E8091360EB81206C00091350EA8
:10DC40000BA3C12CD12C69C0C12CD12C1BA11B153D
:10DC5000A9F31BA1812E912C28E5289D8001299DE7
:10DC6000100D11240650194FD8018C9183FD27C047
:10DC700009AB1EAF0115110521F11996BC91B9A789
:10DC8000F801F285FDA7D8011B96BC91BDA3F80150
:10DC9000A484458056806780708429A53DA54B2FBC
:10DCA0005A2DC301B2010E9413AA81117FC1C11470
:10DCB000D10439F0D6018C9180FD78C102C0C9AA87
:10DCC000DEAE8BA181508F708BA38091350EB8167C
:10DCD00049F00BA10B1509F4B1CF81E08B0D8F70CA
:10DCE000B82EF3CFC9A8DEACB1CF0BA1802E912CFA
:10DCF00028E5289D8001299D100D11240650194FFB
:10DD0000D8018C9183FD15C05801C114D10459F478
:10DD10008BA18F5F8F708BA365018091360E1BA145
:10DD20001813E3CF2BCAC6010E94EFA08111F0CFD8
:10DD3000B3C15601EDCF89A581508F70989FF00136
:10DD40001124E650F94F208123FF23CA89A71DCA59
:10DD500028E53BA1239FC0011124AC014650594F37
:10DD60001A01DA018C9183FD19C015966D917D9190
:10DD70008D919C9118970E94E2B0F62EE72ED82E36
:10DD8000C92E0115110509F48AC0F801808180FDB2
:10DD90000AC0D1018C9180FD06C081C0FDA4EDA018
:10DDA000D9A8CEAC81C0F801808181608083C80190
:10DDB0000E94EFA081116FC0F8016181728183819F
:10DDC00094810E94E2B02B013C019B01AC0160E018
:10DDD00070E080E89FE30E9453AF4B015C019B0120
:10DDE000AC016F2D7E2D8D2D9C2D0E9478AA69830C
:10DDF0007A838B839C83A50194016DA57DA189A95C
:10DE00009EAD0E9478AA698B7A8B8B8B9C8BAE011E
:10DE10004F5F5F4FBE016F5E7F4FC8010E94713C34
:10DE2000D801D7968C918823B1F12091350D30918E
:10DE3000360D4091370D5091380DF801FE966081F6
:10DE40007181828193810E9478AA2091A60D3091E0
:10DE5000A70D4091A80D5091A90D0E9478AA4B01E1
:10DE60005C019B01AC01C301B2010E9478AA0E942F
:10DE7000C0AFF80173AF62AFA50194016F2D7E2D85
:10DE80008D2D9C2D0E9478AA0E94C0AFD801DD96EE
:10DE90007C936E93DC97F80180818E7F80838F2C3A
:10DEA0009E2CAD2CBC2C81018BA18F5F8F708BA31E
:10DEB000FDA6EDA2D9AACEAE78C9D1018C91816020
:10DEC0008C93C8010E94EFA081116BC0F1016181A8
:10DED0007281838194810E94E2B06B017C019B017D
:10DEE000AC0160E070E080E89FE30E9453AF2B013B
:10DEF0003C012DEC3CEC4CE45DE30E9478AA698384
:10DF00007A838B839C83A3019201B401C5010E9493
:10DF100078AA698B7A8B8B8B9C8BAE014F5F5F4F9E
:10DF2000BE016F5E7F4FC1010E94713CD101D79647
:10DF30008C918823B1F12091350D3091360D4091AF
:10DF4000370D5091380DF101FE966081718182810B
:10DF500093810E9478AA2091A60D3091A70D40913F
:10DF6000A80D5091A90D0E9478AA4B015C019B015C
:10DF7000AC01C701B6010E9478AA0E94C0AFF101AE
:10DF800073AF62AF2DEC3CEC4CE45DE3C501B40132
:10DF90000E9478AA0E94C0AFD101DD967C936E9357
:10DFA000DC97F10180818E7F808307C928E5289D59
:10DFB000F001299DF00D1124E650F94F808181FD7B
:10DFC0003FC0C114D10431F0F601C580D680E7808E
:10DFD000F08408C08BE0C82E87EDD82E83E2E82EAF
:10DFE0008BE3F82E28E5289DF001299DF00D1124E2
:10DFF000E650F94F81899289A389B489BC01CD018A
:10E0000090589B01AC010E9477AED8011D962D91CE
:10E010003D914D915C9150970E9478AA9B01AC0173
:10E02000C701B6010E9476AE1B016C019B01AC01D9
:10E0300069A57DA58DA19A2D0E9413AA87FF04C012
:10E0400029A43DA4CDA0DA2C9101A601C301B201FF
:10E050000E9413AA882309F434CEB8E5B89DC00104
:10E06000B99D900D1124FC01E650F94F4F018081BC
:10E0700081608083C8010E94EFA0882329F0D40129
:10E080008C918E7F8C931DCEC101D601F4018583C6
:10E090009683A783B08715CED6018C9181FD50C0A1
:10E0A000D60115962D913D914D915C91189729A718
:10E0B0003AA74BA75CA71501B5E02B0E311CF80160
:10E0C0004580568067807084A301920169A57AA576
:10E0D0008BA59CA50E9413AA87FF32C0F6018189F7
:10E0E0009289A389B489BC01CD0190589B01AC01F0
:10E0F0000E9477AED6011D962D913D914D915C9178
:10E1000050970E9478AA9B01AC0169A57AA58BA5BE
:10E110009CA50E9476AE6B017C01A30192010E9436
:10E1200013AA87FF0DC0D8018C9181608C93C50123
:10E130000E94EFA08823E1F0F80180818E7F808328
:10E1400018E5189DF001199DF00D1124E650F94FC6
:10E1500021853285438554856581768187819085C7
:10E160000E9413AA8111D4CD0BA10093350ED0CDFE
:10E17000D101CD92DD92ED92FC9213970BA1009309
:10E18000350EDECFC758DF4F0FB6F894DEBF0FBE97
:10E19000CDBFDF91CF911F910F91FF90EF90DF9056
:10E1A000CF90BF90AF909F908F907F906F905F9037
:10E1B0004F903F902F9008958091360E9091370E9A
:10E1C000891B8F708F3019F40E948790F5CF809152
:10E1D000360E8F5F8F70E091360E98E59E9FF001AE
:10E1E0001124E650F94FDF011D929A95E9F798E066
:10E1F00090834091800E5091810E6091820E7091BB
:10E20000830E458B568B678B708F4091840E509197
:10E21000850E6091860E7091870E418F528F638FAD
:10E22000748F4091880E5091890E60918A0E709182
:10E230008B0E458F568F678F70A340918C0E509137
:10E240008D0E60918E0E70918F0E41A352A363A329
:10E2500074A32091360E9091370E291303C094E6D3
:10E260009093330E8093360E80916F00826080937E
:10E270006F0008959091360E8091370E981719F01F
:10E280000E948790F7CF8091B00D9091B10D892BAE
:10E29000B9F708959091360E8091370E981719F0BE
:10E2A0000E948790F7CF8091B00D9091B10D892B8E
:10E2B000B9F70C944490CF93DF9390916F0091FB4A
:10E2C000222720F991FF05C090916F009D7F9093C8
:10E2D0006F0094E0899FE0011124FE01E954F24FA0
:10E2E0006081718182819381222329F020916F00C6
:10E2F000226020936F000E9419AAC651D94F28812D
:10E3000039814A815B810E9478AADF91CF9108957B
:10E310002F923F924F925F926F927F928F929F9235
:10E32000AF92BF92CF92DF92EF92FF920F931F9323
:10E33000CF93DF93CDB7DEB7E8970FB6F894DEBF83
:10E340000FBECDBF2091510D222309F4E6C01C0160
:10E3500000913C0E10913D0E20913E0E30913F0EEB
:10E360004090400E5090410E6090420E7090430ECF
:10E370004DA65EA66FA678AA8090440E9090450E9A
:10E38000A090460EB090470E4091480E5091490E15
:10E3900060914A0E70914B0E80914C0E90914D0EF3
:10E3A000A0914E0EB0914F0E89AB9AABABABBCAB0C
:10E3B000C090500ED090510EE090520EF090530E3F
:10E3C0008091540E9091550EA091560EB091570E1B
:10E3D0004090580E5090590E60905A0E70905B0EFF
:10E3E0004DAA5EAA6FAA78AE4090380E5090390EB2
:10E3F00060903A0E70903B0E49825A826B827C820A
:10E400008D829E82AF82B886C986DA86EB86FC86CC
:10E410000D871E872F87388B498B5A8B6B8B7C8B94
:10E420008D8B9E8BAF8BB88F8DA59EA5AFA5B8A900
:10E43000898F9A8FAB8FBC8F49A85AA86BA87CA8EC
:10E440004D8E5E8E6F8E78A28DA99EA9AFA9B8ADB4
:10E4500089A39AA3ABA3BCA320E030E040E450E43E
:10E46000D1016D917D918D919C910E9477AE69A7AC
:10E470007AA78BA79CA72DEC3CEC46E353E4F10173
:10E4800064817581868197810E9476AE6DA37EA39B
:10E490008FA398A7C10108969F938F93CE0185966D
:10E4A0009F938F9304969F938F938DB79EB7849776
:10E4B0000FB6F8949EBF0FBE8DBFADB7BEB7119615
:10E4C00084E2FE01319601900D928A95E1F70E9457
:10E4D000EE4420E030E040E450E469A57AA58BA545
:10E4E0009CA50E9476AED1016D937D938D939C93F4
:10E4F00013972DEC3CEC46E353E46DA17EA18FA174
:10E5000098A50E9477AEF101648375838683978313
:10E510000FB6F894DEBF0FBECDBFE8960FB6F894E5
:10E52000DEBF0FBECDBFDF91CF911F910F91FF9046
:10E53000EF90DF90CF90BF90AF909F908F907F90A3
:10E540006F905F904F903F902F900895CF92DF9201
:10E55000EF92FF920F931F93CF93DF93CDB7DEB768
:10E5600028970FB6F894DEBF0FBECDBF2091510D96
:10E57000222309F462C0C52ED42E8B017C0120E039
:10E5800030E040E450E4FC0160817181828193813C
:10E590000E9477AE6D837E838F8398872DEC3CEC51
:10E5A00046E353E4F80160817181828193810E9486
:10E5B00076AE69837A838B839C83CF92DF92CE0180
:10E5C00001969F938F9304969F938F938DB79EB7D9
:10E5D00084970FB6F8949EBF0FBE8DBFADB7BEB780
:10E5E000119684E2E8E3FEE001900D928A95E1F74E
:10E5F0000E94EE4420E030E040E450E46D817E81F2
:10E600008F8198850E9476AEF70160837183828343
:10E6100093832DEC3CEC46E353E469817A818B8152
:10E620009C810E9477AEF80160837183828393831B
:10E630000FB6F894DEBF0FBECDBF28960FB6F89484
:10E64000DEBF0FBECDBFDF91CF911F910F91FF9025
:10E65000EF90DF90CF900895CF92DF92EF92FF92EC
:10E660008091AE0D882371F1C090AA0DD090AB0DB2
:10E67000E090AC0DF090AD0D20E030E0A901C701B5
:10E68000B6010E9413AA8823E9F020E030E040E0C0
:10E690005FE3C701B6010E9478AA9B01AC010E940A
:10E6A00078AA2BED3FE049E450E40E9478AA9B0150
:10E6B000AC0160E070E080E89FE30E9453AF6B0123
:10E6C0007C0106C0C12CD12C80E8E82E8FE3F82E07
:10E6D000C0920304D0920404E0920504F092060470
:10E6E0006091230270912402072E000C880B990B75
:10E6F0000E9419AA2AE037ED43E25CE30E9478AA5F
:10E70000A70196010E9478AA6093250270932602C1
:10E710008093270290932802FF90EF90DF90CF9094
:10E7200008958F929F92AF92BF92CF92DF92EF9215
:10E73000FF920F931F93CF93DF93CDB7DEB72C9744
:10E740000FB6F894DEBF0FBECDBF8B0140E050E0A6
:10E7500068EC72E44D835E836F83788740E050E01D
:10E7600060EA70E449835A836B837C83FC01808177
:10E77000813019F0823039F02AC0BE016F5F7F4FBF
:10E78000C801089646C0F801208531854285538529
:10E790006091190E70911A0E80911B0E90911C0EB3
:10E7A0000E9477AE6B017C0120E030E04FE153E442
:10E7B0000E9413AA87FD06C0C12CD12C8FE1E82E40
:10E7C00083E4F82EC986DA86EB86FC861DC080902D
:10E7D000190E90901A0EA0901B0EB0901C0EF8010E
:10E7E000C084D184E284F3849401A501B601C701F9
:10E7F0000E949DB0181614F064017501C601D7017E
:10E8000089879A87AB87BC87BE016F5F7F4FCE0138
:10E8100009960E94CB30B8016C5F7F4FAE014B5F11
:10E820005F4FC8010E94AA302C960FB6F894DEBF45
:10E830000FBECDBFDF91CF911F910F91FF90EF9051
:10E84000DF90CF90BF90AF909F908F90089591E010
:10E850009093B7049091C10095FD04C09091C000C1
:10E8600095FD40C02091B5042F5F2F710FB607FCB6
:10E8700034C09091B604291322C09091C00095FF36
:10E880001DC09091B6044091B504491791F0E92F4D
:10E89000F0E0EB56FB4F30819F5F9F713093C600D5
:10E8A0009093B6043091C00030643093C000491397
:10E8B00005C09091C1009F7D9093C100DACFE09197
:10E8C000B504F0E0EB56FB4F80832093B5048091B4
:10E8D000C10080628093C10008959091B60429130D
:10E8E000EECFFBCF8093C6008091C0008064809300
:10E8F000C0000895CF93DF931F921F92CDB7DEB76C
:10E90000789484B5826084BD84B5816084BD85B50A
:10E91000826085BD85B5816085BD80916E00816016
:10E9200080936E00109281008091810082608093BC
:10E9300081008091810081608093810080918000BE
:10E940008160809380008091B10084608093B100E9
:10E950008091B00081608093B000809191008260CE
:10E9600080939100809191008160809391008091CB
:10E9700090008160809390008091A10082608093DC
:10E98000A1008091A10081608093A1008091A000EE
:10E9900081608093A0008091210182608093210199
:10E9A000809121018160809321018091200181600B
:10E9B0008093200180917A00846080937A00809116
:10E9C0007A00826080937A0080917A0081608093DF
:10E9D0007A0080917A00806880937A001092C1005A
:10E9E00082E08093C0001092C50087E08093C4004D
:10E9F0008091C10080618093C1008091C1008860D6
:10EA00008093C1008091C10080688093C100809193
:10EA1000C1008F7D8093C1001092B704EAE3F1E159
:10EA200084918F010F5F1F4F882319F010DFF801C9
:10EA3000F7CFEEEDFEE184918F010F5F1F4F88232A
:10EA400019F005DFF801F7CF14B710FF0CC0E1E3B0
:10EA5000F1E184917F019FEFE91AF90A882319F007
:10EA6000F6DEF701F6CF11FF0CC0E0E2F1E1849190
:10EA70007F019FEFE91AF90A882319F0E8DEF70110
:10EA8000F6CF12FF0CC0EEE0F1E184917F019FEF21
:10EA9000E91AF90A882319F0DADEF701F6CF13FF35
:10EAA0000CC0EDEFF0E184917F019FEFE91AF90AC4
:10EAB000882319F0CCDEF701F6CF15FF0BC0ECEE82
:10EAC000F0E184918F010F5F1F4F882319F0BFDEA3
:10EAD000F801F7CF14BEE5EEF0E184918F010F5FEE
:10EAE0001F4F882319F0B3DEF801F7CF80E2AFDEC5
:10EAF000EEEDF0E184918F010F5F1F4F882319F035
:10EB0000A6DEF801F7CF8AE0A2DEEEEDFEE1849109
:10EB10008F010F5F1F4F882319F099DEF801F7CF9F
:10EB2000EEECF0E184918F010F5F1F4F882319F005
:10EB30008EDEF801F7CFEAEBF0E184918F010F5FF1
:10EB40001F4F882319F083DEF801F7CFE1E8F0E1E9
:10EB500084918F010F5F1F4F882319F078DEF80131
:10EB6000F7CFEEEDFEE184918F010F5F1F4F8823F9
:10EB700019F06DDEF801F7CFEAE6F0E184918F013C
:10EB80000F5F1F4F882319F062DEF801F7CFEEED1B
:10EB9000FEE184918F010F5F1F4F882319F057DE2C
:10EBA000F801F7CF2091C00E3091C10ECE01019631
:10EBB0002115310519F4865C9E4002C0821B930B1F
:10EBC0009A83898369817A818BE590E10E94AD44C3
:10EBD00060E875E084E490E10E94AD448AE037DEAD
:10EBE00081E08093EC048093ED048093EE048093A5
:10EBF000EF048093F0040E949D9C8CE0E0EEF4E032
:10EC0000A1E1BEE001900D928A95E1F70E94B83231
:10EC10006D9A8091010180618093010180910101D1
:10EC20008860809301019D9A8091010180628093A8
:10EC3000010188E00E9478A580910101886080939D
:10EC4000010186E00E9478A587ED80937A001092FA
:10EC50007E0010927D0080917E00816080937E0016
:10EC600080917E00846080937E0080E888BD8091E2
:10EC70006E00846080936E006AEF70E080E090E048
:10EC80000E94AF3885E090E09093BD048093BC046F
:10EC900060E080912D0290912E020E94443E20E07F
:10ECA00030E040EA50E40E9413AA87FF0AC0809136
:10ECB0002D0290912E02409790932E0280932D0268
:10ECC000E7CF81E391E09093300280932F0260E0E0
:10ECD0008091BA049091BB040E94443E20E030E849
:10ECE00048E953E40E949DB0181654F48091BA0488
:10ECF0009091BB0440969093BB048093BA04E7CFF5
:10ED000080912B0290912C020E94C83F20E030E0BD
:10ED100040EA50E40E9413AA87FF0AC080912B02A8
:10ED200090912C02409790932C0280932B02E8CF75
:10ED30008091B8049091B9040E94C83F20E030E06F
:10ED400046E153E40E949DB0181654F48091B80433
:10ED50009091B90440969093B9048093B804E8CF99
:10ED60001092CA041092C6041092C7041092C804EC
:10ED70001092C9041092C2041092C3041092C404E9
:10ED80001092C5041092BE041092BF041092C004E9
:10ED90001092C10482E390E00E94D9AD863119F04F
:10EDA0000E94C93408C040E150E063E370E08CEC9D
:10EDB00094E00E94C9AD81E08093CB0426982E9AFE
:10EDC00025982D9A24982C9A3F98479A0A98129A37
:10EDD0000998119A8093DD048093DC0480910A01E4
:10EDE000886080930A0180910A01806180930A0102
:10EDF00080910A01806280930A010E943BA0809169
:10EE00002101887F816080932101999A989A80914D
:10EE100007018068809307019A9A809107018064B6
:10EE200080930701809107018062809307018091A0
:10EE300007018860809307018091070180618093BA
:10EE4000070128E0E22E23E0F22E10E0F7016191A5
:10EE50007F01812F0E94C99F1F5F1530B9F78091F4
:10EE60000A01826080930A0180910A018160809387
:10EE70000A0180910A01846080930A0180910A014D
:10EE8000806480930A010F9A179A0E9A169A0D9A27
:10EE9000159A0C9A149A389A4098179A8091DE0421
:10EEA0008E7F8093DE04399A4198169A8091DE0411
:10EEB0008D7F8093DE043A9A4298159A8091DE0401
:10EEC0008B7F8093DE043B9A4398149A8091800054
:10EED0008C7F8093800080918100877E8860809302
:10EEE0008100809180008F738093800080918100E9
:10EEF000887F82608093810080E090E49093890015
:10EF000080938800109285001092840080916F0099
:10EF1000826080936F0081E08093DD0478940E948A
:10EF200032841092DF048091010188608093010196
:10EF300098E288E10FB6F894A895809360000FBE20
:10EF40009093600080E6D82E90E0E92E90E0F92EB4
:10EF50008091D406853030F40E944232811102C083
:10EF60000E9429318091D406882309F439C0009188
:10EF7000D306D09E800111240E501B4F8091F104C6
:10EF800080FF17C0EEEDFEE184915F019FEFA91AAB
:10EF9000B90A811102C0580103C059DCF501F4CF50
:10EFA000F50181915F01882311F051DCF9CF8AE0EE
:10EFB0004EDCC8010E946A9D81E00E945910809138
:10EFC000D406882369F081508093D4068091D306BB
:10EFD0008F5F853018F48093D30602C01092D30659
:10EFE0008091100E882309F436C09091100E809104
:10EFF000D206981781F1EEEDFEE184918F010F5F4B
:10F000001F4F882319F023DCF801F7CFEDE4F1E17D
:10F0100084918F010F5F1F4F882319F018DCF801CE
:10F02000F7CF8091100E80FD23C08091100E84FDDB
:10F030001FC08091100E81FD24C08091100E85FDAF
:10F0400020C08091100E82FD25C08091100E86FD9B
:10F0500021C08AE0FCDB8091100E8093D2060E94D2
:10F060008790E114F10409F473CF0E94000070CF7F
:10F0700080E021D9AB01BC0189E491E10E94AF435A
:10F08000D8CF81E018D9AB01BC0185E491E10E94A1
:10F09000AF43D7CF82E00FD9AB01BC0181E491E14E
:10F0A0000E94AF43D6CF8F929F92AF92BF92EF92C2
:10F0B000FF921F93CF93DF93CDB7DEB7A0970FB624
:10F0C000F894DEBF0FBECDBF6115710581059105B6
:10F0D00079F110E0842E912CA12CB12CEE24E39434
:10F0E000F12CEC0EFD1EE10EF11C17FDFA94A501AA
:10F0F00094010E941FAEF7016083B901CA011F5F2E
:10F10000611571058105910549F7115010F1E1E094
:10F11000F0E0EC0FFD1FE10FF11D17FDFA95808166
:10F120008A3010F097E301C090E3890F90DBEDCFB8
:10F1300080E3A0960FB6F894DEBF0FBECDBFDF917F
:10F14000CF911F91FF90EF90BF90AF909F908F90C5
:10F150007ECBA0960FB6F894DEBF0FBECDBFDF9179
:10F16000CF911F91FF90EF90BF90AF909F908F90A5
:10F170000895CF92DF92EF92FF926B017C0197FF8F
:10F180000AC08DE264DBF094E094D094C094C11C7A
:10F19000D11CE11CF11C4AE0C701B601FF90EF90C1
:10F1A000DF90CF9080CF8F929F92AF92BF92CF92FD
:10F1B000DF92EF92FF92CF936B017C01B42E20E09F
:10F1C00030E0A9010E9413AA87FF06C08DE23FDB51
:10F1D000F7FAF094F7F8F094C0E060E070E080E0B7
:10F1E0009FE3CB1541F02DEC3CEC4CEC5DE30E9431
:10F1F00078AACF5FF6CF9B01AC01C701B6010E9490
:10F2000077AE6B017C010E94C0AF4B015C014AE00C
:10F210004ADFCC2379F1C501B4010E9417AA9B01F2
:10F22000AC01C701B6010E9476AE6B017C018EE293
:10F230000EDB20E030E040E251E4C701B6010E945D
:10F2400078AA4B015C010E94BBAF6B01770FEE08FF
:10F25000FF08C701B6018DDFC701B6010E9419AAD8
:10F260009B01AC01C501B4010E9476AE6B017C012B
:10F27000C150F9F6CF91FF90EF90DF90CF90BF9003
:10F28000AF909F908F9008958091930490919404F3
:10F29000891759F0E92FF0E0ED5EFB4F80819F5F09
:10F2A0009F779093940490E008958FEF9FEF0895D7
:10F2B000CF93DF938F389240A1F0ECE4FFE184918B
:10F2C000EF012196882319F0C2DAFE01F8CFECE5B0
:10F2D000F1E18491EF012196882329F0B8DAFE014B
:10F2E000F8CF80E001C081E0DF91CF9108952F92A7
:10F2F0003F924F925F926F927F928F929F92AF92C6
:10F30000BF92CF92DF92EF92FF920F931F93CF9312
:10F31000DF93CDB7DEB7C556D1090FB6F894DEBF7F
:10F320000FBECDBF2DB63EB66B961FAE1EAE6B9711
:10F3300084E690E069969FAF8EAF699701E09E01E9
:10F34000275A3F4F44E050E0BE01655B7F4FCE013E
:10F35000895A9F4F0E94AA9C9E01275A3F4F42E024
:10F3600050E0BE016B5A7F4FCE01895A9F4F0E94D9
:10F37000AA9C43E050E0BE01655B7F4F8DE093E0C7
:10F380000E9480B1892B09F438C02F968FAD2F973A
:10F39000882339F08FE32C968FAF2C972D961FAED4
:10F3A0002D97EEEDFEE184918F010F5F1F4F8823B3
:10F3B00019F04DDAF801F7CFEFE1F2E184918F0116
:10F3C0000F5F1F4F882319F042DAF801F7CFBE0113
:10F3D000655B7F4F86E192E10E94C644E8E0F2E17E
:10F3E00084918F010F5F1F4F882319F030DAF801E5
:10F3F000F7CF81E08093D506E2C42DB73EB7A4963F
:10F400003FAF2EAFA4972B961CAE1DAE1EAE1FAE07
:10F410002B976B961FAE1EAE6B9701E09E01275A8D
:10F420003F4F41E050E0BE01605A7F4FCE01895A04
:10F430009F4F0E94AA9C80E1EDE5F2E0DE019196EB
:10F4400001900D928A95E1F780E1EDE6F2E0DE01B0
:10F45000519601900D928A95E1F780E1EDE7F2E097
:10F460009E012F5F3F4F7901D90101900D928A953E
:10F47000E1F7A1964FADA19750E04D5F5F4F440F6C
:10F48000551F440F551F8DB79EB7841B950B0FB6A4
:10F49000F8949EBF0FBE8DBFEDB7FEB731964F01FA
:10F4A00000E0285A3F4FBF01CE01895A9F4F0E946A
:10F4B000AA9C9E01275A3F4F44E050E06AE67DE057
:10F4C000CE01895A9F4F0E94AA9CA1966FACA1972A
:10F4D000712CF3E06F0E711C660C771C660C771CA8
:10F4E0002DB73EB7261937090FB6F8943EBF0FBEA9
:10F4F0002DBF8DB79EB701965C01EDB7FEB7E6193B
:10F50000F7090FB6F894FEBF0FBEEDBF2DB73EB79B
:10F510002F5F3F4F69019E01275A3F4FA301BC0156
:10F52000CE01895A9F4F0E94AA9C9E01275A3F4FA5
:10F53000A301B601CE01895A9F4F0E94AA9C8091D7
:10F54000280D882309F4A3C000E09E01275A3F4FED
:10F5500044E050E066E77DE0CE01895A9F4F0E946B
:10F56000AA9C9E01275A3F4F44E050E062E77DE0AD
:10F57000CE01895A9F4F0E94AA9C9E01275A3F4F55
:10F5800044E050E06EE67DE0CE01895A9F4F0E9434
:10F59000AA9C9E01275A3F4F44E050E066E67DE07A
:10F5A000CE01895A9F4F0E94AA9C9E01275A3F4F25
:10F5B00044E050E062E67DE0CE01895A9F4F0E9410
:10F5C000AA9C9E01275A3F4F40E150E062E57DE052
:10F5D000CE01895A9F4F0E94AA9C9E01275A3F4FF5
:10F5E00044E050E0BE01695B7F4FCE01895A9F4FD6
:10F5F0000E94AA9C9E01275A3F4F4CE050E060EECB
:10F6000074E0CE01895A9F4F0E94AA9C9E01275AFE
:10F610003F4F44E050E0BE01695B7F4FCE01895A05
:10F620009F4F0E94AA9C9E01275A3F4F44E050E002
:10F63000BE01695B7F4FCE01895A9F4F0E94AA9CF1
:10F6400001E09E01275A3F4F41E050E0BE01615A60
:10F650007F4FCE01895A9F4F0E94AA9C9E01275A34
:10F660003F4F41E050E0BE01625A7F4FCE01895AC0
:10F670009F4F0E94AA9CA0968FADA0976F96EFAC6B
:10F680006F978E9D70011124C12CD12C5FC0A19663
:10F690002FADA19730E02E5F3F4F8AE89DE0A69600
:10F6A0009FAF8EAFA697AAE9BDE06AE77DE080E054
:10F6B00090E040E050E02417350714F0840104C0C6
:10F6C00001E210E00C0F1D1F080F191FF801408008
:10F6D000518062807380FB014192519261927192DC
:10F6E000BF012417350714F0850104C001E110E0C3
:10F6F0000C0F1D1F080F191FF801408051806280F8
:10F7000073804D925D926D927D922417350714F0AF
:10F71000860101C08701080F191FF8014080518040
:10F7200062807380A696EEADFFADA697419251928E
:10F7300061927192A696FFAFEEAFA6974F5F5F4FB3
:10F7400004964430510509F0B6CFFECECE14DF0446
:10F7500091F000E09E01275A3F4F44E050E0BE0187
:10F76000695B7F4FCE01895A9F4F0E94AA9CFFEF91
:10F77000CF1ADF0AEBCF6B96EEACFFAC6B976996B6
:10F780008EAD9FAD6997909332028093310200E075
:10F790009E01275A3F4F44E050E061E27EE0CE01F7
:10F7A000895A9F4F0E94AA9C6B96FFAEEEAE6B9754
:10F7B0009E01275A3F4F44E250E068E37EE0CE01CD
:10F7C000895A9F4F0E94AA9C01E09E01275A3F4FF1
:10F7D00041E050E0BE01635A7F4FCE01895A9F4FEE
:10F7E0000E94AA9C9E01275A3F4F41E050E0BE0173
:10F7F000645A7F4FCE01895A9F4F0E94AA9C00E015
:10F800009E01275A3F4F44E050E0BE01695C7F4FA4
:10F81000CE01895A9F4F0E94AA9C9E01275A3F4FB2
:10F8200044E050E0BE016F5C7F4FCE01895A9F4F8C
:10F830000E94AA9C6E968FAD6E976D96EFAC6D97F9
:10F840008E9D70011124C12CD12C00E09E01275AFD
:10F850003F4FCE14DF0471F044E050E0BE01695B1D
:10F860007F4FCE01895A9F4F0E94AA9C2FEFC21A48
:10F87000D20AEBCF41E050E0BE016F597F4FCE017D
:10F88000895A9F4F0E94AA9C9E01275A3F4F41E0F0
:10F8900050E0BE01655A7F4FCE01895A9F4F0E94AA
:10F8A000AA9C9E01275A3F4F44E050E0BE016D5B89
:10F8B0007F4FCE01895A9F4F0E94AA9C9E01275AD2
:10F8C0003F4F44E050E0BE01615C7F4FCE01895A5A
:10F8D0009F4F0E94AA9C9E01275A3F4F44E050E050
:10F8E000BE01655C7F4FCE01895A9F4F0E94AA9C42
:10F8F00010E000E09E01275A3F4F44E050E0BE0177
:10F90000695B7F4FCE01895A9F4F0E94AA9C1111BB
:10F9100043C02B96CCACDDACEEACFFAC2B9720E01B
:10F9200030E84BE355E4C701B6010E9413AA8823CF
:10F9300099F18091280D811108C0C0924D0DD0928F
:10F940004E0DE0924F0DF092500D00E09E01275AAF
:10F950003F4F44E050E069E47DE0CE01895A9F4F7B
:10F960000E94AA9C9E01275A3F4F44E050E065E464
:10F970007DE0CE01895A9F4F0E94AA9C9E01275A82
:10F980003F4F44E050E0BE01695B7F4FCE01895A92
:10F990009F4F0E94AA9C14C084E0F82EFA94FF2086
:10F9A00079F000E09E01275A3F4F44E050E0BE014D
:10F9B000695B7F4FCE01895A9F4F0E94AA9CEECF70
:10F9C0001F5F153009F095CF00E09E01275A3F4F89
:10F9D00042E050E0BE016D5A7F4FCE01895A9F4FE1
:10F9E0000E94AA9C9E01275A3F4F44E050E0BE016E
:10F9F000695B7F4FCE01895A9F4F0E94AA9C2B962C
:10FA0000CCACDDACEEACFFAC2B9720E030E84BE3A8
:10FA100055E4C701B6010E9413AA882329F18091F9
:10FA2000280D811108C0C092410DD092420DE09284
:10FA3000430DF092440D00E09E01275A3F4F44E0F1
:10FA400050E06DE37DE0CE01895A9F4F0E94AA9C51
:10FA50009E01275A3F4F44E050E069E37DE0CE012C
:10FA6000895A9F4F0E94AA9C00E09E01275A3F4F4F
:10FA700042E050E0BE016F5A7F4FCE01895A9F4F3E
:10FA80000E94AA9C9E01275A3F4F41E050E0BE01D0
:10FA90006F597F4FCE01895A9F4F0E94AA9C19E04F
:10FAA000115000E09E01275A3F4F112359F044E0C6
:10FAB00050E0BE01695B7F4FCE01895A9F4F0E9483
:10FAC000AA9CEECF41E050E06EEA7DE0CE01895A7B
:10FAD0009F4F0E94AA9C00E09E01275A3F4F44E09E
:10FAE00050E0BE01695B7F4FCE01895A9F4F0E9453
:10FAF000AA9C8091280D811110C011110EC02B9667
:10FB00008CAD9DADAEADBFAD2B978093AA0D9093FC
:10FB1000AB0DA093AC0DB093AD0D1F5F1530D9F6B2
:10FB20001CE0115079F000E09E01275A3F4F42E05F
:10FB300050E0BE01615B7F4FCE01895A9F4F0E940A
:10FB4000AA9CEFCF1CE0115000E09E01275A3F4FC6
:10FB5000112359F044E050E0BE01695C7F4FCE01B3
:10FB6000895A9F4F0E94AA9CEECF46E050E0BE010A
:10FB70006F5C7F4FCE01895A9F4F0E94AA9C9E01C5
:10FB8000275A3F4F44E050E065E37DE0CE01895ABB
:10FB90009F4F0E94AA9C13E0115090F034E0139FF5
:10FBA000B0011124675D724F00E09E01275A3F4F5C
:10FBB00044E050E0CE01895A9F4F0E94AA9CECCFAE
:10FBC0001CE1115079F000E09E01275A3F4F44E0BC
:10FBD00050E0BE01695B7F4FCE01895A9F4F0E9462
:10FBE000AA9CEFCF14E0115079F000E09E01275A53
:10FBF0003F4F44E050E0BE01695B7F4FCE01895A20
:10FC00009F4F0E94AA9CEFCF1BE0115079F000E0BB
:10FC10009E01275A3F4F44E050E0BE01695B7F4F91
:10FC2000CE01895A9F4F0E94AA9CEFCF69968EAD54
:10FC30009FAD6997845691093BDB8093D506882355
:10FC400001F1EEEDFEE184918F010F5F1F4F8823DC
:10FC500021F00E942774F801F6CF69966EAD7FAD52
:10FC600069976456710980E092E10E94AD446FE8A3
:10FC700072E088EF91E10E94AD448AE00E9427740F
:10FC80008BC06B962EAD3FAD6B9767968EAD9FADDB
:10FC900067972817390709F444C081E08093D50697
:10FCA000ECE4FFE184918F010F5F1F4F882321F067
:10FCB0000E942774F801F6CFE8EDF1E184918F01FD
:10FCC0000F5F1F4F882321F00E942774F801F6CFA1
:10FCD00067966EAD7FAD679780E090E04AE0E3D92C
:10FCE000E3EDF1E184918F010F5F1F4F882321F035
:10FCF0000E942774F801F6CF6B966EAD7FAD6B97BF
:10FD000080E090E04AE0CFD9E3ECF1E184918F010B
:10FD10000F5F1F4F882309F43FC00E942774F8012A
:10FD2000F5CF8091280D811137C0EEEDFEE1849171
:10FD30008F010F5F1F4F811103C00DE013E004C05E
:10FD40000E942774F801F3CFF80181918F01882375
:10FD500019F00E942774F8CF69966EAD7FAD699750
:10FD60006456710986EA91E10E94AD446B964EADEE
:10FD70005FAD6B9760E070E089E991E10E9492438A
:10FD8000E6E9F1E184918F010F5F1F4F882321F095
:10FD90000E942774F801F6CF8091280D811106C0CA
:10FDA0008091D506811102C00E944DA0A4962EAD6F
:10FDB0003FADA4970FB6F8943EBF0FBE2DBF809104
:10FDC000280D811102C00E94B6969091D50681E05F
:10FDD00089270FB6F8943EBE0FBE2DBECB59DF4F1C
:10FDE0000FB6F894DEBF0FBECDBFDF91CF911F914C
:10FDF0000F91FF90EF90DF90CF90BF90AF909F90CA
:10FE00008F907F906F905F904F903F902F900895CC
:10FE10008F929F92AF92BF92CF92DF92EF92FF921A
:10FE20000F931F93CF93DF93CDB7DEB7CA59D10994
:10FE30000FB6F894DEBF0FBECDBFCB57DF4F188291
:10FE400019821A821B82C558D04085E492E5A2E54A
:10FE5000B0E0CF57DF4F88839983AA83BB83C15813
:10FE6000D040CF56DF4F19821882C159D04084E666
:10FE700090E0C157DF4F99838883CF58D0401092CC
:10FE8000D5069E012F563F4F44E050E0BE016F570C
:10FE90007F4FCE0181579F4F0E94F79CC157DF4F84
:10FEA00088819981CF58D0400296C157DF4F9983FE
:10FEB0008883CF58D040CF56DF4F19821882C1595E
:10FEC000D04081E0C656DF4F8883CA59D0409E019A
:10FED0002F563F4F41E050E0BE0166567F4FCE01A6
:10FEE00081579F4F0E94F79C9E012F563F4F40E144
:10FEF00050E06AE77DE0CE0181579F4F0E94F79C5A
:10FF00009E012F563F4F44E050E06AE67DE0CE016F
:10FF100081579F4F0E94F79C9E012F563F4F40E113
:10FF200050E06AE97DE0CE0181579F4F0E94F79C27
:10FF30009E012F563F4F40E150E06AE87DE0CE0140
:10FF400081579F4F0E94F79C9E012F563F4F44E0E0
:10FF500050E066E77DE0CE0181579F4F0E94F79CFD
:10FF60009E012F563F4F44E050E062E77DE0CE0116
:10FF700081579F4F0E94F79C9E012F563F4F44E0B0
:10FF800050E06EE67DE0CE0181579F4F0E94F79CC6
:10FF90009E012F563F4F44E050E066E67DE0CE01E3
:10FFA00081579F4F0E94F79C9E012F563F4F44E080
:10FFB00050E062E67DE0CE0181579F4F0E94F79CA2
:10FFC0009E012F563F4F40E150E062E57DE0CE01BB
:10FFD00081579F4F0E94F79C8AE097EDA3EABCE30C
:10FFE000CB57DF4F88839983AA83BB83C558D04002
:10FFF0009E012F563F4F44E050E0BE016B577F4FAC
:020000021000EC
:10000000CE0181579F4F0E94F79C9E012F563F4F74
:100010004CE050E060EE74E0CE0181579F4F0E94AB
:10002000F79C80E090E0A0E2B1E4C358DF4F888302
:100030009983AA83BB83CD57D0409E012F563F4F53
:1000400044E050E0BE0163587F4FCE0181579F4F7F
:100050000E94F79CCB57DF4F188219821A821B82AD
:10006000C558D04083E0C756DF4F8883C959D04078
:10007000C856DF4F8883C859D0409E012F563F4F46
:1000800044E050E0BE016B577F4FCE0181579F4F38
:100090000E94F79C9E012F563F4F41E050E0BE0169
:1000A00067567F4FCE0181579F4F0E94F79C9E015C
:1000B0002F563F4F41E050E0BE0168567F4FCE01C2
:1000C00081579F4F0E94F79C1AE0115071F09E01DA
:1000D0002F563F4F44E050E0BE016B577F4FCE019B
:1000E00081579F4F0E94F79CF0CFCF56DF4F08817A
:1000F0001981C159D040C157DF4F88819981CF58AC
:10010000D04090933202809331029E012F563F4F90
:1001100044E050E061E27EE0CE0181579F4F0E94B3
:10012000F79CCF56DF4F19830883C159D0409E01F9
:100130002F563F4F44E250E068E37EE0CE01815706
:100140009F4F0E94F79C83E0C956DF4F8883C759B1
:10015000D040CA56DF4F8883C659D040ED961CAEBA
:100160001DAE1EAE1FAEED97E9961CAE1DAE1EAEC7
:100170001FAEE997CB57DF4F188219821A821B8274
:10018000C558D0409E012F563F4F41E050E0BE0180
:1001900069567F4FCE0181579F4F0E94F79C9E0169
:1001A0002F563F4F41E050E0BE016A567F4FCE01CF
:1001B00081579F4F0E94F79C9E012F563F4F44E06E
:1001C00050E0BE016B587F4FCE0181579F4F0E9478
:1001D000F79C9E012F563F4F44E050E0BE01675808
:1001E0007F4FCE0181579F4F0E94F79C0AE010E09D
:1001F0000150110971F09E012F563F4F44E050E02D
:10020000BE016B577F4FCE0181579F4F0E94F79CD5
:10021000EFCFCB56DF4F1882C559D0408FEFCC5669
:10022000DF4F8883C459D0409E012F563F4F41E095
:1002300050E0BE016B567F4FCE0181579F4F0E9409
:10024000F79C9E012F563F4F41E050E0BE016C5697
:100250007F4FCE0181579F4F0E94F79C88EC90E022
:10026000E3969FAF8EAFE39780EF90E0E5969FAF68
:100270008EAFE59786E490E0AF969FAF8EAFAF97D5
:100280008EE690E0E1969FAF8EAFE197AB961FAE02
:100290001EAEAB97AD961FAE1EAEAD979E012F560C
:1002A0003F4F44E050E0BE016F587F4FCE01815771
:1002B0009F4F0E94F79C9E012F563F4F44E050E015
:1002C000BE0163597F4FCE0181579F4F0E94F79C1B
:1002D0009E012F563F4F44E050E0BE0167597F4FCB
:1002E000CE0181579F4F0E94F79C10E0C12C80E8FF
:1002F000D82E8BE3E82E85E4F82E812C912C90E803
:10030000A92E9FE3B92E11113AC09E012F563F4FDF
:1003100044E050E06DE47DE0CE0181579F4F0E94A4
:10032000F79C9E012F563F4F44E050E069E47DE08A
:10033000CE0181579F4F0E94F79C9E012F563F4F41
:1003400044E050E065E47DE0CE0181579F4F0E947C
:10035000F79CCB57DF4F88829982AA82BB82C5580F
:10036000D0409E012F563F4F44E050E0BE016B57F6
:100370007F4FCE0181579F4F0E94F79C2EC0CB57D5
:10038000DF4FC882D982EA82FB82C558D0409E01E5
:100390002F563F4F44E050E0BE016B577F4FCE01D8
:1003A00081579F4F0E94F79CCB57DF4F18821982CD
:1003B0001A821B82C558D04004E0015071F09E01A2
:1003C0002F563F4F44E050E0BE016B577F4FCE01A8
:1003D00081579F4F0E94F79CF0CF1F5F153009F0A7
:1003E00092CF84E190E0C357DF4F99838883CD5843
:1003F000D0409E012F563F4F42E050E0BE01635770
:100400007F4FCE0181579F4F0E94F79C9E012F5630
:100410003F4F44E050E061E47DE0CE0181579F4FC3
:100420000E94F79C9E012F563F4F44E050E06DE341
:100430007DE0CE0181579F4F0E94F79C9E012F5671
:100440003F4F44E050E069E37DE0CE0181579F4F8C
:100450000E94F79C80E290E0C557DF4F9983888324
:10046000CB58D0409E012F563F4F42E050E0BE0196
:1004700065577F4FCE0181579F4F0E94F79CCD5605
:10048000DF4F1882C359D04080E2EDE8F2E0DE0190
:100490009D9601900D928A95E1F79E012F563F4F50
:1004A00041E050E0BE016D567F4FCE0181579F4F16
:1004B0000E94F79C9E012F563F4F40E250E0BE0144
:1004C000635D7F4FCE0181579F4F0E94F79C9E0135
:1004D0002F563F4F41E050E06EEA7DE0CE0181575C
:1004E0009F4F0E94F79C10E0111110C08091AA0D3F
:1004F0009091AB0DA091AC0DB091AD0DCB57DF4FEE
:1005000088839983AA83BB83C558D0409E012F5608
:100510003F4F44E050E0BE016B577F4FCE01815703
:100520009F4F0E94F79C1F5F1530F1F6BE01635B81
:100530007F4F86E1FB0111928A95E9F79E012F56C4
:100540003F4F46E150E0CE0181579F4F0E94F79CFC
:100550008CE2EDEAF2E0DE01119601900D928A95AF
:10056000E1F79E012F563F4F4CE250E0BE016F5F16
:100570007F4FCE0181579F4F0E94F79CBE016D595E
:100580007F4F86E0FB0111928A95E9F79E012F5675
:100590003F4F46E050E0CE0181579F4F0E94F79CAD
:1005A0009E012F563F4F44E050E065E37DE0CE01D1
:1005B00081579F4F0E94F79C13E0115088F0F4E0A0
:1005C0001F9FB0011124675D724F9E012F563F4F50
:1005D00044E050E0CE0181579F4F0E94F79CEDCF41
:1005E000CB57DF4F188219821A821B82C558D04020
:1005F0001CE1115071F09E012F563F4F44E050E036
:10060000BE016B577F4FCE0181579F4F0E94F79CD1
:10061000F0CFCB57DF4F188219821A821B82C55840
:10062000D04014E0115071F09E012F563F4F44E02E
:1006300050E0BE016B577F4FCE0181579F4F0E9404
:10064000F79CF0CFCB57DF4F188219821A821B829A
:10065000C558D0401BE0115071F09E012F563F4FFE
:1006600044E050E0BE016B577F4FCE0181579F4F52
:100670000E94F79CF0CF8091D506811167C0C157C9
:10068000DF4FE880F980CF58D04084E6E81AF108BF
:10069000CF56DF4F88819981C159D040C757DF4F6E
:1006A00099838883C958D04084E690E0C157DF4FD2
:1006B00099838883CF58D0409E012F563F4F44E006
:1006C00050E06DE073E0CE0181579F4F0E94F79C90
:1006D0009E012F563F4F42E050E0BE0167577F4FCB
:1006E000CE0181579F4F0E94F79CEEEDFEE1849171
:1006F0008F010F5F1F4F882321F00E942774F8019C
:10070000F6CFB70184E891E10E94AD44C757DF4FAF
:1007100048815981C958D04060E070E087E791E195
:100720000E949243E4E7F1E184918F010F5F1F4F34
:10073000882321F00E942774F801F6CFC7010E9498
:1007400058799091D506892B8093D5069091D5063E
:1007500081E08927C656DF4F0FB6F894DEBF0FBE83
:10076000CDBFDF91CF911F910F91FF90EF90DF9060
:10077000CF90BF90AF909F908F9008958091360E4C
:100780009091370E891B8F7019F480E090E00895E6
:100790009091330E992351F0833030F48FEF890F0D
:1007A00019F08093330EF1CF1092330EE091370E93
:1007B00088E5E89FF0011124E650F94F808180FD23
:1007C000E4CF8091370E8F5F8F708093340E9091BD
:1007D000370E8091350E981304C08091340E8093AB
:1007E000350ECF0108950F930FB70F9300916E0050
:1007F0000F930B7F00936E0000916F000D7F0093AD
:100800006F000F930BB70F930CB70F921F922F939C
:100810003F934F935F936F937F938F939F93AF9388
:10082000BF93EF93FF9311245DD0FF91EF91BF91A0
:10083000AF919F918F917F916F915F914F913F9178
:100840002F911F900F900CBF0F910BBF0F91026063
:10085000F89400936F000F9100936E000F910FBFFB
:100860000F9118958091800C80FF07C080910B013B
:100870008270809309018FEF07C080910B018095F2
:1008800082708093090181E080937A0C8091800CC2
:1008900081FF08C080910B018095817080930901D0
:1008A0008FEF06C080910B0181708093090181E078
:1008B00080937B0C8091800C82FF07C080910B019C
:1008C0008470809309018FEF07C080910B018095A0
:1008D00084708093090181E080937C0C000000000B
:1008E000000008952F923F924F925F926F927F92F5
:1008F0008F929F92AF92BF92CF92DF92EF92FF9230
:100900000F931F93CF93DF9300D000D0CDB7DEB706
:10091000F8948FEF9FEF90938900809388002AE0EE
:100920002E83212C312C78948091CA0C9091CB0C81
:10093000A091CC0CB091CD0C892B8A2B8B2B09F07C
:10094000CDC18091AF0D8823D1F01092AF0D809171
:10095000B50D9091B60D892B91F01092C10C1092AB
:10096000B60D1092B50D9091360E8091370E9817F6
:1009700031F08091370E8F5F8F708093370E8091AA
:10098000B50D9091B60D892B09F4A8C14091C60C04
:100990005091C70C6091C80C7091C90C9091B40C27
:1009A0000091C20C1091C30C2091C40C3091C50C65
:1009B000041B150B260B370B892F90E0A0E0B0E04D
:1009C000081719072A073B0710F4D901C801E82FB7
:1009D000840F951FA61FB71F8093C60C9093C70C5A
:1009E000A093C80CB093C90C20918400309185006D
:1009F000225E3F4F40919A0C50919B0C60919C0C51
:100A000070919D0C80918A0C90918B0CA0918C0C14
:100A1000B0918D0C840F951FA61FB71F80939A0C61
:100A200090939B0CA0939C0CB0939D0CB7FD1CC0A5
:100A3000409A4091C30D5091C40D6091C50D7091C5
:100A4000C60D80917A0C082E000C990BAA0BBB0BDB
:100A5000840F951FA61FB71F8093C30D9093C40DDD
:100A6000A093C50DB093C60D40919E0C50919F0C64
:100A70006091A00C7091A10C80918E0C90918F0CC4
:100A8000A091900CB091910C840F951FA61FB71FD9
:100A900080939E0C90939F0CA093A00CB093A10CFC
:100AA000B7FD1CC0419A4091C70D5091C80D60918F
:100AB000C90D7091CA0D80917B0C082E000C990B0A
:100AC000AA0BBB0B840F951FA61FB71F8093C70DE2
:100AD0009093C80DA093C90DB093CA0D4091A20C7C
:100AE0005091A30C6091A40C7091A50C8091920C74
:100AF0009091930CA091940CB091950C840F951F3C
:100B0000A61FB71F8093A20C9093A30CA093A40CD4
:100B1000B093A50CB7FD1CC0429A4091CB0D5091EB
:100B2000CC0D6091CD0D7091CE0D80917C0C082E76
:100B3000000C990BAA0BBB0B840F951FA61FB71FA8
:100B40008093CB0D9093CC0DA093CD0DB093CE0D93
:100B50004091A60C5091A70C6091A80C7091A90C23
:100B60008091960C9091970CA091980CB091990C53
:100B7000840F951FA61FB71F8093A60C9093A70CF8
:100B8000A093A80CB093A90CB7FD3AC0C090CF0DAC
:100B9000D090D00DE090D10DF090D20D40917D0C11
:100BA000042E000C550B660B770B4C0D5D1D6E1D56
:100BB0007F1D4093CF0D5093D00D6093D10D709356
:100BC000D20D4091860C5091870C6091880C7091E9
:100BD000890C841B950BA60BB70B8093A60C9093E6
:100BE000A70CA093A80CB093A90C9091800C8091B5
:100BF000B20C93FF02C0815001C08F5F8093B20C92
:100C0000809184009091850082179307C8F38091AA
:100C10009A0C90919B0CA0919C0CB0919D0CB7FDEF
:100C200015C04091860C5091870C6091880C709192
:100C3000890C841B950BA60BB70B80939A0C909391
:100C40009B0CA0939C0CB0939D0C409880919E0CA3
:100C500090919F0CA091A00CB091A10CB7FD15C074
:100C60004091860C5091870C6091880C7091890C92
:100C7000841B950BA60BB70B80939E0C90939F0C37
:100C8000A093A00CB093A10C41988091A20C9091DC
:100C9000A30CA091A40CB091A50CB7FD15C0409178
:100CA000860C5091870C6091880C7091890C841B84
:100CB000950BA60BB70B8093A20C9093A30CA0935B
:100CC000A40CB093A50C4298E15041F080918400AF
:100CD0009091850082179307C8F38ACE80913C02D9
:100CE00090913D02A0913E02B0913F02892B8A2B48
:100CF0008B2B09F09AC08091B30C882309F455C05E
:100D0000C090C60CD090C70CE090C80CF090C90CF5
:100D10004091AE0C5091AF0C6091B00C7091B10C41
:100D20008091B20C4C155D056E057F0588F420910D
:100D30007E0C30917F0CE091830CF091840CE217D3
:100D4000F30730F481508093B20C2150310915C063
:100D5000C416D506E606F706E8F420917E0C30911D
:100D60007F0C4091810C5091820C2417350790F430
:100D70008F5F8093B20C2F5F3F4F30937F0C209397
:100D80007E0C409138025091390260913A02709184
:100D90003B020EC08FEF9FEFDC01809338029093EF
:100DA0003902A0933A02B0933B024FEF5FEFBA01D2
:100DB0008091B20C87FD03C080910B0103C080912C
:100DC0000B018095807480930901209184003091FB
:100DD0008500225E3F4F8091B20C8823F1F0439A48
:100DE000809184009091850082179307C8F38091C9
:100DF000B20C87FF02C08F5F01C081508093B20C9C
:100E000043988091B20C882331F3809184009091B3
:100E1000850082179307C8F3DCCF40933C025093C0
:100E20003D0260933E0270933F028091CA0C909104
:100E3000CB0CA091CC0CB091CD0C892B8A2B8B2B99
:100E400009F063C3A091B50DB091B60D109739F1BB
:100E5000C090C60CD090C70CE090C80CF090C90CA4
:100E60004091C20C5091C30C6091C40C7091C50CA0
:100E7000C416D506E606F706C8F01092C10C10920B
:100E8000B60D1092B50D9091360E8091370E9817D1
:100E900031F08091370E8F5F8F708093370EA0ED09
:100EA0008A2EA7E09A2EA12CB12C81C14091BD0CB5
:100EB0005091BE0C6091BF0C7091C00C4C155D053B
:100EC0006E057F0508F46EC04091B90C5091BA0CC4
:100ED0006091BB0C7091BC0CD2960D911D912D911F
:100EE0003C91D597EE27419FF12D529FC001629F03
:100EF000900D619F800D911D429FF00D811D9E1FE1
:100F0000519FF00D811D9E1F609FF00D811D9E1F42
:100F1000509FF10D8E1F9E1FF6958E1F9E1F349FB2
:100F2000800D911D359F900D1124FD01EA5BFF4F4F
:100F30000081118122813381080F191F211D311D6C
:100F40000093B50C1093B60C2093B70C3093B80CEB
:100F5000349780809180A280B38080169106A2068B
:100F6000B30640F48092B50C9092B60CA092B70CE8
:100F7000B092B80C8090B50C9090B60CA090B70CC5
:100F8000B090B80C88E39AE177247394FC01059142
:100F9000159125913491081519052A053B0508F48A
:100FA0002EC338C32091AE0C3091AF0C4091B00CE1
:100FB0005091B10C29833A834B835C832C153D05FA
:100FC0004E055F0508F068C04091AA0C5091AB0C2B
:100FD0006091AC0C7091AD0CD2960D911D912D913C
:100FE0003C91D597EE27419FF12D529FC001629F02
:100FF000900D619F800D911D429FF00D811D9E1FE0
:10100000519FF00D811D9E1F609FF00D811D9E1F41
:10101000509FF10D8E1F9E1FF6958E1F9E1F349FB1
:10102000800D911D359F900D11248C0120E030E042
:101030004090B50C5090B60C6090B70C7090B80C06
:10104000FD01E65BFF4F041515052605370580F405
:1010500080809180A280B380401A510A620A730A8C
:10106000481459046A047B0438F42401350104C08F
:10107000408051806280738088E39AE131E03D8353
:10108000FC0105911591259134910415150526054E
:10109000370508F43CC348C38091B20C8823D9F0CB
:1010A000D8964D915C91D99760E070E0009138023C
:1010B0001091390220913A0230913B020417150732
:1010C0002607370741F010923C0210923D02109221
:1010D0003E0210923F0240913402509135026091DD
:1010E00036027091370277FF5AC0AE5BBF4F8D91C9
:1010F0009D910D90BC91A02D28E33AE141E0F901CA
:10110000C590D590E590F490C816D906EA06FB067E
:1011100058F4B695A79597958795440F2C5F3F4F48
:101120005AE12435350759F74093B40C80329105C4
:10113000A105B10508F4E7C38097A109B10981159C
:10114000E8E09E07A105B10508F4B8C324E0929F2A
:10115000F00111249F01285C394EF9013296459126
:101160005491EE27859FB001849F610D7E1F0694E8
:101170006E1F7E1F1124AB0160E070E0F9018591C4
:101180009491A0E0B0E0841B950BA60BB70B809365
:10119000340290933502A0933602B09337028090C8
:1011A000340290903502A0903602B09037028091C0
:1011B000B50D9091B60D892B09F09FC1DFDA9093A0
:1011C000B60D8093B50D892B09F497C1E091B50D4B
:1011D000F091B60D808183FF3EC085899689A789ED
:1011E000B08D8093C30D9093C40DA093C50DB093A3
:1011F000C60D818D928DA38DB48D8093C70D909374
:10120000C80DA093C90DB093CA0D858D968DA78D7D
:10121000B0A18093CB0D9093CC0DA093CD0DB09346
:10122000CE0D81A192A1A3A1B4A18093CF0D9093E3
:10123000D00DA093D10DB093D20D9091360E809128
:10124000370E981709F4BACF8091370E8F5F8F70E1
:101250008093370EB3CFC588D688E788F08C81E0BD
:10126000C114D104E104F10409F480E0018D128D70
:10127000238D348D011511052105310509F082609A
:10128000458D568D678D70A141155105610571051C
:1012900009F084608093C10C1092AA0C1092AB0CE0
:1012A0001092AC0C1092AD0C1092B90C1092BA0CBA
:1012B0001092BB0C1092BC0C85A196A1A7A1B0A561
:1012C0008093C20C9093C30CA093C40CB093C50C34
:1012D000882499245401881A990AAA0ABB0A809280
:1012E000A60C9092A70CA092A80CB092A90C809288
:1012F000A20C9092A30CA092A40CB092A50C809288
:101300009E0C90929F0CA092A00CB092A10C809287
:101310009A0C90929B0CA0929C0CB0929D0CCC0CC1
:10132000DD1CEE1CFF1CC0928A0CD0928B0CE0924C
:101330008C0CF0928D0C000F111F221F331F009395
:101340008E0C10938F0C2093900C3093910C440FC3
:10135000551F661F771F4093920C5093930C609318
:10136000940C7093950C41A152A163A174A1440FF8
:10137000551F661F771F4093960C5093970C6093F0
:10138000980C7093990C880F991FAA1FBB1F80930C
:10139000860C9093870CA093880CB093890C1092C4
:1013A000C60C1092C70C1092C80C1092C90C82A5E2
:1013B00093A5A4A5B5A58093BD0C9093BE0CA09356
:1013C000BF0CB093C00C86A597A5A0A9B1A9809326
:1013D000AE0C9093AF0CA093B00CB093B10C81A560
:1013E0008093850C97A99093B30C992361F024AD59
:1013F00035AD3093840C2093830C22AD33AD309304
:10140000820C2093810C96A92091800C92130AC023
:101410002091330230E0482F082E000C550B421764
:10142000530729F09093800C809333021BDA0E94BB
:1014300005348FEF9FEFDC018093340290933502E7
:10144000A0933602B0933702E091B50DF091B60D3E
:10145000EA5BFF4F80819181A281B3818093B50CBB
:101460009093B60CA093B70CB093B80C28E33AE174
:1014700041E0F901C590D590E590F490C816D906E1
:10148000EA06FB0658F4B695A79597958795440FFD
:101490002C5F3F4FEAE124353E0759F74093B40CE7
:1014A00080329105A105B10508F455C28097A109C4
:1014B000B1098115E8E09E07A105B10508F428C22D
:1014C000F4E09F9F90011124285C394EF901329677
:1014D00045915491EE27859FB001849F610D7E1F39
:1014E00006946E1F7E1F1124F90185909490A12C03
:1014F000B12C861A970AA108B1088092CA0C909262
:10150000CB0CA092CC0CB092CD0C0091CA0C1091D7
:10151000CB0C2091CC0C3091CD0C40913C025091E1
:101520003D0260913E0270913F02F02EE12EF22FBB
:10153000E32F401751076207730720F4F42EE52EBE
:10154000F62FE72F8F2D9E2DAF2FBE2F0097E1E0B6
:10155000AE07B10520F08FEF9FEFA0E0B0E0081BD1
:10156000190B2A0B3B0B0093CA0C1093CB0C209346
:10157000CC0C3093CD0C4F3FFFEF5F076F077F0719
:1015800061F0481B590B6A0B7B0B40933C02509354
:101590003D0260933E0270933F02F89420918400D4
:1015A00030918500205F3F4F4E8141504E83442350
:1015B00039F0280E391E2216330608F4B4C901C0CA
:1015C00019013092890020928800789426960FB6EF
:1015D000F894DEBF0FBECDBFDF91CF911F910F9169
:1015E000FF90EF90DF90CF90BF90AF909F908F9043
:1015F0007F906F905F904F903F902F900895B6949A
:10160000A79497948794770C0496EAE184359E0713
:1016100009F0BCCC7092B40C80E288169104A1044D
:10162000B10408F41CC190E2891A9108A108B1081C
:101630008114E8E09E06A104B104F8F0F4E09F9E56
:10164000C0011124885C994EFC0132962591349199
:10165000F82DEE27F39F8001F29F010D1E1F0694C7
:101660000E1F1E1F1124FC0185909490A12CB12CFB
:10167000801A910AA108B10823C09501840136950A
:10168000279517950795F801EC7F9F01285C3D4E43
:10169000F90185919491F901329605911491E82D03
:1016A000E770E09F9001E19F300D1124F3E0369543
:1016B0002795FA95E1F74C01821A930AA12CB12CD7
:1016C000480D591D6A1D7B1D4093B90C5093BA0CEF
:1016D0006093BB0C7093BC0C8091B30C882359F0C1
:1016E000472D50E060E070E0C416D506E606F70628
:1016F00009F06CC084C02FEF3FEFA901209338029E
:101700003093390240933A0250933B029AC0769448
:101710006794579447942D81220F2D8304963AE1C4
:101720008435930709F0ACCC2D812093B40C30E2C2
:10173000431651046104710408F4BAC080E2481AE7
:10174000510861087108411498E059066104710458
:1017500008F48BC0E4E05E9EC0011124885C994EC1
:10176000FC01329605911491F42DEE27F19F900122
:10177000F09F210D3E1F06942E1F3E1F1124FC01D9
:1017800085909490A12CB12C821A930AA108B108DB
:10179000480D591D6A1D7B1D4093AA0C5093AB0C3C
:1017A0006093AC0C7093AD0C8091B30C8823F1F175
:1017B00049815A816B817C812D81420F511D611DB0
:1017C000711D4C155D056E057F05C8F48091B20C46
:1017D000882309F4ECCCD8964D915C91D99760E0C0
:1017E00070E0009138021091390220913A02309154
:1017F0003B02041715072607370709F4D8CC1092C7
:101800003C0210923D0210923E0210923F02D89686
:101810008D919C91D997A0E0B0E08093380290938D
:101820003902A0933A02B0933B02C1CC8FEF9FEFF5
:10183000DC018093380290933902A0933A02B0936E
:101840003B028091B20C882309F4B1CC10923C0287
:1018500010923D0210923E0210923F02A8CC00E28C
:10186000802E912CA12CB12CDECE930182013695D5
:10187000279517950795F801EC7FCF01885C9D4E61
:10188000FC0185909490FC01329625913491E42DD1
:10189000E770E29FC001E39F900D112423E096952D
:1018A00087952A95E1F7881A990AA12CB12C70CF57
:1018B000F0E24F2E512C612C712C40CFAC01BD01B8
:1018C0007695679557954795FA01EC7FAF01485C8F
:1018D0005D4EFA0125913491FA0132964591549169
:1018E0008770849FB001859F700D1124CB01F3E0B8
:1018F00096958795FA95E1F7A901481B590BCA01FE
:10190000A0E0B0E044CC80E290E0A0E0B0E014CCF5
:10191000AC01BD017695679557954795FA01EC7F27
:101920009F01285C3D4EF90185909490F901329613
:10193000259134918770829FA001839F500D1124BF
:10194000CA0123E0969587952A95E1F7881A990AA6
:10195000A12CB12CD2CD80E290E0A0E0B0E0A6CDE9
:101960008F929F92AF92BF92CF92DF92EF92FF92AF
:101970000F931F93CF93DF9300D01F92CDB7DEB7A5
:101980008AE7882E8DE0982E9AE9A92E9DE0B92E3F
:101990000AED16E0C12CD12C7601C394F4016191BB
:1019A0007191819191914F01F50121913191419175
:1019B00051915F0129833A834B835C830E9417AA6C
:1019C00029813A814B815C810E9478AA0E94C0AF34
:1019D000F80161937193819391938F01C616D70695
:1019E000E806F90610F46B017C01FAE88F16FDE0B9
:1019F0009F06A1F66FEF7FEFCB01A70196010E9432
:101A00001FAE2093D6063093D7064093D806509346
:101A1000D9060F900F900F900F90DF91CF911F91EB
:101A20000F91FF90EF90DF90CF90BF90AF909F907D
:101A30008F9008958F929F92AF92BF92EF92FF92F4
:101A40000F931F93CF93DF937B018A01E901FC0180
:101A500080809180A280B38020919A0D30919B0D5F
:101A600040919C0D50919D0DC501B4010E9478AA32
:101A70000E94A8B06093800E7093810E8093820EB6
:101A80009093830E20919E0D30919F0D4091A00D5B
:101A90005091A10DF70160817181828193810E9433
:101AA00078AA0E94A8B06093840E7093850E8093EC
:101AB000860E9093870E2091A20D3091A30D409138
:101AC000A40D5091A50DF8016081718182819381EF
:101AD0000E9478AA0E94A8B06093880E7093890E25
:101AE00080938A0E90938B0E2091A60D3091A70DB6
:101AF0004091A80D5091A90D688179818A819B81BF
:101B00000E9478AA0E94A8B060938C0E70938D0EEC
:101B100080938E0E90938F0E8092700E9092710E25
:101B2000A092720EB092730EF70180819181A28112
:101B3000B3818093740E9093750EA093760EB0933C
:101B4000770EF80180819181A281B3818093780E14
:101B50009093790EA0937A0EB0937B0E8881998131
:101B6000AA81BB8180937C0E90937D0EA0937E0E04
:101B7000B0937F0E9091360E8091370E981761F0DA
:101B8000DF91CF911F910F91FF90EF90BF90AF9099
:101B90009F908F900C94DC700E943A7180916F003E
:101BA00081FB992790F981FF05C080916F008D7F9F
:101BB00080936F004091800E5091810E6091820E53
:101BC0007091830E4093C30D5093C40D6093C50D67
:101BD0007093C60D4091840E5091850E6091860ED3
:101BE0007091870E4093C70D5093C80D6093C90D37
:101BF0007093CA0D4091880E5091890E60918A0EA3
:101C000070918B0E4093CB0D5093CC0D6093CD0D06
